:020000040800F2
:1000000000000120396C0508D56C0508DDB1010838
:1000100031B00108D56C0508D56C0508000000005A
:10002000000000000000000000000000D56C050882
:10003000D56C050800000000D56C05087DCB0008D4
:10004000D56C0508D56C0508D56C0508D56C050878
:10005000D56C0508D56C05080DA0000815A0000892
:100060001DA0000825A000082DA00008059E00087E
:10007000199E00082D9E0008419E0008559E00080C
:10008000699E00087D9E0008D56C0508D56C0508A2
:10009000D56C0508D56C0508D56C050835A0000899
:1000A000CDC20008C9C10008DDC20008B9C10008FE
:1000B000F1C1000801C2000811C20008259A000819
:1000C000199A0008599A00084D9A0008D56C05083D
:1000D000D56C05080DA8040819A8040825A804086B
:1000E0003DA00008D56C0508D56C0508EDC20008D8
:1000F000A5C20008D56C050895C20008919E0008AD
:10010000D56C0508D56C050821C20008D56C05081A
:1001100031A804083DA8040831C20008D1EC040845
:10012000A59E0008B99E0008CD9E0008E19E00082B
:10013000F59E000800000000000000000000000024
:1001400000000000000000000000000041E2040880
:10015000099F00081D9F0008319F000849A8040856
:100160008D9A0008819A0008D56C0508D56C0508A1
:10017000D56C0508D56C05080000000000000000E3
:10018000D56C0508D56C0508D56C0508D56C050837
:10019000D56C0508D56C050800000000D56C050875
:1001A000000000000000000000000000D56C050801
:1001B000D56C0508D56C05080000000000000000A3
:1001C000000000000000000000000000000000002F
:1001D000000000000000000000000000D56C0508D1
:10800000084A0346D0F8EC005268D3F8F810121A68
:1080100000209142B8BFC3F8F820012283F8242140
:10802000704700BF001000E030B4046900234168CD
:108030004025E46882690C3154624469956053605C
:1080400093631160C2E90333C2E90533C2E9073320
:10805000C2E90A33C2E90C3394B1C2694FF48030EB
:10806000E468116054629062C2E90133C2E90333EB
:10807000C2E90533C2E90733C2E90B33C2E90D3364
:1080800030BC7047114A037A0168D35C10B4CC58F5
:10809000CA1824F00104CC501368DB07FCD4037D1C
:1080A0001F2B09D9203B20225DF8044B02FA03F371
:1080B00043F01803CB60704720225DF8044B02FAAE
:1080C00003F343F018038B60704700BF900F06085E
:1080D0001B4B016803F57D7C02E02C3363452BD0FC
:1080E0001A688A42F9D170B593F804E0427996454E
:1080F0000BD02C33634505D01A688A42F4D02C3358
:108100006345F9D14FF0FF3070BD9E468468002270
:10811000DEF80C50A54208D001320EF10C0E032AF5
:10812000E7D0DEF80C50A542F6D1DEF81050C66854
:10813000B542F1D150B270BD4FF0FF30704700BF73
:10814000688B05084368426D30B49A61EFF3118281
:10815000502383F312884168D2B2856C0B68046D9A
:1081600023EA050323430B6082F311884369816886
:108170001A68096822F00102D0E908541A60826A7C
:108180001D605C615A60D0E90B429C60DA6000239C
:10819000B0F86C2030BCCA6203777047002A4FEAFF
:1081A000014C034630B508BFE64600F1C00514BFD8
:1081B0008E468C46002419680C3353F8042C43F87F
:1081C000084C41EA0C0142EA0E02AB4243F80C1C97
:1081D00043F8042CEFD1D0F8C03043EA0E03C0E9D5
:1081E0003144C0F8C03030BD83695969B3F810C05C
:1081F0000A6830B49C6822F0010224680A60E268D0
:1082000022EA0C02E260027D00681F2A06D9203AA9
:108210000824456894402C4242D0FEE708240568B3
:1082200094402C42F9D1202404FA02F28260254ABB
:108230001278002A32D01A7F012A36D0D3F80021D2
:108240000132C3F80021EFF31181502282F312882A
:108250005868C9B29D6C0268DC6C22EA05022243B0
:10826000026081F311885A699968D3E90D40096861
:1082700014605061D3E90F40546090605C6CB3F8B7
:10828000B400D4600124C8621068204310601A8AC8
:108290001C7783F8FD40CB681343CB6030BC70473C
:1082A000202404FA02F2C260C1E70022D3F80401DC
:1082B00083F8FD2001300A68C3F8040122F00102AE
:1082C0000A60EBE7A801002010B40C4C6368002B97
:1082D00011DD002004F1080C0146DCF8AC3003F19C
:1082E000C00259600C339342FBD1013063680CF536
:1082F000867C8342F1DC5DF8044B7047A8010020C6
:10830000704700BF024B03EB401393F855047047CE
:10831000A8010020D0E90920131A5842584170479B
:1083200090F8573830B53BB990F85518012490F8BB
:108330005638DAB2914200D830BD04FA03F2B0F8F0
:108340005E5801332A43A0F85E28F2E7037902461B
:1083500013F0010006D0D2E90731D2685B1A013A66
:1083600003EA0200704710B50379044613F00103D5
:108370000ED0FFF7EBFF034650B1226A6369E16854
:108380009B5C0132B2FBF1F0DBB201FB10222262F6
:10839000184610BD03799B070AD5436A8269D154F8
:1083A000436A02690133B3FBF2F102FB113343620A
:1083B00070477047017170470379014613F002005E
:1083C00007D00B69D1E90921013B521A1A40D2B2F8
:1083D000981A704710B584464FEA810E102312F4A4
:1083E000004F4FEA420214BF0E240724013B92B211
:1083F000CCF80040F444F2D100EB81128C0103511F
:10840000122042F8213010BD10B584464FEA810E8B
:108410000424130B013C4FEA021203EB430392B214
:1084200003F11803CCF80030F444F2D100EB01134F
:108430000A018450062043F8214010BD704700BF58
:10844000704700BF00EB4000024B03EBC00393F802
:1084500049057047A8010020064B93F8F825824291
:1084600006D900EB400003EBC003D3F84C0570477E
:1084700000207047A80100200B4890F8FC1589B136
:1084800001EB4101002300F5A760490010B41C4630
:1084900050F82320063302B114608B42F8D15DF806
:1084A000044B7047704700BFA80100200B4890F8AC
:1084B000FC1589B101EB4101002300F5A7604900DB
:1084C00010B41C4650F82320063302B114608B42CE
:1084D000F8D15DF8044B7047704700BFA801002039
:1084E000214B1B78002B3DD12DE9F0431F4C94F814
:1084F000FC25AAB304F5A7624FF0500E1C4F4FF0B5
:108500002C0C1C4E1D4607E0013394F8FC1552F864
:10851000180B8B42056023DA117C0029F4D05068D7
:108520004FF0FE08810AA1F580115229314498BF0D
:1085300091F8F483EFF311818EF31288D0F8249030
:108540000CFB0878C9B209F10109C8F82890D0F8E5
:10855000148048F00108C0F8148081F31188D3E733
:10856000BDE8F083704700BF00000120A801002093
:1085700090190120688B050800EE100AB8EE400A39
:10858000704700BFBCEEC00A10EE103A98B27047B8
:1085900007280AD800EB8000054B03EB4013B3F823
:1085A0000006B0FA80F0400970470020704700BF15
:1085B000A8010020072807D8044B00EB8000012207
:1085C00003EB401383F80226704700BFA801002088
:1085D000072808D8044B03EB401393F8542412B136
:1085E000012283F83A247047A8010020072808D800
:1085F000054B03EB4013B3F83804B0FA80F04009A0
:1086000070470020704700BFA8010020054B93F879
:10861000F825824204D903EB4013D3F84404704791
:1086200000207047A80100200346012200205A774D
:10863000704700BF826908B50346006BD96A0244DF
:108640009A6101B18847002008BD00BF436A024615
:108650001B681B6A5B685B7813F0010008BF5077EA
:10866000704700BFC2628161704700BF704700BFA2
:10867000043070470C4B93F89822D3F894120244BC
:108680000144D2B2C3F8941283F8982293F8982246
:10869000120605D593F8982282F0800283F898227A
:1086A000024B01225A7070479019012000000120EE
:1086B0002DE9F84F164FD7F89C52ED0A23D000262B
:1086C000DFF850A007F52879B0467419D7F8A01242
:1086D0004FF01003524648BF0134D1F828B0484645
:1086E000C7F8CC826410E102D8470F280BDD094B94
:1086F00003F1100153F8042B013207D18B42F9D159
:108700002546B542E1DCE802BDE8F88F661CF8E7D3
:108710009019012000000020194BD3F8D412D3F88F
:10872000D8228A1A322A05DCD3F8EC228A1A002AC7
:1087300011DC7047D3F8DC1249B193F8E82288883D
:1087400002F001020968120100FA02F28A610022B5
:10875000C3F8EC227047D3F8DC226AB110683231DA
:10876000928810B44469C3F8EC1222425DF8044BBD
:1087700018BF1204826170473231C3F8EC1270479F
:1087800090190120074AD2F8DC324BB192F8E82266
:108790009988186802F001031B0101FA03F3836151
:1087A0000020704790190120044B4FF4007C0020FA
:1087B000D3F8F832A2F800C00B607047901901207E
:1087C000002070470120704701207047002070474B
:1087D000134BD0F8E0105B68D0F8E82010B50446E1
:1087E000581A824200DC22B9D4F8EC200A44C4F8BA
:1087F000E42094F8D820C4F8E030012A05D0D4F859
:10880000DC300133C4F8DC3010BD04F1F001201D70
:1088100041F0B2FAD4F8DC300133C4F8DC3010BDDA
:10882000001000E0CB070DD430B590F828308DB0A3
:10883000C468012B07D0B4F1807F01D901230377ED
:108840000DB030BD7047194B456AD3E9CA13B1EB7F
:10885000930F4FEA93024FF0020306D252085B00D7
:1088600091429BB201D2FF2BF8D9B4F1807FAB804B
:10887000E6D90122002301A9B724027728460492F1
:108880008DF814208DF828208DF804400B93CDE945
:10889000021302A9CDE90633CDE9083341F06CFAA1
:1088A0002A68136A002BFCD1CAE700BF9019012087
:1088B00030B590F828308BB00446012B08D0407FAB
:1088C00010B901200BB030BD002363770BB030BD71
:1088D000456A2B681A7B22BB637F002BF1D01349BA
:1088E0000220002301220290081D8DF80C208DF833
:1088F00020200993CDE9001069462846CDE90433CC
:10890000CDE9063341F038FA2A68136A002BFCD10E
:10891000074B5B7DD84303F0010300F00100637750
:10892000D4E71B6A002BD7D00020CBE71000002033
:108930000000002030B504468BB094F82830012B9D
:1089400008D0637F0BB10023637701200BB030BDEB
:108950001B6A23B1656A2B681A7B002AF8D1637FF2
:10896000002BF2D010490220002301220290081DA2
:108970008DF80C208DF820200993CDE90010694670
:108980002846CDE90433CDE9063341F0F5F92A68EC
:10899000136A002BFCD1054B5B7D03F00102DB0762
:1089A0006277D2D5C9E700BF100000200000002088
:1089B000214A002330B5044695B0101D1F4D069383
:1089C000019002200B931093139311930290207F38
:1089D00000920495CDE90E3301238DF80C300793F6
:1089E0008DF820308DF834308DF8483002F10803CE
:1089F000083A0593031D0A920C93114B0993636A7D
:108A00001A68136A002BFCD1A0B10E480A0E00F1BF
:108A10001A0342760A0A9970080C69465A7018704F
:108A2000606A41F0A9F9636A1A68136A002BFCD1E5
:108A300015B030BD044BEDE7200000204D86000846
:108A400029860008000000201900002010B594B00D
:108A500004465022074968464FF0D2FC6946606AD6
:108A600041F08AF9636A1A68136A002BFCD114B0CA
:108A700010BD00BFB08F0508F8B50546406A006814
:108A8000046A002CFCD12C7FA869002C36D0234E20
:108A9000040E052786F82D402E36B0704FEA104C94
:108AA000000A1F4C86F800C0012B70704FF00000C8
:108AB0000E68676326641668A6642E63A06520D0DE
:108AC000022B1AD15368012220651E444968E365D0
:108AD000144B84F84C0061652E6384F86020636653
:108AE000114B6A7FA3F11401686A002A08BF194676
:108AF00041F042F9EB6A5BB1286BF8BD04270B4EDD
:108B0000CBE7084A84F84C306065E0652265E7E70A
:108B10006B6A1A68136A002BFCD1EDE70000002095
:108B20000000012035860008180001202D000020DB
:108B300000B583B08161019201A9049A00930123D9
:108B4000C2626A46FFF798FF03B05DF804FB00BFFE
:108B500070B51D46436A94B006461B681C6A002C1B
:108B6000FCD1314B0B9203F13C0230480694009249
:108B700003F14002049003F13400019202220590B7
:108B8000029201228DF820408DF80C208DF83420BF
:108B90008DF84820327F0C95101D1394CDE90944BF
:108BA000CDE90E44CDE910440790002A3AD00A0ED0
:108BB000363303F8012C0A0C99701D4C090A1A70FF
:108BC0005970706AD4E9CA32B3EB920F4FEA92013E
:108BD0004FF0020206D2490852008B4292B201D2F3
:108BE000FF2AF8D9737F8280D3B1694641F0C4F877
:108BF000706A03681A6A002AFCD10222D4E9CB34D5
:108C0000B4EB930F4FEA930106D2490852008C420D
:108C100092B201D2FF2AF8D98280284614B070BDE2
:108C200005A9E3E73533C6E7000000204D860008BC
:108C3000901901208269F0B592F8E4308BB00546B6
:108C4000012B27D0023B012B2FD892F85431EC4650
:108C5000D2F89C2063F07F03154C13708669D6F818
:108C6000A0305F1C0FCCACE80F00D6F89C30CDE9EB
:108C700000370FCCACE80F0094E803008CE8030049
:108C8000694606F1100041F077F8AA6911690B6A8C
:108C9000002BFCD1D2F8A0305A8852BAEA819A88C7
:108CA00052BA2A82DB885BBA6B8201200BB0F0BD1E
:108CB00000900508F0B590F8E4308BB00446D0F889
:108CC000A060012B4BD034D9023B012B2ED890F859
:108CD0005531EC46D0F89C2063F07F03434D137070
:108CE000D0F8A0305F1C0FCDACE80F00D4F89C305A
:108CF000CDE900370FCDACE80F0095E803008CE814
:108D00000300694604F1100041F036F82269136A45
:108D1000002BFCD173885BBAA4F8D030B3885BBA5F
:108D2000A4F8D230F3885BBAA4F8D43001200BB099
:108D3000F0BDD0F89C304FF0FF3205211A605A6028
:108D40009A60DA60D0F8E830C0F8F810B3F57A7FAE
:108D50001FD8032380F8E43001200BB0F0BD90F859
:108D6000542190F855319B1A5B100133DBB236F871
:108D7000132006EB430653BAA0F8D03073885BBAD1
:108D8000A0F8D230B3885BBAA0F8D43001200BB081
:108D9000F0BD03691A7B2AB35B691BB390F8983066
:108DA00003B390F854310122D0F89C0063F07F03A4
:108DB000C4F8A4400E49037094F8553194F8540156
:108DC00084F808211B1A84F8E420D4F8A020073383
:108DD000C4F80C110132D4F89C10C4E94023C4F843
:108DE000FC10A3E7022384F8E4309FE70090050815
:108DF00001800008F8B50C4B1D685A691540054004
:108E00005D617DB1094F0126B5FA85F4C4F11F04F7
:108E100007EB840306FA04F4D3F834030368984795
:108E2000A543F1D1F8BD00BF003C014090190120DD
:108E300002692DE9F843C36812EA030828D0054601
:108E40000E464FF00047B8FA88F327FA03F21B3BAF
:108E5000D24308EA02082A61042B16D8DFE803F09F
:108E60003B30251A0300B36A002B3FD003F1FF39D2
:108E700000231FFA89F9B362746A34B1236820466B
:108E8000494698476468002CF8D1B8F1000FDAD150
:108E9000BDE8F88370680028F7D0696B036889B271
:108EA0009847B8F1000FCED1F2E7B0680028ECD0B7
:108EB000A96B036889B29847B8F1000FC3D1E7E7FF
:108EC000F0680028E1D0E96B036889B29847B8F1EF
:108ED000000FB8D1DCE730690028D6D0296C0368D0
:108EE00089B29847B8F1000FADD1D1E7EB6A1FFA0C
:108EF00083F9C1E72DE9F041DFF8B48008EB4017B2
:108F000097F854340BB9BDE8F08104460D4646018C
:108F10004FF0E6FDC0BB2448464400EB4410A6F8E1
:108F200038544FF0EDFD98F80030D6F85024A3B136
:108F3000D6F83C140124D2F8AC308C4003F1C001C7
:108F4000420010F4004F90B202D15A6822435A6096
:108F50000C339942F4D1BDE8F081D6F83C140124D9
:108F6000D2F8AC3001F1100203F1C001944042008C
:108F700010F4004F90B202D15A6822435A600C3369
:108F80008B42F4D1BDE8F081084B93F8D42302EB77
:108F9000420203EBC203234493F88153002DBAD05D
:108FA000012387F83A34B6E7E00500209019012044
:108FB000A801002010B504464EF0BAFD0146204637
:108FC00089B2BDE8104095E738B50B4D00EB400085
:108FD00005F5A763C40003EBC003254493ED027AB3
:108FE000D3ED037AE7EE007AB0EE670A4EF0A0FD0B
:108FF000D5F83835186038BDA8010020836910B550
:109000001A4C04EB8303D3F8F80344F0F1F9B4F8F5
:1090100018340C2B0ED8DFE803F0220D0D0D1B0DBC
:109020000D0D070D0D0D1400D4F8D823D36823F4CB
:109030000063D3600122002384F8152484F81A34D5
:1090400010BDD4F8D823D36823F48053D360F1E75C
:10905000D4F8D823D36823F48063D360EAE7D4F844
:10906000D823D36823F40073D360E3E79019012079
:1090700080699C3044F0BCB9F8B5830AA3F580132D
:10908000522B52D804465748034493F8F4030D2852
:109090004BD8554D860105EB8013D3F81C74A742BD
:1090A00043D00139C3F81C4489B2C3F82814D5F859
:1090B0002C13B1FBF2F100220139C3F82C24C3F8C0
:1090C0002424C3F8302493F85924C3F8201402F060
:1090D000FF015AB345490223AF1901EB8011204625
:1090E00087F85934043144F0B9FD0123B4F1804FBD
:1090F00087F859343E4BA4EB0303B3FA83F34FEAEA
:10910000531316D0ABB93B4A944257D002F5806254
:10911000944253D0384902F57C42944218BF8C42A5
:109120002FD002F5705294422BD0F8BD83F858141A
:10913000D0E7AA1992F858140129F6D0022182F832
:1091400059142E49A06801400020A160012182F835
:109150005914AA19022182F859146268A16803B946
:1091600008B122F470022E4422F0700221F0800136
:10917000012000236260A16086F8590486F8583403
:10918000F8BDAA1992F858140129CED0022182F80C
:1091900059141A49A06801401948A1600121201AF8
:1091A00082F859140021B0FA80F082F85814124A5B
:1091B00040099442CDD00028CBD1F8BDAB1993F82B
:1091C0005824012AB1D002210C4A83F85914A0680E
:1091D0000240A260012283F8592483F8591462687E
:1091E000A168C0E7688B050890190120AC1D01201B
:1091F0000000014000040040000C00408800FEFF19
:1092000000040140F8B5A0F507642379DB0725D5F4
:10921000657994F8543805F001073D46FBB1D4F860
:1092200048341A68D36A5B08536294F8583823B1FB
:10923000B4F862380133A4F8623885F00101606C3B
:109240004BF060FD012384F85738002384F855382B
:1092500084F85638A4F85E3884F85438F8BD94F889
:109260005768012E03D194F8553884F856382046B3
:10927000FFF756F84EB9012385EA030184F8573801
:10928000606CBDE8F8404BF03DBD0023394684F8E2
:109290005738F5E770B505460726084C013E00D162
:1092A00070BD94F9000014F011FC031E04DB61781A
:1092B000EA189171A278EA540434EFE7289005087F
:1092C00038B58569002D3DD02C68236A1B7B5BBBBC
:1092D00020464DF0E5FB236A5B6803B3236A5A68B6
:1092E000236A22F01F025968236A01F01F019B685C
:1092F0001F33194421F01F01BFF34F8F00290ADDEE
:1093000002F12003114410488B42C0F85C221A4637
:1093100003F12003F8D1BFF34F8FBFF36F8F2846BF
:10932000BDE8384040F0F8BFAB68002BD0D01A68D9
:1093300020469B8893614DF0B3FB236A5B68002B4A
:10934000CCD1ECE738BD00BF00ED00E038B5846952
:1093500004B938BD256828464DF0A2FB2B6A1B7B5B
:1093600023B92046BDE8384040F0D6BFA368002BA3
:10937000F7D01A6820469B889361BDE8384040F0DA
:10938000CBBF00BF2DE9F843DDF820800F4616461D
:109390000021202204461D464FF028F9B8F1000FA5
:1093A0000CD0D8F80030B8F80A20E3811B0C2382D7
:1093B000D8F804306282E3821B0C238338464DF0D8
:1093C000C9FBF30619D4431EB8B107EB000C01E04A
:1093D000013B12D31CF801EDBEF12E0FF8D1C01ADB
:1093E00003F10109421EB944032AA8BF0322082B36
:1093F000A8BF082390461A4606E008280246B94648
:109400004FF00008A8BF08224FF02033394620460D
:10941000236063604EF0F4FF164B04F108004246EF
:109420004946238183704EF0EBFF611EE21D11F867
:1094300001CFACF16103ACF1200C192B98BF81F87E
:1094400000C09142F3D104F10A0011F8013FA3F1E9
:109450006102203B192A98BF0B708142F5D1182375
:1094600065832D0CE6722373099BA582E361BDE839
:10947000F88300BF202020002DE9F04FDFF8509442
:1094800085B0D9F8D402C9F8D802002B5ED00C46BA
:10949000154601F5FE7603EB020B1DE0002D62D0B0
:1094A000D9F80433AB4200F0C580D9F80033AB42A1
:1094B00000F0F780D9E9C231AB424BD88D42C0F001
:1094C0007281691A204648F0F1FD013504F50074F7
:1094D00006F500765D4539D0D9F81023AA42DDD8CB
:1094E000AA1AD9F82073D308396B02F0070802339F
:1094F0008B4202D3BA6B93420BD939461846039379
:1095000048F0A4FD039B0746002800F06C81C9F8D1
:1095100020033A79002A40F01D81D7F828A0BAF13B
:10952000000F00F059813A6B013520464FF400716D
:109530009B1AFA6804F5007406F5007608EBC30878
:109540003B4602EB4822D0475D45C5D1002005B01F
:10955000BDE8F08F8D42B4D24FF400720021204656
:109560004FF044F8B1E74FF40072294620464FF01F
:109570003DF88023CA4A84F8BE310C2384F8C231F6
:10958000D9F80013D9F8F8329142C4F8C611C4F8DA
:10959000CA3100F30D81C34A013BC34F82FB010274
:1095A000C81787FB01C70A44C0EB6212C0EB273023
:1095B000BE4F87FB02C7C2EB821C84F8C10180103A
:1095C000A1EB0C01174420F03F0001310843D117F3
:1095D000C1EBE71184F8C0010A4484F8BF21B04A06
:1095E000934200F3F180AF4AAF4882FB0312D917D0
:1095F00080FB03701A44C1EB6212C1EB2031AB480F
:1096000080FB0270C2EB821784F8C5118910DB1B46
:10961000104421F03F0101331943D317C3EBE0138A
:1096200084F8C4111A4484F8C3214AF65523A4F8D7
:10963000FE314AE74FF0FF3300274FF4F072201D50
:1096400084F8EC31394684F8ED3184F8EE3184F851
:10965000EF315223237063706123A37084F8E731E4
:109660004123E37084F8E631722384F8E43184F80E
:10967000E531D9F81833C4F8E8314EF0B7FF552377
:10968000C4F8F07184F8FE316FF05503C4F8F4713A
:10969000C4F8F87184F8FC7184F8FD7184F8FF3126
:1096A00013E74FF40072002120464EF09FFF804BDD
:1096B000022203CB45F6EB0322742273238090230E
:1096C000A273A370F82384F82C200822C4F80300A6
:1096D0006273C4F807106375D9F80013D9F8F8322B
:1096E0005B1A2362D9E9C2135B1A4AF655216362F9
:1096F0000023E372E3736377A377E37784F82D3075
:1097000084F82E3084F82F3084F83130694BA3610F
:109710003E232377012384F83030802384F84030BF
:10972000654BC4F84230654B84F84620A4F8FE111E
:10973000634A03CBC4F84B101988C4F847009B78E0
:10974000A4F84F1084F8513003CAC4F85200C4F88A
:109750005610BAE64FF40072002120464EF046FF44
:109760003B6CB8F1000F45D104F1200A002B00F04A
:1097700081803B6B112253492046CDE90088FFF7D9
:1097800001FE3B6C1A6C002A00F081801B6B504676
:1097900011224D49CDE90088FFF7F4FD04F1400A9C
:1097A0004FF4E07871E0E91A204648F07FFC8CE63F
:1097B000FF22013B84F8C1214FF6FF72A4F8BF21BC
:1097C000374A93427FF70FAFFF2384F8C5314FF636
:1097D000FF73A4F8C33128E751464FF400722046C6
:1097E0004EF004FF71E6231F384A43F8042F9E42CF
:1097F000FBD16AE6002B7F6C14BF02230123C3EB6D
:109800000813002F3FF461AE013BBF6C002B01DD5C
:10981000002FF9D1A2464FF40078002F3FF455AE47
:109820000AEB080303959A460BE00025A8F12008EF
:10983000CDE900E5FFF7A6FDBF6CCFB1B8F11F0F72
:1098400016D93D7907F11C0E112239683B6BAAEB42
:109850000800002DE9D17A79A8F120083D6942F08D
:109860002102CDE900E5FFF78DFDBF6C002FE5D1AA
:10987000039D2AE6CDE9008843464FF4F07808229C
:10988000D9F8FC122046FFF77DFD7F6CC5E75046F6
:10989000434611220C49CDE90088FFF773FD7DE7AF
:1098A000FF03FB008320088297554541818080801B
:1098B000DC0E06083F00FF0029940E0DE80E060896
:1098C000F40E0608D40E0608D80E0608DEADBEEF6C
:1098D0009019012010B490F8443000F10801484A72
:1098E000012BC2F8DC176DD08368464CD968A342BF
:1098F00021F46001D960D96841F46001D960996BA5
:1099000021F440119963996B41F480119963996B2B
:1099100021F4F8419963996B41F4884199639968FE
:1099200021F47021996099689960996821F4401137
:10993000996099689960596821F480615960596803
:1099400021F48051596059696FF30B0159615969CC
:10995000596148D0D9682B4C21F0E061A342D9600D
:10996000D96841F0E061D960996B21F440119963A5
:10997000996B41F480119963996B21F47821996373
:10998000996B41F410219963996821F470219960D1
:1099900099689960996821F4401199609968996073
:1099A000596821F480615960596821F480515960E7
:1099B00099696FF30B019961996999611AD0002334
:1099C00080F844301048114B848DC18D408D091BA7
:1099D000C2F8E447C2F8E0075DF8044B93FBF1F3EB
:1099E000C2F8E8377047D4F8041341F40001C4F812
:1099F0000413AFE706494B6843F400034B60DEE70E
:109A00009019012000200140007AF01F80380100E9
:109A100000230140704700BF014843F0BDBD00BFB7
:109A200090210120084810B4D0F80038D0F834480C
:109A300099691A682CB1234600F500605DF8044B63
:109A400018475DF8044B704790190120014843F016
:109A5000A3BD00BFF0210120084810B4D0F8603841
:109A6000D0F8944899691A682CB1234600F506602D
:109A70005DF8044B18475DF8044B704790190120BE
:109A8000014843F089BD00BF50220120084810B4AE
:109A9000D0F8C038D0F8F44899691A682CB1234638
:109AA00000F50C605DF8044B18475DF8044B7047F7
:109AB00090190120F0B506688C680F68B569002F11
:109AC00056D02E4B3B40B3F1005F4FD007F01F0C38
:109AD00004F11F0327F01F029C442CF01F0CBFF35E
:109AE0004F8FBCF1000F0BDD944402F12003DFF82F
:109AF00090E06345CEF868221A4603F12003F8D1BE
:109B0000BFF34F8FBFF36F8F02684FF480636B61B9
:109B100053696F602C6243B34B68F56963B31E46AB
:109B2000164B3340B3F1005F1AD006F01F0226F047
:109B30001F011F32224422F01F02BFF34F8F002A61
:109B40000ADD0A4401F120030D489342C0F8701267
:109B5000194603F12003F8D1BFF34F8FBFF36F8F86
:109B60004FF480636E606B612C62F0BD3246CCE7CF
:109B70003B463246034FCAE7034EF3E70000FFFFC0
:109B800000ED00E044000020480000202DE9F041F5
:109B90000468D4E904351A7DD3E90061002D4DD065
:109BA0001F2AA86138D820202F6800FA02F242F05C
:109BB0001802B2602A7D1F2A39D9203A202000FAE3
:109BC00002F242F01802FA606A6800200860106031
:109BD0003046116841F01001116093F80880A269C5
:109BE00041464AF03FFE2D7AE269384629464AF05E
:109BF00039FE274B626813F80800595D335843F06B
:109C0000010333507B5843F001037B50536843F00A
:109C100003035360BDE8F081203A20202F6800FA4A
:109C200002F242F01802F2602A7D1F2AC5D82020D5
:109C300000FA02F242F01802BA60C5E71F2A9861E2
:109C40001ED8202000FA02F242F01802B260002270
:109C500030460A600A6842F010020A601D7AA26962
:109C600029464AF0FFFD0A4B6268595D735843F07C
:109C700001037350536843F002035360BDE8F08161
:109C8000203A202000FA02F242F01802F260DEE7E9
:109C9000900F060810B1036882889A61704700BF70
:109CA00018B1838802681B0493617047D3B2012BFB
:109CB0001DD802EB42020F4B10B54FEA820E03F59E
:109CC000217C0EF1080402E01C3363450DD01A78A4
:109CD0008242F9D15A788A42F6D11A59002AF3D031
:109CE0000EF1040E03EB0E0010BD002010BD00208D
:109CF000704700BF4090050810B40C4C002304F6D8
:109D00006C1C01E0152B0CD003EB430201331CF853
:109D100002108142F6D1144494F96E095DF8044BA7
:109D200070474FF0FF305DF8044B704790190120E9
:109D3000D3B2022B21D802EB420270B54FEA820E59
:109D40000F4C002223460EF10C0503E001322C33A8
:109D5000172A10D01E68B042F8D193F804C08C4581
:109D6000F4D15E59002EF1D02C210EF1080301FB35
:109D70000233E01870BD002070BD0020704700BFA6
:109D8000688B0508002838D0002330B51B4D90F8AB
:109D900004C005F66C1401E0152B2CD003EB430234
:109DA0000133A15C6145F7D11544046890F805E0E2
:109DB00095F96E39DAB2022A1DD803EB4303104835
:109DC00000224FEA830C03460CF10C0503E001323C
:109DD0002C33172A0FD019688C42F8D119797145A4
:109DE000F5D159590029F2D02C210CF1080301FBBF
:109DF0000233184430BD002030BD70479019012057
:109E0000688B05080348D0F88C300BB17C301847BC
:109E1000704700BF000001200348D0F8B0300BB1FC
:109E2000A0301847704700BF000001200348D0F859
:109E3000D4300BB1C4301847704700BF0000012078
:109E40000348D0F8F8300BB1E8301847704700BF2E
:109E5000000001200348D0F81C3113B100F58670D2
:109E600018477047000001200348D0F8403113B173
:109E700000F5987018477047000001200348D0F89B
:109E8000643113B100F5AA70184770470000012033
:109E90000348D0F8883113B100F5BC7018477047FB
:109EA000000001200348D0F8AC3113B100F5CE70AA
:109EB00018477047000001200348D0F8D03113B193
:109EC00000F5E07018477047000001200348D0F803
:109ED000F43113B100F5F27018477047000001200B
:109EE0000348D0F8183213B100F5027018477047D4
:109EF000000001200348D0F83C3213B100F50B708C
:109F000018477047000001200348D0F8603213B1B1
:109F100000F5147018477047000001200348D0F87E
:109F2000843213B100F51D701847704700000120FE
:109F30000348D0F8A83213B100F5267018477047CF
:109F40000000012001380D4B0D4A00EBC000116BE1
:109F500003EB800310B4DB6F83B00A4CA34214BF41
:109F60004FF480034FF4001319431163126B134035
:109F70000193019B03B05DF8044B70470000012082
:109F800000380240006002400138F8B500EBC00024
:109F9000114C1D46114B04EB800417460E46E06F32
:109FA000984214BF9620952048F062FD94F99100E4
:109FB000B909C4F88C60C4F8945048F0B7FC94F91F
:109FC0009130002B07DB03F01F0001225B090449DD
:109FD000824041F82320F8BD0000012000600240CB
:109FE00000E100E0800AA0F58010522808D8054B57
:109FF000034493F8F4330D2B02D8034AD05670472C
:10A0000000207047688B0508800F06080120FEF7C6
:10A01000F1BE00BF0220FEF7EDBE00BF0420FEF738
:10A02000E9BE00BF0820FEF7E5BE00BF1020FEF726
:10A03000E1BE00BF4FF47870FEF7DCBE4FF47C4009
:10A04000FEF7D8BE30B1036882881B691A4214BF7C
:10A0500001200020704700BF2DE9F04F0E4683B06D
:10A0600004461546002800F0C7800268644B13447C
:10A070009B0A644AC6F34119134493F85C0748F0FD
:10A08000F7FCC6F38103B4F804E006F0030124688A
:10A0900001939EFAAEF0B0FA80F001F1FF383EFA7B
:10A0A00000F367D001220327009603E001303EFA57
:10A0B00000F35ED002FA00F313EA0E03F6D0D4F8F0
:10A0C00000C093FAA3FBBBFA8BFB93FAA3FABAFA8C
:10A0D0008AFA4FEA4B0BB8F1010F4FEA4A0A07FA26
:10A0E0000BFB01FA0AFA2CEA0B0C4CEA0A0CC4F836
:10A0F00000C04ED9D4F80CC093FAA3FBBBFA8BFB7B
:10A1000093FAA3FABAFA8AFA4FEA4B0B02294FEAFA
:10A110004A0A07FA0BFB09FA0AFA2CEA0B0C4CEA7A
:10A120000A0CC4F80CC0C1D193FAA3FABAFA8AFA9D
:10A130004FEA132CBAF1070F45DCD4F820C093FA8C
:10A14000A3FABAFA8AFA93FAA3F34FF00F0BB3FA11
:10A1500083F34FEA8A0A01309B000BFA0AFA05FAE8
:10A1600003F32CEA0A0C4CEA030323623EFA00F3E1
:10A17000A0D1009EB8F1010F08D86268C6F30013A1
:10A1800022EA0E020EFB03F31343636003B0BDE843
:10A19000F08FD4F808C093FAA3FBBBFA8BFB93FAB9
:10A1A000A3FABAFA8AFA4FEA4B0B019E4FEA4A0A1F
:10A1B00007FA0BFB06FA0AFA2CEA0B0C4CEA0A0C1B
:10A1C000C4F808C096E7D4F824A09CFAACFBBBFA0C
:10A1D0008BFB9CFAACF34FF00F0CB3FA83F34FEA0E
:10A1E0008B0B9B000CFA0BFC05FA03F32AEA0C0A12
:10A1F0004AEA0303636259E74FF0FF3339E700BFD0
:10A200000000FEBF688B050800B125E770472DE907
:10A21000F84FBB4F6023064603FB0073D3F8EC47AF
:10A22000D3F8F487D3F8F857002C00F05D81B8F12B
:10A23000000F04D098F90630002B40F0558125B16D
:10A2400095F90630002B40F04F81731CDBB2B8F15A
:10A25000000F04D0152288F8073088F8062015B1C1
:10A260001622EB71AA714FF0600A207E48F000FCC4
:10A2700029460AFB06FA40464CF036F8404607EB02
:10A280000A09042240F2145899F8FC37002B0CBF3D
:10A290004FF01E0B4FF03E0B5946FFF7B5FF284617
:10A2A000984D042259465544FFF7AEFF4C22002139
:10A2B00028464EF09BF9D9F8EC379FED937AB0EE33
:10A2C000084A5B68F7EE003AB9F8FEA74FF0000CB9
:10A2D000C9F800388D4B9FED8E5A9A688D4BC2F3AA
:10A2E0008222134493F86427D7F82C33D34007EE27
:10A2F000903AF8EE677AC7EE275A07EE90AA9FEDDC
:10A30000867AF8EEE77AC7EE274ADFED847AB0EE78
:10A31000007AE5EE877AA5EE875A25EE844A37EE75
:10A32000856A74EEE72ABAF5C87F0CF1010ED5BF35
:10A330004FF4967278226423322307EE90EAD8BF56
:10A340004FF416791344A2F13202F8EEE76AC8BF5F
:10A350004FF4827907EE903AD4BF41464FF4FA7138
:10A3600066EEA56AB8EEE77AC7EE267A07EE102AFF
:10A3700001EB0902B8EEC77A37EE447A77EEE37A5A
:10A38000FCEEE77A17EE903AC7EE267AFCEEE77A13
:10A3900017EE900A07EE909AB8EEE73A07EE902A89
:10A3A000F8EEE77A23EE243A83EE277A37EE453A41
:10A3B00032EEC77AC3EE267A77EEE37AFCEEE77ADE
:10A3C00017EE901AC7EE267A77EEE37AFCEEE77A7C
:10A3D00017EE902A02F1020909EB010BB0EE467A62
:10A3E00007EE90BAF8EE677AA6EEA77AF4EEC74ABF
:10A3F000F1EE10FA7CDC43EA00095FFA89F9B9F161
:10A400000F0F77D841EA02091FFA89F9B9F1FF0F56
:10A4100070D81B05000403F07F6392B200F47F0044
:10A4200003433F4843EA0C7300EA01210B43134303
:10A430006022284602FB06760027C6F8043801236E
:10A44000C6F80878C6F80C38C6F81078C6F814783C
:10A45000C6F81C78C6F820784AF056FF96F84138BE
:10A46000202BD9B21AD196F84038012B16D02423CC
:10A4700086F84138D6F800381A6822F001021A60CE
:10A480001A6822F480521A601A681A601A6842F038
:10A4900001021A6086F8411886F84078002194F984
:10A4A0001A0048F043FA94F91A20A37E002A08DB28
:10A4B0005909012203F01F0302FA03F3194A42F873
:10A4C0002130002194F9190048F030FA94F919204C
:10A4D000637E002A08DB5909012203F01F0302FAF8
:10A4E00003F3104A42F82130BDE8F88FF4461AE72A
:10A4F000013171E7BEF10F0FF8D1002398E700BFDB
:10A500009019012090210120286B6E4E00380240E6
:10A5100000001643688B050800247449000070424F
:10A5200000FFFF0000E100E008B1002294E5704761
:10A5300070B50E4C94F8F865AEB104F5876400254B
:10A5400003E001352034B5420DD0237F002BF8D035
:10A55000E06800220028F4D00135217DFFF77CFD62
:10A560002034B542F1D1012070BD00BFA801002008
:10A5700070B590F8B2311C09013C052C0FD81A4E69
:10A58000054603F00F0306EB4402B2F86C0740FAED
:10A5900003F2D20703D595F8B521012A01D0012095
:10A5A00070BD9A402644013A10404EF0FFF896F8EC
:10A5B00078370E4A034402EBC30452F83320A388D1
:10A5C00010691840ECD0002395F8B32102212046F1
:10A5D00085F8B531FFF740FDD5F82021136843F029
:10A5E00008031360DBE700BF688B05083C230120EC
:10A5F000014B53F82000704750280040014B43F8AE
:10A600002010704750280040204B2148196C214AE7
:10A6100041F0805130B482B01964196CFF2401F00C
:10A62000805101910199016841F480710160CA2053
:10A63000196C41F480611964196C01F48061009116
:10A640005321009D5462506251625B6FDB0013D452
:10A65000114B00221149C3F85428C3F85828C3F8F5
:10A660005C28C3F86028C3F86428C3F86828C3F8D6
:10A67000501802B030BC7047A2F50062074BD2F808
:10A6800050289A42E4D102B030BC704700380240F2
:10A690000070004000280040002000403166654204
:10A6A0002DE9F84FD0F894700446524B00F164063F
:10A6B000FDB227F0FF09826800F1180A103D4846F4
:10A6C000D2F80080A3FB05352D0929464AF012F97E
:10A6D000626D0023B2F5807F84F858307ED00DD8AB
:10A6E000102A00F083805CD8012A45D0042A16BFC6
:10A6F0006FF400616FF008013C230EE0B2F5805F5B
:10A7000070D0B2F5803F3AD0B2F5806F15BF6FF4CC
:10A7100000616FF008013C230423324608F118065B
:10A72000404656F803C001EA0C01F150D4F854B089
:10A73000594649F0EBFEBBF5807F2DD023D8BBF105
:10A74000100F3ED036D8BBF1010F02D0BBF1040F81
:10A7500033D14FF0080C336852462946484643EA45
:10A760000C033360402323624AF07CF83B6843F0DB
:10A7700010033B60BDE8F88F6FF00801CDE76FF084
:10A7800008013C23C9E7BBF5805F22D0BBF5803FC1
:10A790001AD0BBF5806F10D108F11C064FF0080CE1
:10A7A000D9E7402A15BF6FF400616FF008013C2320
:10A7B0000023B2E7BBF1400FCBD03C364FF4006C26
:10A7C000C9E74FF4006CC6E708F154064FF0080CD7
:10A7D000C1E708F11C064FF4006CBCE76FF00801FC
:10A7E00004239AE76FF40061042396E76FF4006195
:10A7F00093E700BFABAAAAAAD0F8AC312DE9F04F7D
:10A8000093F9298083B005790446B8F1000F93F8D5
:10A81000299005F00205C0F297814FEA5912C64B04
:10A8200009F01F0153F8226003EB8203CE4006F0CB
:10A830000106002D40F0598101228A40C3F8802092
:10A84000BFF34F8FBFF36F8FD4F8A011086820F4C7
:10A85000F8700860886820F001008860C3F88021E3
:10A86000BFF34F8FBFF36F8F04F59077D4F820A11B
:10A870002423A268C4F89431DAF8003023F00103ED
:10A88000CAF800300023CAF80030CAF80430CAF809
:10A890000830C4F89C3184F89031C4F89431C4F87D
:10A8A0004031C4F89831C4F82421C4E94D336379A8
:10A8B0009A0203F0010102F48052C4F828211A031D
:10A8C00002F40052C4F82C211A0202F48062C4F887
:10A8D0003021227912F0010B00F0F2800420C4F83C
:10A8E000340115B10C20C4F83401002940F0038173
:10A8F00094F8B4214AB1D4F8442142F00802C4F8D3
:10A9000044214FF40042C4F8542113F0080FD4F846
:10A9100094314FF024033846C4F89431DAF800300B
:10A9200023F00103CAF8003000F0268143F09EFABC
:10A9300001281FD0D4F84431002B40F04781DAF8C9
:10A94000043023F49043CAF80430DAF8083023F0D6
:10A950002203CAF80830DAF8083043F00803CAF8CE
:10A9600008303846DAF8003043F00103CAF8003006
:10A970004AF0EAF8BBF1000F64D0D4F8FCA0BAF1B9
:10A98000000F00F0C68000234FF4807C04F13C0BE4
:10A99000C4F83CA0C4E91133C4E91433C4E9183342
:10A9A000C4E91A33D4F80431584623644FF4806361
:10A9B000E3644FF48033C4E916C34BF0A9F858465A
:10A9C00042F03CFCD4F89831C4F88CB1202B676776
:10A9D000019333D1E368626999B27AB3B1FA81F035
:10A9E0004009009051B394F89001012826D0A4F8B2
:10A9F0007811584600999BB2D4F820B1C4F89C1144
:10AA0000C4F88C102221C4F87421C4F898114B4961
:10AA1000A1674B49E1674B49C4F888100BF1240149
:10AA200042F0A6FC002800F0D98010230098C4F85A
:10AA30009C31019B84F89001C4F89431DAF8043019
:10AA4000C4F81431A5B3D4F800513DB3002304F188
:10AA50009C0AC4F89C50C4F8A8305046C4F8B830DA
:10AA6000C4E92C33C4E93033C4E93233D4F80831B3
:10AA7000C4F8A0304023C4F8A4304FF48063C4F875
:10AA8000AC304FF48033C4F8BC304BF041F8504642
:10AA900042F0D4FB002800F09380FEE7D4F8A03108
:10AAA0001A6842F080021A601A6842F040021A6086
:10AAB000B8F1000F01DB002E71D103B0BDE8F08FBB
:10AAC00015B10820C4F8340100293FF411AF9207F2
:10AAD0007FF50EAFD4F8442142F00102C4F84421BE
:10AAE0004FF40032C4F8482102E790F8B251003D1B
:10AAF00018BF0125A0E6D4F84411920741F00201E5
:10AB0000C4F844114FF48031C4F84C117FF5F0AE15
:10AB1000E0E7D4F8A0311A6842F480721A609A68AB
:10AB200042F001029A601A6842F020021A601A6824
:10AB300042F010021A6085E700E100E071B50408F8
:10AB4000A1B50408A5B50408D0F8A03125B190F846
:10AB5000B251003D18BF01251A6822F4F8721A603C
:10AB60009A6822F001029A60BFF34F8FBFF36F8F94
:10AB7000002604F5907779E643F078F901283FF450
:10AB8000F9AED4F844312BBBDAF8043023F4904307
:10AB9000CAF80430DAF8083023F02A03DFE64FEA77
:10ABA0005911194A09F01F09012302EB810003FA28
:10ABB00009F3C0F8803142F8213003B0BDE8F08FCE
:10ABC000C4F888A1C4F8D470686071E7384643F0CF
:10ABD000C1FAB4E6384643F0BDFAD5E784F89001EF
:10ABE000DBF8003043F48073CBF80030DBF808303A
:10ABF00043F00103CBF80830DBF8083043F04003A2
:10AC0000CBF808301AE700BF00E100E038B50409CE
:10AC1000013C052C1AD80F4D00F00F0305EB440240
:10AC2000B2F86C0740FA03F212F0010210D00122D0
:10AC3000254402FA03F3013B18404DF0B7FD95F8A7
:10AC40007837054A034402EBC30038BD002038BD05
:10AC5000104638BD688B05083C23012070B586B0CE
:10AC60000024054600F5887E0DF1040CC0F80C4167
:10AC700044F23B360594C0E93F44C0E94144CDE984
:10AC80000144CDE90344BCE80F00AEE80F00CEF864
:10AC9000004095F82901A5F8546108B906B070BDC7
:10ACA000FFF7B4FF2946064698B126232246C38003
:10ACB0000C4B41F80C3F4AF099FCB2880A494FF01E
:10ACC0000043B2FA82F20868D34003430B6006B037
:10ACD00070BD044B024641F80C3F06B0BDE8704021
:10ACE0004AF084BCD1870008003C01402DE9F84FB0
:10ACF0006D4EC0EB001306EBC303D3F8AC4C002C35
:10AD000000F08A8093F81C8D05460701404647F005
:10AD1000AFFE01224FEA581308F01F08013B02FA68
:10AD200008F2032B08D8DFE803F0ADB302B95F499E
:10AD30000B6A23EA02030B627B1B05F1010B06EB96
:10AD4000C3035FFA8BFB93F8B00CFFF75FFF8046FD
:10AD500018B1122380F807B083717B1B06EBC30385
:10AD600093F8B10CFFF752FF824618B1132380F815
:10AD700007B083717B1B06EBC30393F8B20CFFF79C
:10AD800045FF814618B1142380F807B083717F1BFB
:10AD900050462E2106EBC70696F8B42CFFF734FA7E
:10ADA00096F8B52C48460E21FFF72EFA96F8B32CEC
:10ADB0002E214046FFF728FA23683D4A23F040033E
:10ADC000944223602AD03B4B9C4231D103F500339F
:10ADD0001A6A42F480421A621A6A22F480421A62A3
:10ADE000636843F48053636023685B060CD4206877
:10ADF00040F217323049314B01400A432260626809
:10AE0000134043F4E0636360E36923F40063E361A8
:10AE1000236843F040032360BDE8F88F234B5A6A50
:10AE200042F480525A625A6A22F480525A62D7E738
:10AE3000234B9C421BD0234B9C420DD0224B9C4267
:10AE4000CED103F568435A6A42F480125A625A6AB4
:10AE500022F480125A62C3E703F582335A6A42F43D
:10AE600000525A625A6A22F400525A62B8E703F555
:10AE7000FE331A6A42F400421A621A6A22F400424D
:10AE80001A62ADE709494B6923EA02034B6153E7B4
:10AE900006494B6A23EA02034B624DE703490B69FB
:10AEA00023EA02030B6147E79019012000380240B2
:10AEB00000300140003800404000FFFFFBF0FFFF82
:10AEC000003C0040003401400050014008B51D2006
:10AED000FFF79CFE10B190F9063053B11E20FFF72A
:10AEE00095FE10B190F9063003B108BD5523C3801B
:10AEF00008BD5523C380F1E72DE9F04F002391B041
:10AF0000A24E0293A24BA6F67C0ADFF88C9293F82D
:10AF10009EEEA04D0EF1FF37CDF80CE0FBB2019391
:10AF2000DFF88CB2DBF80070BB0AA3F58013522B5C
:10AF300000F2CF80534493F8F4330D2B00F2C98014
:10AF400015F90380039B012B00F01681039B022B54
:10AF500002D1B8F1080F3AD10024214640460FF043
:10AF60009BF90FF021FA90F900C0BCF1000F18BF57
:10AF7000BCF1540F14BF4FF0010C4FF0000C40F027
:10AF8000F1800434A4B2102CE7D1029B002B00F016
:10AF9000AB80814A0CE0534493F8F4330D2B0ED868
:10AFA000EB5643450ED002F586724A4500F0988074
:10AFB00091680B689B0AA3F58013522BEBD90023F1
:10AFC0004345F0D14B799BF805109942EBD10BF139
:10AFD0001C0B5E45A6D1029B09F586790133042B33
:10AFE00002939DD16D4A4FF0010B92F8F83502F5AE
:10AFF000876A01330493049B5B4567D0644BDAF89E
:10B000000C7093F8B22E9AF810300193002F5DD097
:10B0100062493B684D686248B988002D1844039323
:10B0200002914FEA902040F3C8805B49002405E07C
:10B03000013401F58671AC4200F0BC800B6883429C
:10B04000F6D1554B4FF48672029D02FB0434019BEE
:10B050000322CAF80C708AF81030029BCAF8184014
:10B06000B3FA83F6C6F11F035800CAF80430BA7168
:10B0700087F807B002FA00F7A16C0122D4F854C097
:10B08000394302FA00F002FA03F3A164216D01438F
:10B09000D4F8AC00216541490F7899B2002F00F037
:10B0A000708143EA0C036365039B9D61FDF776F8AD
:10B0B0000BF1010B2046FDF745F80AF1200A40F29A
:10B0C0000113BBF1090F2AF8043C94D111B0BDE87B
:10B0D000F08F019B012B7FF67AAF4FF000083BE722
:10B0E000BCF1000F7FF473AF5846FCF7F1FF9BF8FB
:10B0F00005E0C3B2022B00F2958300F1010C294A4E
:10B100000CEB4C0C02F57D704FEA8C0C03E02C32FA
:10B11000904200F0878313689F42F8D113797345FA
:10B12000F5D152F80C30002BF1D01F4800214268B5
:10B130009A4207D00131243010293FF448AF4268C9
:10B140009A42F7D14B1C194ADBB2013B03EBC30314
:10B1500002EB830393F99830002B7FF438AFC9F8E2
:10B1600008B038E7029B002B7FF413AF0BF11C0BE8
:10B170005E457FF4D7AE2EE7B8F1010F3FF4ECAE99
:10B180000BF11C0B5E457FF4CDAE24E7E49305087C
:10B1900090190120800F0608B0010020A8010020AE
:10B1A0000000FEBF688B05087C0001200000012024
:10B1B000E8920508042C00F0F2804FF48671B54B3C
:10B1C00001FB053319690691002900F0FB829860A4
:10B1D000013054210792C4B2AE4A83F8101183F8AB
:10B1E00011416B1C5360069B18461E685B790593E2
:10B1F000FCF76EFFC3B2022B00F2148300F1010EC4
:10B20000A5494FF0000C079A0EEB4E0EDDF8149096
:10B210004FEA8E0E06E00CF1010C2C31BCF1170F39
:10B2200000F000830B689E42F5D10B794B45F2D1BB
:10B2300051F80E30002BEED098462C2300EB400046
:10B24000954903FB0CF3DFF8809203EB80039148F0
:10B250000B4419694FF4867303FB05034846C3E9A1
:10B26000078143680021434507D00131243010296C
:10B270003FF42CAF43684345F7D14B1C8749DBB201
:10B28000013B03EBC30301EB830393F998100029FF
:10B290007FF41CAF4FF48671814883F899404FF0DA
:10B2A0008C0C01FB05F17B4C062A07914FEAA101AA
:10B2B00000FB01F17B4800F54C7E07982044039C7D
:10B2C000C0F800C10CFB01FC01EB4101C46001EBC3
:10B2D0000111744C0EEB4C0E04EB81044FF0540141
:10B2E000C0F8FCE083F898104FF033030799C0F8DA
:10B2F000B8306D4BC0F8B44003EB01046B4BD3F88E
:10B300002C1300F04D82072A694B6A486A4A18BF1D
:10B310001A466A4B18BF03465E48B1FBF3F3B1FB14
:10B32000F2F2013B4FF48671013A01FB05019BB239
:10B33000A1F8BC20A1F874302366079B03F15801E3
:10B3400000F10803304619440023A4F8583063661E
:10B35000E36549F023FA3368059A43F080033360CC
:10B360000C2A23D8DFE812F0C301220022002200B9
:10B37000A101220022002200E3012200220022007B
:10B380007D01C6F12F062D0402FA06F33A4643EA80
:10B390000C036365039B9D61FCF700FF88E60323B4
:10B3A000424A82F8B33E11B0BDE8F08F394A4FF4FB
:10B3B0008673304603FB05230222596933680391E3
:10B3C00023F00103336000230A930D930F9360234E
:10B3D00008934FF480730E93012309930A23CDE958
:10B3E0000B3208AA49F092F80399B1F5807F00F07A
:10B3F000FD8100F2D881102900F0028200F2E9817B
:10B40000012900F0FA81042915BF4FF400630823D5
:10B410003C20002006F118010A5813430B50069BEC
:10B420001879002840F0AB81336843F001033360A2
:10B430000023D9F804200133904500F09B81102BA4
:10B4400009F12409F5D14FF0FF334FF00008134AFA
:10B4500003EBC30302EB8303D86F194B984214BF6D
:10B460009620952047F004FB059B0C2B00F27F8172
:10B47000094A02EB4303B3F87CC84FF48673054ACC
:10B48000104803FB052300F26471A3F818C00023E1
:10B4900023E000BFA8010020688B05080000012000
:10B4A0006B4CA40774120020B001002090190120F9
:10B4B00044950800D0DD06001055220040771B009F
:10B4C00000600240A01200207C000120964200F0A3
:10B4D00088810133042B00F0A88151F83320002A21
:10B4E000F4D1D0F884270132C0F8842700EBC300E0
:10B4F000DB00C0F8646719444046234690228E88DA
:10B500004CEA060C0026A1F804C0BF49FEF73CFD3A
:10B510004FF48673BD4A40214FF4403CBC4803FBC6
:10B5200005280423D8F81C502A6842F010022A602B
:10B530002A6842F014022A60C4F8A860C4E91F66B1
:10B54000C4E92866D8F82020A1674FF48061C4F8C8
:10B5500098C04FF4804CC4F88410E9B2C4F89C3011
:10B56000C4F8942010390392D8F8B820A0FB010148
:10B5700025F0FF00C4F890204FF48052D8F80C90CA
:10B58000D940C4F88820079B09F1180209F1100975
:10B59000226703F170029F4B1A44D8F8B430C4F804
:10B5A0008CC06367CDE9050149F05CF9D5F800E08E
:10B5B000079BC4F820E0D5F814E003F1B802954BDE
:10B5C000C4F824E0D5F804E01A44039BC4F828E04A
:10B5D000D5F808E0C4F82CE0D5F80CE0C4F8DC306D
:10B5E0000423C4F8C860C4F8E4304FF48063C4F89E
:10B5F000F060C4F8CC304FF40033C4F830E0C4F845
:10B60000E030C4E93066C4E93A664FF40066D8F821
:10B610000031C4F8B890C4F8D0604FF48046C4F844
:10B62000D830D8F8FC30C4F8D460C4F8BC30DDE9B8
:10B63000050149F017F92B6863636B69A3636B68B5
:10B64000E363AB682364EB6863642B6843F0100327
:10B650002B602B6843F014032B603B68BD88039379
:10B66000F5E433684FF4867268494FF0020E23F018
:10B670000103304602FB05124FF48051516108AAC4
:10B68000336000230A930D930F93602308934FF4C4
:10B6900080730E93012309930A23CDE90B3E48F0F2
:10B6A00035FF4FF400630420B4E633684FF486722C
:10B6B0005649022023F0010302FB051210215161BB
:10B6C00008AA336000230A930D930F936023089315
:10B6D0004FF480730E93012309930A23CDE90B30B5
:10B6E000304648F013FF00204FF4006392E63368C1
:10B6F0004FF486724549304623F0010302FB0512E0
:10B700000121516102223360002309910A930D93B4
:10B710000F93602308934FF480730E930A23CDE9AF
:10B720000B3208AA48F0F2FE0020082372E63368C4
:10B730004FF486723549022023F0010302FB051203
:10B740004FF4807151616022336000230E910A939F
:10B750000D930F930123CDE908230A2308AACDE90D
:10B760000B30304648F0D2FE0823042052E64FF05A
:10B77000000C82E65FFA83F808F1FF3367E6FFF713
:10B7800045FA039038B10699CA790221FEF764FCA4
:10B790005423039AD380736C43F40043736443E6E9
:10B7A0001D4A1E4BB8E5B1F5805F22D0B1F5803F50
:10B7B00019D0B1F5806F15BF4FF4006308233C200A
:10B7C000042027E60223164A82F8B33E11B0BDE8F2
:10B7D000F08F402915BF4FF4006308233C20002060
:10B7E00018E6DB0087E608233C2013E60823042044
:10B7F00010E64FF4006304200CE60020082309E65D
:10B8000000204FF4006305E6E9810008A80100204C
:10B81000ABAAAAAAB0010020882A1100A0BB0D0083
:10B820009019012000235B68FFDE00239B88FFDE68
:10B830002DE9F04F9A4C8BB094F8B47E1FB90020DC
:10B840000BB0BDE8F08F00222F2138460EF002FE2B
:10B8500006460028F3D090F80590D0F800A0A4F890
:10B860001894FEF78FFA0028E9D0D0E9015B002D8B
:10B87000E5D0DFF864820023424601E0102BDED0E1
:10B880005168013324328D42F8D1DBB2013B03EB26
:10B89000C302844B03EB820292F998100029CED1A7
:10B8A0002F20C4F8D8A3A2F89800D4F82C037E4A1D
:10B8B000904280F0D880000AC4F8DC137B49002253
:10B8C000A1FB00017A48C4F8E823C4F8E0230A0980
:10B8D0000909A0FB0202C4F8E4135208A4F8B82E28
:10B8E0005200A4F8B62E94F8152402F0FF01002AA5
:10B8F00000F0C580022250466E4984F8152442F0BB
:10B90000ADF90122384684F81524FFF77FF9654B1D
:10B91000C4F8BC0E30B12F21C1804E21F279FEF760
:10B920009BFB604B644A0021C4F8C4BEB9F10C0F04
:10B93000C4F8CC1EC4F8DC1EC4F8E41EC4F8EC1E27
:10B94000C4F8F01E106BC4F8C05E40F40010106321
:10B95000106B00F4001000900098106B40F4800011
:10B960001063126B02F480020192019A4FF04002C0
:10B97000C4F8C82E4FF48062C4F8D02E4FF4805221
:10B98000C4F8D42E4FF48042C4F8D82E4FF40032BD
:10B99000C4F8E02E4FF00302C4F8E82E72D8474AEC
:10B9A00002EB4902B2F89878BA4608374448414653
:10B9B000002204EB870CCCF8D803A0F6E820C4F8EA
:10B9C000F80E486801322431854260D0102AF8D13F
:10B9D0004FF0FF3202EBC20203EB8203D86F394B08
:10B9E000984214BF9620952047F042F80023D8F8DB
:10B9F0000420013308F12408954246D0102BF6D1DB
:10BA0000002004EB8704534660222F49FEF7BCFA5E
:10BA1000D4F8D80341F012FC00287FF410AFB479B9
:10BA200000276026089063004A4602A9274803F0D1
:10BA300002030493E300CDE9026703F00803002644
:10BA400000270593CDE9066746F0B8FC00287FF48F
:10BA5000F6AEA30749461D481CD542F0E3F9B0FAFB
:10BA600080F04009ECE61A4A1A490244A1FB02217F
:10BA7000890D013989B24A1CB0FBF2F01BE784F84A
:10BA8000141437E78A460F468FE7D8B2B9E7D2B227
:10BA9000013A9FE742F0B2F8B0FA80F04009CFE6F1
:10BAA0009019012000000120006CDC02598B4F012D
:10BAB000ABAAAAAA6C1D012000380240688B0508B9
:10BAC0005028012000600240FD8F0008681D012001
:10BAD00000366E01819F5E167C000120F8B50E4C89
:10BAE00094F8F8759FB104F5C064C7F109070925FA
:10BAF000013D0ED0A6683079FFF788F8217DF279F4
:10BB000008B1FEF7A9FAAF4204F1A004F0D1012078
:10BB1000F8BDAB68FFDE00BFA80100202DE9F041B1
:10BB20000446EFF31185502383F3128803799B07B2
:10BB300002D590F8B2313BB9012384F8A431EDB2BB
:10BB400085F31188BDE8F081D0F800311B6813F04F
:10BB50000103F4D1D0F89421D0F898110A4302F0EF
:10BB60002102212AEBD0D0E909129142E4D090B20F
:10BB70003ED8194623691B1A9BB2D4F89461A1627E
:10BB80000021202E84F8A411D9D1A1698918D6D01A
:10BB9000B3FA83F77F09002BD1D094F89021012AC2
:10BBA000CDD00122D4F88801A4F8723184F8902114
:10BBB0002122C4F89C71D4F82081C4F86C11A4F837
:10BBC0007031C4F89421B0B1114A0765C263114ABB
:10BBD0000264114AC26408F1280241F0C9FB50B165
:10BBE000102384F89071C4F89C31C4F89461A6E7DE
:10BBF000081A83B2C1E700234022C8F8202084F845
:10BC00009031D8F8083043F08003C8F8083096E740
:10BC100049B504086DB50408A5B504082DE9F84335
:10BC20000379054613F0020604D090F8B261003E95
:10BC300018BF0126D5F820412768D4F8088017F0EE
:10BC4000200958D1FB0540F18880E369DA0701D566
:10BC50000123236218F0010F7BD0E3699B0701D514
:10BC600002232362E369580701D504232362E369B1
:10BC700019076BD4002E5FD07A0628D5E3695E06DB
:10BC800025D54023236295F8B561002E00F0908001
:10BC9000D5F80031002B68D02846FFF73FFF95F814
:10BCA000A431A3B195F8B5418CB995F8B201FEF76E
:10BCB000ADFFD5F820210121136823F0080313609C
:10BCC00085F8B51118B122462021FEF7C5F9D5F83F
:10BCD0000031002B49D0F9060BD5D5F82031DA69AF
:10BCE000D20606D56A6B12B19047D5F820311022E2
:10BCF0001A62BDE8F883E369980614D5606AEB6AB6
:10BD0000C0B2002B48D0296B9847D5F82041236852
:10BD100023F480732360A36823F00103A360A36965
:10BD200043F00803A361F9058FD418F0010F94D1F3
:10BD3000E36919079ED509E0236823F0C003236057
:10BD4000E3695B06C7D540232362C4E70823236267
:10BD500090E7B9F1000F8DD089E718F0010F89D075
:10BD6000E3699B077FF57EAF7AE73C06B3D5D5F84C
:10BD70002021D3691806AED5D5E909138B422AD004
:10BD8000A969C95C0133C9B291622A69B3FBF2F1B6
:10BD900002FB1133AB629EE7EB696A69D054EB6931
:10BDA000EA680133B3FBF2F102FB1133EB61ACE75C
:10BDB00095F8B201FEF72AFF236823F008032360F9
:10BDC000012385F8B53100283FF462AF32462021C7
:10BDD000FEF742F95CE7136823F0800313607AE70B
:10BDE000BFF34F8F0549064BCA6802F4E062134364
:10BDF000CB60BFF34F8F00BFFDE700BF00ED00E059
:10BE00000400FA0508B572B6FFF7EAFF70B582B014
:10BE1000FEF7FAFB0320FEF7EBFB01284ED0334C74
:10BE20000025334A0523C4F89850C4F89C50C4F840
:10BE3000A020C4F89430BFF34F8FBFF36F8F4FF63D
:10BE4000FF01E2682B4B0A402B4E13432B4AE36061
:10BE5000536FC6F8203F41F053FC294B2949A3FBFF
:10BE60000023D4F8FC209B0C42F08072C4F8FC2024
:10BE7000C6F8243FD6F82C33234AA1FB03132349E9
:10BE80009B09C2F8B01F5560013B1168B3F1807F78
:10BE900041F00101116007D34FF0E022136943F034
:10BEA0000403136102B070BD4FF0E022F021536132
:10BEB000072384F8231095611361EDE70221032025
:10BEC000FEF79CFB0D4B12485A6C124942F480421B
:10BED0005A645B6C03F480430193019A02680B6817
:10BEE000026083F308884B689847FEE700ED00E0A6
:10BEF0001B0000060005FA059019012000380240D9
:10BF000083DE1B43D34D6210001000E055CEACC55C
:10BF1000003801400000F01F800AA0F58010522870
:10BF20001CD80F4B034493F8F4330D2B16D801396A
:10BF300010B40C4C04EB831CD4F82C438BB2DCF80B
:10BF40001C040CF58461CCF82834B4FBF2F2013AFD
:10BF50005DF8044BCCF8202441F080BE704700BF50
:10BF6000688B05089019012070B50468A30AA3F531
:10BF70008013522B05D82D4E334493F8F4530D2DD6
:10BF800000D970BD2046FDF777F8294BA8010222A1
:10BF900003EB8515D5F81C1485F85924254A8D68BE
:10BFA0002A40062A06D0B2F5803F03D00A6842F044
:10BFB00001020A601A180121002382F859141E494F
:10BFC00051F8332094420AD001330E2BF8D10121CD
:10BFD000002046F0ABFC194B01221A6070BD06EB45
:10BFE000C306012196F9B94896F8B958204646F09B
:10BFF0009DFC002CC5DB05F01F0201216B090F4CD5
:10C0000001FA02F21B2D44F8232006D1192046F034
:10C010008DFC4FF00073236070BD2E2DB1D12C200C
:10C0200046F084FC4FF48053636070BD688B050854
:10C0300090190120070001001C94050800E100E0B0
:10C0400003689B0AA3F58013522B52D8F0B5344CE9
:10C05000234493F8F4330D2B4AD844790225314810
:10C060004FEA831E24FA05FC00EB831605FA0CF553
:10C07000644603EB830CD6F81C6403EB4C0C0029DC
:10C080003BD0A444F4682C4300EB8C0569606A61E2
:10C09000F460EFF3118C502282F312882C2101FB03
:10C0A00003F2845802442CB3211D546203EB830233
:10C0B0001D4D03EB4202920015441032024452F827
:10C0C000044F0CB10C60211DAA42F8D100225FFA86
:10C0D0008CFC0A608CF311882C2202FB03035B6A40
:10C0E000ABB18644DEF81C24D36843F00103D3606F
:10C0F000F0BD704711462431D8E7F768644427EA59
:10C100000505F56000EB840569606A61C1E770446C
:10C11000D0F81C24D36823F00103D360F0BD00BF26
:10C12000688B050890190120B019012003689B0A4B
:10C13000A3F58013522B00D970470F4A134493F88C
:10C14000F4330D2BF8D8022210B40C4C407904EBD8
:10C15000831C20FA02F3DCF81C0402FA03F3C26821
:10C1600029B922EA03035DF8044BC3607047134307
:10C170005DF8044BC3607047688B05089019012077
:10C1800003689B0AA3F58013522B10D8084A134466
:10C1900093F8F4230D2A0AD8407902230549D840A0
:10C1A00001EB82128340D2F81C24DB4313617047F9
:10C1B000688B05089019012001490248FCF738BE38
:10C1C000901901200000014010B5064C0648214698
:10C1D000FCF72EFE04F5C6710448BDE81040FCF7DC
:10C1E00027BE00BF9019012000000140004401401B
:10C1F00002494FF08040FCF71BBE00BFBC19012074
:10C2000001490248FCF714BEE8190120000400406F
:10C2100001490248FCF70CBE141A01200008004036
:10C2200001490248FCF704BE401A0120000C0040FE
:10C23000F8B5164D164E2A69EB681A404FF00040CB
:10C24000B2FA82F3EAB120FA03F3012A6FEA030398
:10C2500002EA03012B610A46F2D1D6F804718FB1CC
:10C26000013F0023BFB2C6F80431D6F8004134B113
:10C2700023682046394698476468002CF8D100228C
:10C28000DCE7F8BDEF6ABFB2EFE700BF0010004087
:10C290009019012001490248FCF7CABDC41A0120C7
:10C2A0000004014010B5064C064804F59A71FCF7ED
:10C2B000BFFD04F504710448BDE81040FCF7B8BDAB
:10C2C0009019012000040140001C0040014902486F
:10C2D000FCF7AEBDF01A01200040014001490248C0
:10C2E000FCF7A6BD481B0120004801400149024857
:10C2F000FCF79EBD741B0120001800402DE9F041A1
:10C300004FF425728EB000215E484CF06FF95E4B01
:10C310005E4D4FF000085A6C40F22227A5F6241615
:10C32000A5F1700442F001025A645A6C02F0010255
:10C330000092009A1A6C42F001021A641A6C02F020
:10C3400001020192019A1A6C42F002021A641A6CFC
:10C3500002F002020292029A1A6C42F004021A647B
:10C360001A6C02F004020392039A1A6C42F008025B
:10C370001A641A6C02F008020492049A1A6C42F0D1
:10C3800010021A641A6C02F010020592059A1A6CD7
:10C3900042F020021A641A6C02F020020692069AF9
:10C3A0005A6C42F002025A645A6C02F0020207927E
:10C3B000079A5A6C42F480325A645A6C02F4803202
:10C3C0000892089A5A6C42F400325A645A6C02F489
:10C3D00000320992099A5A6C42F480225A645A6CCB
:10C3E00002F480220A920A9A1A6C42F040021A64FD
:10C3F0001A6C02F040020B920B9A1A6C42F0800207
:10C400001A641A6C02F080020C920C9A1A6C42F4B4
:10C4100080721A641B6C03F480730D930D9B55F8A6
:10C420002810002354F83320914226D001330E2BDC
:10C43000F8D1002008F1070846F01AFBB845EED104
:10C440004FF0000840F2222755F82810002354F836
:10C45000332091420CD001330E2BF8D1002008F18B
:10C46000070846F005FBB845EED10EB0BDE8F081F7
:10C4700006EBC30393F8B808F1E706EBC30393F8A0
:10C48000B808D7E790190120003802408C940508BD
:10C49000800AA0F5801052280ED8084B034493F868
:10C4A000F4230D2A08D8064B03EB8213D3F81C247F
:10C4B000136843F001031360704700BF688B0508E1
:10C4C0009019012037B590F867380446032B2FD117
:10C4D0000023204D8DF807309DF8073094F8682828
:10C4E0009A4201D803B030BD9DF8073005EBC30375
:10C4F00093F82C3F8BB181F0010383B19DF8073095
:10C5000005EBC303D3F8280FFDF7C4FB9DF80730F4
:10C510000133DBB28DF80730DEE70B46EDE79DF81F
:10C52000073005EBC303D3F8280FFDF7B9FBEDE7A0
:10C53000D0E910039B7903F00103994204D003B0C2
:10C54000BDE83040FDF7A6BB03B0BDE83040FDF7C5
:10C55000A7BB00BF9019012038B5044600790D46ED
:10C5600050B1FEF753FB08B10323C380E27929469B
:10C57000BDE83840FDF748BE38BD10B5044622215D
:10C58000FFF7EAFF2046FFF7FBFD20460121BDE84B
:10C590001040CBE510B504460121FFF7DDFF002177
:10C5A0002046BDE81040C1E538B510F8133CA0F6B0
:10C5B0006C041BBB94F858388BBBD4E909239A420E
:10C5C0001CD05A1CA169A262CB5C21695B008A4223
:10C5D00028BF002243F40073A262A4F85C380A2347
:10C5E00084F85A38012384F8583894F86738012BB6
:10C5F00001D0042B02D1606CFFF7CCFF94F85438C3
:10C60000002B6DD194F855380133DBB2092B84F837
:10C61000553825D12046BDE83840FBF781BE94F956
:10C620005A586DB1B4F85C18013D20464B0801F032
:10C630000101A4F85C38FFF745FF84F85A58DDE79C
:10C64000D4E9092384F858589A42D7D194F8673826
:10C65000012B01D0042BD1D1606CFFF78EFFCDE709
:10C660000A2B3DD194F857382BB9B4F85E3843F013
:10C670000103A4F85E382379D9070AD5B4F85E0817
:10C68000820501D4C30718D4B4F864380133A4F880
:10C6900064380122002384F8542894F8572884F839
:10C6A0005538012A1CD16179606C84F8573801F043
:10C6B0000101BDE8384048F025BBE36AC0F34700FC
:10C6C00013B1216B9847E4E7E3696269D054E369E9
:10C6D000E2680133B3FBF2F102FB1133E361D8E707
:10C6E00038BD00BF2DE9F041A14CA4B0D4F85C38AE
:10C6F000022B00F030829F489F4AA049121A4BF04B
:10C700007FFE9F489F4AA049121A4BF079FED4F849
:10C710005838012B00F2C08003EB43039B4A9C4E28
:10C7200002EB430032F8132041888388C6E9AF2129
:10C73000C6F8C432974C984D984BB2FBF1F2984929
:10C7400001FB02F20021C5F82C23D4F8882042F422
:10C750007002C4F888201A6842F001021A609960D9
:10C76000904A1868024090481A60C0F308078F4A40
:10C770005A601A6822F480221A60D96007B1FEE775
:10C780008B49A0604FF6FF000A688A4B42F40072A2
:10C790000A60E26802401343E36046F079FCBFF3AD
:10C7A0004F8FBFF36F8FC4F85072BFF34F8FBFF33B
:10C7B0006F8F636943F400336361BFF34F8FBFF33F
:10C7C0006F8FC4F88470BFF34F8FD4F8803043F676
:10C7D000E07CC3F3C90EC3F34E33580100EA0C01E9
:10C7E000734641EA8372013B5F1CC4F86022F8D1B2
:10C7F000203810F1200FF1D1BFF34F8F636943F45C
:10C8000080336361BFF34F8FBFF36F8F6849634B12
:10C810000A6842F480720A60196C674A41F08051DC
:10C820001964196C01F0805102910299116841F468
:10C83000404111601268D6F8BC4202F440420192B5
:10C84000019A9A6802F00C02042AD6E9B07100F04D
:10C850008B809A6802F00C02082A00F081804F4A0F
:10C86000136843F480331360D5F8680F04E0D5F8FB
:10C87000683F1B1A642B72D813689B03F7D5474A8D
:10C88000936803F00C03082B69D0136823F08073BE
:10C890001360D5F8680F08E03D4ED6E9AF2149E7AF
:10C8A000D5F8683F1B1A022B59D813689E01F7D49C
:10C8B0000B06790843EA8413013943EA01433F49EF
:10C8C00019435160136843F080731360334AD5F8FD
:10C8D000681F04E0D5F8683F5B1A022B3FD8136845
:10C8E0009801F7D5136C43F080531364136C324AEC
:10C8F00003F080530393039B136843F48033136066
:10C90000D5F8681F05E0D5F8683F5B1AB3F57A7F64
:10C910002DD85368DB03F6D51368274943F4003359
:10C920001360D5F8682F05E0D5F8683F9B1AB3F57A
:10C930007A7F1CD84B689E03F6D54FF400124FF057
:10C94000006304A804924FF4C07221930723CDE939
:10C95000082303230A9340F0F9FE88B3FEE7FEE7BD
:10C960005B685A027FF57BAF0C4B1B6887E7FEE7DD
:10C970000020004000000000683C000030A90608CC
:10C9800000000020A8010020230B0708149D0508C3
:10C990000000012000ED00E0901901200038024065
:10C9A00040420F00FFFFF6FE000000081030002498
:10C9B000003C02400003FA050070004010004020D7
:10C9C000684A136803F00F03062B0AD8136823F094
:10C9D0000F0343F007031360136803F00F03072BE3
:10C9E00069D1614B9A6842F4E0529A609A6842F4C5
:10C9F00060429A609A6822F0F0029A601A68900188
:10CA000059D59A6841F2883022F0030242F00202BE
:10CA10009A60D5F8681F04E0D5F8682F521A824250
:10CA200049D89A6802F00C02082AF5D14D4A1368D9
:10CA300019070AD5136823F00F0343F007031360A7
:10CA4000136803F00F03072B35D1DFF81C81474E25
:10CA5000D8F8083023F4E05343F4A053C8F8083062
:10CA6000D8F8083023F4604343F40043C8F8083092
:10CA700040F046FED8F80830C3F30313334493F86C
:10CA8000C03020FA03F3C5F82C3346F001FB002335
:10CA900004A8CDE91333CDE91533CDE91733CDE93A
:10CAA0001933CDE91B33CDE91D33314B049340F0ED
:10CAB0004DFE08B1FEE7FEE702234FF0007204A826
:10CAC000CDE90633D823CDE9042301230B9340F0AD
:10CAD0003DFE00B1FEE7D8F88C3023F08073C8F833
:10CAE0008C30D8F88C3043F08073C8F88C30D8F88C
:10CAF000083003F00C03082B12D01E4B1E49B4FB68
:10CB0000F7F201FB02F218498968C1F303110E44E0
:10CB100096F8C010CB409A42C5F82C3318D0FEE7E7
:10CB2000D8F80430D8F80420124902F03F02D8F8AF
:10CB30000430B1FBF2F2C3F3881302FB03F30A4A99
:10CB40005268C2F3014201325200B3FBF2F3D5E75F
:10CB500024B0BDE8F08100210320FDF74FFDFFF771
:10CB60003FF900BF003C024000380240609C0508CD
:10CB7000C0FF03000024F40040420F0010B4EFF3A4
:10CB80001182102383F312880C4B4FF0E020002415
:10CB9000D2B2D3F8D4120131C3F8D4128169C3F8E8
:10CBA0006C1FC3F8704F016982F31188D3F8682FA6
:10CBB0005DF8044B0132C3F8682F704790190120CB
:10CBC00010B4EFF31181102383F312884FF0E022A9
:10CBD0009469136913F4803F0D4B03D00120C3F80F
:10CBE000700F9469D3F8D402C9B2D3F8702F81F3CF
:10CBF00011880244D3F8241F4FF47A7000FB01F32C
:10CC00001B1B5DF8044BB3FBF1F300FB02307047D4
:10CC100090190120134B5B68C3F3080303BBEFF3C8
:10CC20001183EBB9104B4FF0E02C10B4D3F8D422A1
:10CC3000DCF81800D3F8D4128A42F7D1D3F86C1F6D
:10CC40008842F3D8D3F8244F4FF47A7101FB04F3F0
:10CC50001B1AB3FBF4F35DF8044B01FB0230704781
:10CC6000AEE700BF00ED00E0901901202DE9F04F84
:10CC7000374C83B023781BB9012003B0BDE8F08F97
:10CC8000344F04F58764DFF8D0B04FF0000AD7F8CE
:10CC9000D4324FF6FF7894F8C0910BF53875ABF5A8
:10CCA000F166019314E0B0F5606F43D0A881B0EB5A
:10CCB0000801019A584618BF01210CF0C5FD0AF180
:10CCC000010A0BF15C0B20341435BAF1080F2AD09D
:10CCD000CA4528D0A0696268D0E93D014BF008FF41
:10CCE0004FF6FE7397F8752F984214D0542A04D14A
:10CCF000B7F8782F0132A7F8782FD6F8702A404578
:10CD000002F10102C6F8702ACDD1D6F86C2A0132A0
:10CD1000C6F86C2ACBE7542AD1D1B7F87A2F013262
:10CD2000A7F87A2FCBE70123012086F86C3B03B0EC
:10CD3000BDE8F08F97F8D42302EB420207EBC20262
:10CD4000524492F881230D2AB0D18022AA77AEE70F
:10CD5000A801002090190120281A002070B54BF07E
:10CD6000E3FE80B31A484568002D10DD002410F85A
:10CD7000086B16B1037F012B1FD04269013400F507
:10CD800086701368AC4243F001031360F1D1FFF7E2
:10CD900041FF104BD3F88447002C0DDD03F2647380
:10CDA00003EBC4041968083333F8042CC868A342A1
:10CDB00042EA0002CA60F5D170BD002380F8FC3061
:10CDC000FBF7C0F9D9E749F089FB0028CAD170BD4B
:10CDD000A8010020A01200202DE9F04F894C87B057
:10CDE00023781BB9012007B0BDE8F08F864BD3F83C
:10CDF000D4320493FFF70EFF94F8F8250192002A2D
:10CE000000F0F880814A04F5C0640027D2F8783B2E
:10CE100002F5F16B02F6682A2646A0EB030805949A
:10CE2000B8F1000F03DBF36D434500F3C98007EB56
:10CE30008703744A02EB431393F8583603F0FF0E4E
:10CE4000002B00F08780D6F89410B36870481A68F9
:10CE5000CBB221F0FF01103BA0FB03036D481B097F
:10CE6000C35C0B44B1895C68D368A4B223EA0103B4
:10CE7000C4F11604D360072C6CD9644A0121D2F89E
:10CE8000703A89460133C2F8703A0022D6F89C30D5
:10CE9000154618689C46CDE902E715E0142D1EDC06
:10CEA00017F1080E48BF07F1170E4FEA2E1705EBD2
:10CEB0002E1507F1FF3E013102FA07F709FA0EFEBF
:10CEC0008C424EEA07020AD307468C425CF8040FF4
:10CED000A0EB0707E2D8C5F115071525E9E7152DE1
:10CEE000DDE902E762D14C4CC2F38421C2F3441065
:10CEF00004EB810104EB8000D1F85011D0F850010F
:10CF0000090241EA001102F01F00C2F3C43204EB2F
:10CF1000800004EB8202D0F85001D2F85021014386
:10CF200041EA023282EA122181EA111101F00F0175
:10CF30000F293BD1C2F30F124FF6FF718A4235D051
:10CF4000B2F5606F40D0AAF80C207146049A58469A
:10CF50000CF07AFC30460137FDF7A2FB019BA036AE
:10CF60000BF15C0BBB420AF1140A7FF459AF019B31
:10CF70000121059C002203EB8303244804EB4313A7
:10CF800080F86C1BC0F8782BA268A03414F8901CB1
:10CF9000126854F84C0C11F0020F116A14BF41EAE8
:10CFA00080010143A3421162EED11BE71749D1F87A
:10CFB0006C2A0132C1F86C2AB7B14FF0000EC4E7F9
:10CFC000002007B0BDE8F08F0F4991F8D43303EB90
:10CFD000430301EBC3033B4493F881330D2BB2D1E0
:10CFE00080238AF81E30B0E7194658220B484BF0D0
:10CFF00007FAE2E7054B0122019983F86C2BC3F88D
:10D00000781BEFE6A801002090190120A012002053
:10D01000ABAAAAAA900F0608609C0508B41D0020C0
:10D020002DE9F0472F4FFFF7F5FDDFF8C090804660
:10D030007E6800202C4C002E48DD00234FF48671C2
:10D040001D4601FB0372013392F805219E4245EA19
:10D050000205F6D128435FFA80FAD9F80430C3F309
:10D06000080383BBEFF311836BBB4FF0E02CD4F8C4
:10D07000D432DCF81810D4F8D4229342F7D1D4F883
:10D080006C2F9142F3D8D4F824CF4FF47A7202FB7C
:10D090000CF0401AB0FBFCF002FB0300A0EB08030D
:10D0A000B3F5FA6FCCBF002005F001000028C2D113
:10D0B000BAF1000F04D00C4B93F8752F542A08D006
:10D0C0005046BDE8F087FFF77BFDE7E78246002585
:10D0D000C3E7B3F87C2F50460132A3F87C2FBDE89C
:10D0E000F08700BFA80100209019012000ED00E0AA
:10D0F0002DE9F04F874C83B00746D4F8E09294F8BE
:10D10000E8320191B9F1000F0BD083F00202B9F8B7
:10D110000410C2F34002120101FA02F2D9F8001021
:10D120008A61D4F8DC82B8F1000F09D003F0010362
:10D13000B8F804201B0102FA03F3D8F80020936129
:10D14000013F754E4FF0E0254FF47A7BFBB2009320
:10D15000B9F1000F08D0D9F80010B9F804304869C7
:10D16000034218BF1B048B61B8F1000F00F0C980A7
:10D17000D8F80010B8F80430486903424FF00100B5
:10D1800018BF1B048B610DF019F8DDF804A073685B
:10D19000C3F30803002B40F0B080EFF31183002BA2
:10D1A00040F0AB80D4F8D472A869D4F8D4128F427E
:10D1B000F8D1D4F86C1F8842F4D8D4F8243F0BFB84
:10D1C00003F1091AB1FBF3F10BFB07177368C3F303
:10D1D0000803002B40F08A80EFF31183002B40F00E
:10D1E0008580D4F8D432A969D4F8D4028342F8D126
:10D1F000D4F86C0F8142F4D8D4F8242F0BFB02F042
:10D20000401AB0FBF2F00BFB0300C31BB3F57A7FAF
:10D21000DCD3BAF1010ABAD1B9F1000F08D0D9F8BC
:10D220000010B9F804304869034218BF1B048B6131
:10D23000B8F1000F69D0D8F80010B8F80430486988
:10D2400003424FF0000018BF1B048B610CF0B6FFC7
:10D25000DDF804A07368C3F30803002B49D1EFF392
:10D260001183002B45D1D4F8D472A869D4F8D41214
:10D270008F42F8D1D4F86C1F8842F4D8D4F8243FF8
:10D280000BFB03F1091AB1FBF3F10BFB07177368F2
:10D29000C3F308033BBBEFF3118323BBD4F8D432B1
:10D2A000A969D4F8D4028342F8D1D4F86C0F814232
:10D2B000F4D8D4F8242F0BFB02F0401AB0FBF2F0A4
:10D2C0000BFB0300C31BB3F57A7FE0D3BAF1010A6D
:10D2D000C0D1009B5F1EFBB2FF2B00937FF438AFE1
:10D2E00003B0BDE8F08FFFF76BFCEBE7FFF768FCDE
:10D2F0008BE7FFF765FC0746C9E7FFF761FC0746C8
:10D3000064E701200CF05AFF3FE740460CF056FF5F
:10D310009EE700BF9019012000ED00E02DE9F041EB
:10D320000746DFF86080FFF775FC154C4FF0E025ED
:10D330000646D8F80430C3F30803EBB9EFF31183C2
:10D34000D3B9D4F8D432A969D4F8D4229342F8D10D
:10D35000D4F86C2F9142F4D8D4F824CF4FF47A72D9
:10D3600002FB0CF0401AB0FBFCF002FB0300831B35
:10D37000BB42DED3BDE8F081FFF722FCF7E700BF38
:10D380009019012000ED00E02DE9F041294F461EE3
:10D39000294C7B68C3F30803002B47D1EFF31183BB
:10D3A000002B43D14FF0E020D4F8D4328169D4F877
:10D3B000D4229342F8D1D4F86C2F9142F4D8D4F807
:10D3C000240F4FF47A7202FB00F8A8EB0108B8FBB7
:10D3D000F0F802FB03884FF0E0257B68C3F30803F5
:10D3E0000BBBEFF31183F3B9D4F8D432A969D4F8A5
:10D3F000D4229342F8D1D4F86C2F9142F4D8D4F8C7
:10D4000024CF4FF47A7202FB0CF0401AB0FBFCF010
:10D4100002FB0300A0EB0803B3F57A7FDDD3013EE6
:10D42000B7D2BDE8F081FFF7CBFBF3E7FFF7C8FB0E
:10D430008046D0E700ED00E09019012001302DE991
:10D44000F0475D4E4D1E5D4C5FFA80FA4FF4FA775F
:10D4500032210520FFF74CFE7368C3F30803002B4D
:10D4600040F0A180EFF31183002B40F09C804FF03F
:10D47000E020D4F8D4328169D4F8D4229342F8D190
:10D48000D4F86C2F9142F4D8D4F8240F4FF47A7268
:10D4900002FB00F9A9EB0109B9FBF0F902FB0399C2
:10D4A0004FF0E0287368C3F30803002B78D1EFF343
:10D4B0001183002B74D1D4F8D432D8F81810D4F8D2
:10D4C000D4229342F7D1D4F86C2F9142F3D8D4F8F8
:10D4D00024CF4FF47A7202FB0CF0401AB0FBFCF040
:10D4E00002FB0300A0EB0903B3F57A7FDAD3013F17
:10D4F000B2D14FF47A77FA215046FFF7F9FD7368FD
:10D50000C3F30803002B52D1EFF31183002B4ED14C
:10D510004FF0E020D4F8D4328169D4F8D422934279
:10D52000F8D1D4F86C2F9142F4D8D4F8240F4FF4EA
:10D530007A7202FB00F9A9EB0109B9FBF0F902FBD1
:10D5400003994FF0E0287368C3F308032BBBEFF394
:10D55000118313BBD4F8D432D8F81810D4F8D422DD
:10D560009342F7D1D4F86C2F9142F3D8D4F824CF5A
:10D570004FF47A7202FB0CF0401AB0FBFCF002FB95
:10D580000300A0EB0903B3F57A7FDCD3013FB6D1EA
:10D59000013DBFF45BAFBDE8F087FFF711FBF0E79B
:10D5A000FFF70EFB9EE7FFF70BFB814678E7FFF7DF
:10D5B00007FB8146C5E700BF00ED00E090190120A0
:10D5C000431C0A265D4D5E4C5FFA83FA80B54FF42A
:10D5D000FA7832210520FFF78BFD6B68C3F308034F
:10D5E000002B40F09F80EFF31183002B40F09A80D6
:10D5F0004FF0E020D4F8D4128369D4F8D4229142B9
:10D60000F8D1D4F86C2F9342F4D8D4F8240F4FF407
:10D610007A7202FB00F7FF1AB7FBF0F702FB017703
:10D620004FF0E0296B68C3F30803002B7ED1EFF3C2
:10D630001183002B7AD1D4F8D402D9F818C0D4F8C9
:10D64000D4329842F7D1D4F86C3F9C45F3D8D4F843
:10D65000241F4FF47A7202FB01F3A3EB0C03B3FB1C
:10D66000F1F302FB0033DB1BB3F57A7FDAD3B8F1B9
:10D670000108B2D14FF47A78FA215046FFF738FD0D
:10D680006B68C3F30803002B48D1EFF31183002B21
:10D6900044D14FF0E020D4F8D4128369D4F8D422D6
:10D6A0009142F8D1D4F86C2F9342F4D8D4F8240FD7
:10D6B0004FF47A7202FB00F7FF1AB7FBF0F702FB98
:10D6C00001774FF0E0296B68C3F3080393BBEFF3D6
:10D6D00011837BBBD4F8D402D9F818C0D4F8D43263
:10D6E0009842F7D1D4F86C3F9C45F3D8D4F8241F66
:10D6F0004FF47A7202FB01F3A3EB0C03B3FBF1F3DB
:10D7000002FB0033DB1BB3F57A7FDCD3B8F10108F1
:10D71000B6D1013E7FF45BAF44F048FEFFF750FA0C
:10D720000746CEE7FFF74CFA074679E7FFF748FAD6
:10D73000034698E7FFF744FA0346E3E700ED00E00D
:10D740009019012038B5094C04F5407502E0083401
:10D75000AC420AD094F90620002AF8D120460834B9
:10D760002021FCF779FCAC42F4D138BD3C230120E8
:10D77000094B02460220D3F82C13B2EB910F4FEA6B
:10D78000910307D25B0840009A4280B202D2FF2880
:10D79000F8D97047704700BF901901202DE9F04F6C
:10D7A0007F4E85B0DFF814B24FF0010A4FF0000948
:10D7B0007C4D09E009F101090AF1010A28360BF153
:10D7C000050BB9F1040F34D03378022BF2D19BF959
:10D7D0000330591C00F0CE80DAB296460C230820A4
:10D7E0005FFA89F1039613FB0200D3B2012B17D81D
:10D7F0006D4B02E01C33AB4212D01C78002CF9D1E7
:10D800005E788E42F6D11E58002EF3D0674FB44694
:10D8100002977E6801342437B4450DD0102CF8D11E
:10D8200001320C30D3B29E45E0D20023039E019317
:10D8300027E005B0BDE8F08FE4B25D4E671E0194AD
:10D8400007EBC70406EB840CA4009CF99880B8F1A0
:10D85000000FE5D102EB420207F00707019803EB46
:10D8600082038CF884708CF899A0DB68DDE90216DD
:10D87000CCF88830142321448CF898303161FCF7BF
:10D8800061FB9BF904305A1C70D0D9B288460C2336
:10D8900008275FFA89F0039613FB0177CBB2012BBF
:10D8A00018D8414A02E01C32AA4213D01378012B47
:10D8B000F9D153788342F6D1D659002EF3D03B4BA1
:10D8C0000024B44602935E6801342433B44521D069
:10D8D000102CF8D101310C37CBB24345DFD9019B75
:10D8E000039E002B3DD0019F2422304800247B1E44
:10D8F000746102FB03003061FAF7C4FB3046FAF7AB
:10D9000093FB2346224638462A49FCF73DFB012378
:10D9100033734FE7E4B2264E631E03EBC30E06EBF0
:10D920008E0C4FEA8E0E9CF99860002ED2D101EB3E
:10D93000410103F0070337468CF899A002EB8102FE
:10D940008CF88430DDE90206D3687044CCF8883066
:10D950001323706120468CF89830FCF7F3FA019B92
:10D9600063B900220023C6E9042323E74FF001082E
:10D9700000218CE74FF0010E00222FE77069FAF7C3
:10D9800081FB3069FAF77EFB3046FAF74DFB3B46E8
:10D990003A4620460849FCF7F7FA0123337309E7B2
:10D9A00020290120C4920508409005087C00012030
:10D9B000000001204D930008C1920008C0290120F9
:10D9C00070B50E494FF0010E0D4D0E4C0E4E35F850
:10D9D00002CB00234CFA03F20EFA03F0013312F0EB
:10D9E000010F03D00C60083121F8040C102BF1D189
:10D9F00004F58064B442EAD170BD00BF3C2301202D
:10DA0000D492050800000240001802402DE9F047BA
:10DA10000646086888B00C46850ABDF84080A5F522
:10DA200080159DF844A0522D55D819462D4B2B44F6
:10DA300093F8F4530D2D4ED82B4FFBF71DFB94F8A4
:10DA4000059007EB8517A379BAF1000F01D083F099
:10DA500001035A004FF48071DB00384602F00202E5
:10DA6000CDF8088003F0080303924A46049360232C
:10DA700001934FF40073CDE90613002301A9059328
:10DA800044F09CFCA379384649469F0726D440F0D1
:10DA9000B5F8164BA801022203EB8515D5F81C1426
:10DAA00085F85924124A8D682A40062A06D0B2F514
:10DAB000803F03D00A6842F001020A600344012259
:10DAC00083F859242168637901F1340271600021DF
:10DAD000D0183060D15008B0BDE8F08740F0A2F90E
:10DAE000D7E700BF688B0508AC1D01209019012005
:10DAF000070001000548D0F8A03223B1DB6A13B15A
:10DB000000F5287018470248704700BF901901209F
:10DB1000309E050838B5184C54F8B43C1B8843B9FE
:10DB2000164D002304F8A53C85F89832C5F89432C8
:10DB300038BD54F8B02C002AF2DD54F8AC1C012A90
:10DB4000488806D001230D4D24F8A80C04F8A63C03
:10DB5000E7E78A880132121A9A42F3D1074D002270
:10DB6000D5F8A03205F52870C5F8CC221B69984776
:10DB700048F03CFFD5E700BF882A0120901901201A
:10DB80000748D0F89C321BB1064B13F8A63C0BB1EA
:10DB900000207047D0F8A03200F528705B68184765
:10DBA00090190120882A0120184A10B4184C92F8C4
:10DBB000983244602344174C036092F8980214F89A
:10DBC000A53C834218D892F89802834207D30023D9
:10DBD0005DF8044B1A461846C1E90032704792F8C6
:10DBE00098021A1E5DF8044BC0F180030CBF01209F
:10DBF0000220C1E90032704792F8984200220120C9
:10DC00001B1B5DF8044BC1E90032704790190120DD
:10DC10001C1E0020882A0120104B114A93F89812EC
:10DC200012F8A50C93F89822904293F898220FD8F6
:10DC3000904204D3D3F8943200201844704793F8EC
:10DC40009822D3F89432C2F18002104418447047ED
:10DC5000801AD3F894321844704700BF90190120FD
:10DC6000882A012038B5144D144C55F8B42C937BF8
:10DC7000012B08D0D4F8943203F2FF736FF30A0338
:10DC8000C4F8943238BDD4F8A0325B6A33B104F5DD
:10DC90002870984748F0AAFE55F8B42CD4F894326E
:10DCA0005288013B514213440B4003F2FF736FF360
:10DCB0000A03C4F8943238BD882A01209019012043
:10DCC000F0B51C4C85B01C4B94F898221B4D039367
:10DCD000134415F8A51C94F898220293914294F8E5
:10DCE000983216D899420CD294F898620F46C6F131
:10DCF0008006D9B9334601223F2BCDE900670DD804
:10DD000060B994F89802401AB0FA80F0400905B062
:10DD1000F0BDCB1A002701221E46EDE7694600231D
:10DD200002A848F011FE15F8A51CEAE773180222B4
:10DD3000E2E700BF901901201C1E0020882A012064
:10DD40002DE9F047174684B000293ED0441E294DE6
:10DD5000DFF8AC904FF0000A04EB0108264E0DE00E
:10DD600096F898320846994296F898321DD2C3F137
:10DD7000800318443F281BD8A04526D015F8A50CD1
:10DD800014F8013F411C4844C9B280F87C3B0B06A3
:10DD900005F8A51CE4D5002096F8983205F8A5AC46
:10DDA0000146994296F89832E1D3C01A3F28E3D948
:10DDB00096F898329942DFD0104B5B78002BDBD07D
:10DDC0000020FFF77DFFA045D8D1694602A8FFF7E4
:10DDD000EBFEDDE9003213443F2B00D910B904B04B
:10DDE000BDE8F08702463B4602A848F0ADFD04B00E
:10DDF000BDE8F087882A0120901901200000012049
:10DE0000A012002030B585B0694602A8FFF7CCFE0D
:10DE100058B9094C04F52875D4F8A03228465B6837
:10DE200098470028F8D005B030BD0246012302A86B
:10DE300048F08AFDEDE700BF9019012038B50023B6
:10DE4000124C134DC5F89C3244F07EF944F8AC0CEA
:10DE5000FFF750FE54F8AC3C44F8B40CA3B19A88D8
:10DE60005B88D21A436802FB0333C5F89C32FAF789
:10DE70001FFC14F8A52C044695F898329A4201D05C
:10DE8000FFF7C0FFC5F8944238BD00BF882A0120C3
:10DE9000901901202DE9F041104E154682180446D4
:10DEA000D6F89C320F469A420D4A88BF1D1A12F8C6
:10DEB000A52C96F898329A4201D0FFF7A3FF0020D4
:10DEC00021462B463A46C6F8CC02D6F8A002846A10
:10DED0000448A446BDE8F041604700BF9019012006
:10DEE000882A0120301C01208C46134601466246D8
:10DEF0001846CFE72DE9F043484F93B0484DFFF760
:10DF000009FE97F8983215F8A52C9A4201D0FFF730
:10DF100079FF0024D7F89C62C7F89442002E6DD098
:10DF2000DFF800810AE097F8983215F8A52C9A429C
:10DF300001D0FFF767FF2034A6421BD92246414695
:10DF4000684601F0F7FA684648F004FE01220146EF
:10DF50006846FFF7F5FEA3B2002BE4D1D7F8DC3218
:10DF6000002BE0D09A881B6859690A4218BF120436
:10DF70009A61D8E7FFF776FE97F8983215F8A52C46
:10DF80009A4201D0FFF73EFF0023DFF898909846B1
:10DF90001C46C7F894322246494609A801F0CAFA3D
:10DFA0002122002168464AF021FB202269462046B2
:10DFB000FFF770FF2022054609A968464AF04BFB8F
:10DFC000A3B2203450B9202D08D15BB1A642E2D8CB
:10DFD000B8FA88F0400913B0BDE8F08308F10108F1
:10DFE000002BF3D1D7F8DC32002BEFD01A689B88D6
:10DFF00051690B4218BF1B049361E7E7FFF732FE3C
:10E0000097F8983215F8A52C9A4201D0FFF7FAFE3E
:10E0100000230120C7F89432DDE700BF90190120EA
:10E02000882A0120000F06080B4B93F8CC221AB95E
:10E030000A4A12F8A40C70470949D1F85C28032A4F
:10E04000F6D10020054A4FF0010C83F8CC0202F80B
:10E05000A4CCC1F85C08ECE700000120882A01206C
:10E060000020004008B50322104BC3F85C2872B6AC
:10E070000F4B53E9281251EA020308D100231A4634
:10E080000A49C1F86028C1F86438FDF7BBFE094BA6
:10E090004EF6602CD3F8D4320CFB00F05B1842F142
:10E0A0000002C31842EBE072EAE700BF0020004024
:10E0B000882A0120901901200021032008B5FCF7CF
:10E0C0009DFA72B6FDF78CFE154C08B554F8983CD5
:10E0D00014F8920CABB91420FFF756F900BF54F8AE
:10E0E000983C5BB1196814F8922C9B8809690B4025
:10E0F00012B91BB1FFF7E0FF002BFBD0FAF70CFBC6
:10E10000ECE719689A880B69134020B1002BE2D123
:10E110000B691340FAE7002BDDD00B691340FAE7D7
:10E12000882A0120F8B540F097FF1B20FCF76EFD10
:10E1300008B12923C3801C20FCF768FD08B12923FE
:10E14000C380144CD4F8FC3113B10023C4F8FC3163
:10E15000114E01250027C4F8F86184F8E45104F851
:10E16000907C47F097FA06F11C03C4F8FC3194F850
:10E170002132AB4201D02846F8BD5436D4F81802FB
:10E18000C4F8146247F072F8044B384683F82370E1
:10E19000F8BD00BF882A0120D002012000ED00E078
:10E1A0002DE9F04F00218BB041F69462B8484AF057
:10E1B0001DFA0420FCF71CFA01460520FCF718FAAA
:10E1C00051EA000340F05781B24B03934C220021E7
:10E1D000AF4801244AF00AFA00214C22AC484AF028
:10E1E00005FA039BAA4AD3F87433AB4D1646147153
:10E1F0001560D3611362536244F06AFFFFF71EFE9D
:10E20000002108460BF09AFEFAF752FAB0F1000826
:10E2100040F39B810024A14DDFF8A4E206F14C09F4
:10E220002746A24605F5097B9D4E0294CDF804E0F1
:10E2300004E00AF5006AD04540F3AE80019AD2F8B6
:10E24000D432C2F8D832FAF767FA2022594650463B
:10E25000FFF720FE1222934958464AF0FCF90028A5
:10E26000E7D1BA4525D002998F4B01EB410203EB70
:10E2700082034A1C8D4918460293AAEB07030592B4
:10E28000049301F057F9029B4946059A41F84C3B2B
:10E29000049BC9F80C700292C9E90433D9F81C3008
:10E2A000C9E908330123C9F80830814BC9F828307F
:10E2B0008946039B57461222D3F87433C9F81C30A1
:10E2C000A918335D013291F8241299420BD0002431
:10E2D000202AF5D120375946B845384653DBFFF799
:10E2E000D9FD0022ECE70134152CF1D1D019714F82
:10E2F00020223946FFF7CEFD384600230A2209A91D
:10E30000099701F025FA0746099800230A2209A96E
:10E310000130099001F01CFA0790002309980A22A5
:10E3200009A90130099001F013FA06900023099819
:10E330000A2209A90130099001F00AFA059009A9F9
:10E34000099800230A220130099001F001FA002304
:10E35000049009980A221946013001F0F9F997B1A1
:10E360000599DDE9063243EA4212049B5B0143EA68
:10E37000C123A7F2BC7143EA600342EA412243EAA7
:10E380000243C9F81C30029B642B43D057460AF560
:10E39000006AD0453FF752AF029B642B1ED0BA45AE
:10E3A0001CD00C22404C5E1C404902FB0344AAEBEB
:10E3B00007053246204601F0BDF8D9F81C20C9F8FF
:10E3C0000040C9F80C700296C9E908220122C9F878
:10E3D0000820374AC9E90455C9F82820029B002BB8
:10E3E00003F1010117DC4FEA4803B3F1805FC0F28B
:10E3F000AD80274B9C6834B91A461B791BB1136852
:10E40000002B40F0D980002108460BB0BDE8F04F4A
:10E410000BF094BD65214C261D48DFF8A8A04FF0F5
:10E42000010906FB01F432460021234F0519284655
:10E430004AF0DCF83246002128464AF0D7F81C4E54
:10E44000134804F1100204F11803029940F804A0E3
:10E45000C5F8089002312F62AE6240F80280024493
:10E460000430C2F80480039AD2F87423C2500344E3
:10E470005A606A62B7E74FF47A72002348F072FB81
:10E480000E4B40F2B27240F26D14B0FBF3F31DE09C
:10E49000383201200000012044810608882A01202A
:10E4A000440F0608200F0608CC2C0120340F060864
:10E4B000E9DE0008AC2C01200068214C80510100ED
:10E4C000901901205C0F06085B1A013212F0030557
:10E4D00014BF21464FF4B7718B42F5DA8549002D00
:10E4E00064D003910399D1F844138B42C0F29C800D
:10E4F000814D01245B1A55F8041F01349942F9DD5E
:10E500000133A2F2BC72039D43EA44133C2443EA64
:10E5100042237A4AB0FBF2F102FB11024FF4616030
:10E52000B2FBF0F100FB11221C20C5F84803B2FB3E
:10E53000F4F004FB1022521042EA401242EAC122D7
:10E5400042EA0343C5F8743340E621464C266C4B3F
:10E55000DFF8B891012706FB01F4324600214FF0A5
:10E56000020A1D1928464AF041F832460021284681
:10E570004AF03CF8624B039A04F1180143F8049006
:10E58000C8F10063D2F8740304F11002BB405C4C84
:10E590005C4E85F805A0AF602E62A3502244536004
:10E5A000231D585019444860686222E70C460391C5
:10E5B0001D21C4F8481395E7514800220023214645
:10E5C00026468464C463C0E910230246D56C02F178
:10E5D0004C035DB398684D1E9E64A842C2E9236651
:10E5E000DE630DD04D1CA84210D113F8481C002941
:10E5F0003FF409AF1A6401461A4643F8083CE5E7C0
:10E6000000293FF400AF53F80C2C014600293FF4D9
:10E61000FAAE81427FF4F7AE106CC56B0135C5636D
:10E62000186493641A46D1E7012469E7344A022644
:10E63000294613E0D36B16635B01C2E9041120D0B5
:10E6400003F6FF7300EB133318465363C31A90634A
:10E6500052F84C7F461C1D440134C7B11379701E1B
:10E66000002BE7D1136916637BB103F6FF7300EB50
:10E6700013335769536337B107F6FF7700EB173051
:10E68000E4E73346E0E73046E0E73346F1E7DFF81A
:10E6900080E00138CEF82443820F1B4C8300CEF873
:10E6A00018533F25CEF8FC424024CEF81403CEF890
:10E6B00008433E24CEE9C045D0B140F2FF141B19F7
:10E6C00042F100025B0A43EAC25303F140020C49E3
:10E6D0001344CEF80C2303EBC000CEF810334202F3
:10E6E000CEF8F802C30DCEE9C711CEE9BC238AE605
:10E6F0000123EAE7000001204403012080510100CA
:10E70000383201200068214C780F06086C0F06088B
:10E7100090190120704700BF2DE9F047002BDDF86C
:10E7200020A0884607460CBF4FF020094FF0300963
:10E730005646002A144616F8011B23DD11B3334652
:10E7400001E0002C05DD13F8012B2546013C002AD1
:10E75000F7D1023D3CB149463846C047013DFAD2A7
:10E760009AF8001059B13846C047334616F8011BD5
:10E770000029F8D1A4EB0A041819BDE8F087204657
:10E78000BDE8F087002C04F1FF35E4DC002400290B
:10E79000E9D1F4E703685A1C02601970704700BFA2
:10E7A00010B56FF000440246044404E0B3EB0E00E1
:10E7B00015D1A24214D012F8013BA3F1410019284F
:10E7C00011F8010BA0F1410C98BF203300F1200E8D
:10E7D000BCF1190FEAD91B1A04D10028E9D110BDE8
:10E7E000002010BD184610BD0378202B03D110F86F
:10E7F000013F202BFBD0092BF9D02D2B63D02B2BE5
:10E80000B7EE000A08BF01300278A2F13003D9B296
:10E81000092961D8F2EE046ADFED4D7A07EE103A6D
:10E8200010F8012FB8EEC77AA2F13003D9B2A7EEE3
:10E83000A67A0929F0EE477AF0D92E2A50D003782B
:10E8400003F0DF03452B3BD110B442782D2A73D05F
:10E850002B2A62D0A2F130030130092B63D80024A7
:10E86000002303EB830302EB430310F8012FA2F113
:10E870003001303B0929F4D9B3F59A7F1A46B7EE37
:10E88000007A28BF4FF49A72072B09D91346DFED9F
:10E89000316A083B27EE267A072BFAD802F00702E6
:10E8A0002AB1F2EE046A013A27EE267AFBD1002C57
:10E8B0003BD0C7EE877A5DF8044B20EE270A7047FD
:10E8C00020EE270A704742780130BFEE000AA2F11D
:10E8D0003003D9B209299DD92E2ADFED1D7AAED198
:10E8E00043780130A3F13002D1B20929A8D8B2EEA1
:10E8F000047AF0EE475A06EE902A10F8013FB8EE7F
:10E90000E66AA3F13002D1B2C6EE076A092927EE02
:10E91000257A77EEA67AEED992E782780230A2F1D4
:10E920003003092B9BD9B7EE007A67EE877A5DF842
:10E93000044B20EE270A704782780230A2F13003A0
:10E94000092B01D801248BE7B7EE007AB1E700BFAD
:10E950000000000020BCBE4CF0B5067906F0E003D4
:10E96000402B03D145794FF0FF3406E0602B4FF088
:10E970000105F8D1447905FA04F40023012006F0DA
:10E980000706AB4200D1F0BD052E0FD8DFE806F038
:10E990000308101D242448B1C85CD75C78400FE000
:10E9A00020B1C856D756C71B784278410133E8E7F3
:10E9B0000028FBD031F8130032F81370784080B291
:10E9C00020420CBF01200020F0E70028EED031F9F2
:10E9D000130032F91370E6E70028E7D051F823005E
:10E9E00052F82370DAE7037903F01803102B1DD0D7
:10E9F00003D833B9B0F80B007047182BFAD00020B9
:10EA00007047114BB0F80B0093F90030591C0BD133
:10EA10000E4B1B7803EB430203EB820303EBC303B0
:10EA200000EB430080B27047DBB2F3E7064BB0F86F
:10EA30000B0093F901305A1C04D1044B5B7800EBB6
:10EA40004310EFE7DBB2FAE778030120CC50012056
:10EA5000032870B518D80D4BC943C60003EBC0009E
:10EA600001F00101057D427D81EA0504A2420BD03F
:10EA700002693AB14D1B10689288694269410901E7
:10EA80008A40826133445C7570BD00BFCC50012068
:10EA9000F0B1A0F1800380F0800009281AD8092B7A
:10EAA00018D8DFE803F0190507090B0D0F1711132C
:10EAB0000A4870470A4870470A4870470A48704732
:10EAC0000A4870470A4870470A4870470A48704722
:10EAD0000A4870470A4870470A487047C5A30608A5
:10EAE0002C820608368206083CA406083D820608E9
:10EAF00043820608498206085582060824820608D1
:10EB00002EA306085F820608B5EEC00ADFED357A4F
:10EB10000023F1EE10FA30B5C8BF30EE270A87B0F7
:10EB2000D8BF30EE670ADFED307A054603A90293BD
:10EB300020EE270ACDE90033FDEEC07A17EE904AA9
:10EB400084EAE470A0EBE47041F036FC002C03A8EA
:10EB5000B4BF2D2320238DF8003047F0FBFF0128A0
:10EB60002AD0022834D003281ED003A9684649F0D1
:10EB700045FD684647F0EEFF044669462846033CDB
:10EB8000E4B2224649F03CFC002328462B5547F0CE
:10EB9000E1FF2E22431C0DEB04012A54E81849F032
:10EBA000B3FD284607B030BD302303A968468DF871
:10EBB000013049F023FDDCE743F23002302303A9A2
:10EBC0006846ADF801208DF8033049F017FDD0E715
:10EBD00043F2300303A96846ADF8013049F00EFD59
:10EBE000C7E700BF6F12033A00007A440AF0E6BF9D
:10EBF00038B5054658B14C1E14F8011F284619B9FE
:10EC0000BDE838400AF0EEBF0AF0D8FFF4E738BD9F
:10EC100070B50546B0F809003CF088F8064B04468C
:10EC2000284693F83060FFF7DEFE16B1E36818441B
:10EC300070BDA368FBE700BFCC50012038B5054686
:10EC40000C46FFF7E5FF2A7902F0070302F0E00225
:10EC5000602A29D1052B0CD8DFE803F0030B0F0B3A
:10EC60001B1B6A79012393400278DBB214B1134372
:10EC7000037038BD22EA0303FAE76A79012393405F
:10EC800002889BB214B113430380F2E722EA030324
:10EC9000FAE76B7901229A40036814B113430360C9
:10ECA000E7E723EA0203FAE7052BE2D8DFE803F0FF
:10ECB0000303050507070470DBE70480D9E7046058
:10ECC000D7E708B5202149F0A8FC034618461BB138
:10ECD00002780133202AF9D008BD08B5CB0701D44A
:10ECE000FDF790F808BD2DE9F3410023124D0446CD
:10ECF00000EB8106114F05F8313FB44203D11048B3
:10ED000002B0BDE8F081394628464FF0000849F0CE
:10ED100075FC2146684649F0F7FC2021684649F019
:10ED20007CFC28B969462846043449F067FCE4E7CE
:10ED300080F80080F1E700BFCC500120E6A3060870
:10ED4000FD50012010B58C18A14215D001F1FF3EF5
:10ED5000013C41F2210C1EF8012F082380EA022019
:10ED600002B24000002A8CEA420180B2B8BF88B2E9
:10ED7000013BF5D17445EED110BDF8B5164D6B7859
:10ED8000BE2B26D1AC1C154F022229464FF6FF7030
:10ED9000FFF7D8FF22884AB1A618BE4219D2052A29
:10EDA00017D921463446FFF7CDFFF3E7214602226B
:10EDB000FFF7C8FF0222A1180634FFF7C3FF084B74
:10EDC000641BA3F8524041F60F53C31A58425841EE
:10EDD000F8BD0020FCE700BF0040000800800008EC
:10EDE000CC5001200823484041B240000029C0B265
:10EDF000B8BF5040013BF7D1704700BF30B5056840
:10EE000004468D4218D901F1FF3E681E00231EF80A
:10EE100001CF082183EA0C034FFA83FC5B00BCF1AD
:10EE2000000FDBB2B8BF53400139F5D17045EED1C8
:10EE30006A1C22602B7030BD00236A1C22602B707C
:10EE400030BD00BF9FED067AF7EE007A60EE870ACC
:10EE500060EE800A30EEA70A80EE800A704700BF9D
:10EE6000DB0FC940DFED2D0A08B548F031FDDFEDBD
:10EE70002C7AB4EEE70AF1EE10FA28DDDFED276A0E
:10EE80009FED287AF0EE407A30EE660AF4EEC77A0B
:10EE9000F1EE10FAF6DCDFED247AB4EEE70AF1EEDB
:10EEA00010FA2FDDDFED1E7A37EEC00A20EE007A71
:10EEB0009FED1E6ADFED1E6ADFED1E7AE7EE066A41
:10EEC00020EE076AE6EE877AA6EE270A08BDDFED98
:10EED0001A7AB4EEE70AF1EE10FADCD5DFED0F6A2C
:10EEE0009FED167AF0EE407A30EE260AF4EEC77AFD
:10EEF000F1EE10FAF6D4DFED0C7AB4EEE70AF1EE9B
:10EF000010FACFDCDFED0E7AB4EEE70AF1EE10FA7C
:10EF1000CCD5DFED097A37EEC00AC7E7DB0FC94071
:10EF2000DB0F4940E4CB1641DB0FC93F92E741B903
:10EF30009730083C15A82ABEDB0F49C0E4CB16C1A8
:10EF4000DB0FC9BF10B5B7EE001A0022DFED050ACE
:10EF5000044649F0DDFD0023A36163612362E361A0
:10EF600010BD00BFF304353FB0EEC07AF0EEE06AAA
:10EF7000F0EE407AC6FE875AF5EE405AF1EE10FAEE
:10EF80003BD086FEC75A85EE256A9FED1D2A9FED70
:10EF90001D3A9FED1D4ADFED1D4ADFED1D2AF7EEFC
:10EFA000005ADFED1C3A9FED1C5AA6EE423AE6EEFF
:10EFB000223AA6EE034AE6EE235AE6EE044AA6EE0D
:10EFC000245A85EE250AF4EEC76AF1EE10FA03D54D
:10EFD0009FED127A37EE400AF5EEC00AF1EE10FA14
:10EFE00003D59FED0F7A37EE400AF5EEC07AF1EEC9
:10EFF00010FA48BFB1EE400A70479FED070AE2E7FA
:10F0000039094E3DE3B59E3E88FA163E45FE7F3FE8
:10F0100099FB243F69A2163EA7DFA834DB0FC93F46
:10F02000DB0F49402DE9F04F1646884689B016F8A7
:10F03000011B002900F04382144607469B46002529
:10F0400009E0013534463846C047264616F8011B0C
:10F05000002900F090802529F3D16178302900F053
:10F060008E8002340023A1F1300C5FFA8CF2092A61
:10F070004FF0000260D96C2900F085807829E4D82F
:10F08000572940F2E880A1F158002028DDD801A6D8
:10F0900056F820F073F200084BF000084BF000081F
:10F0A0004BF000084BF000084BF000084BF0000854
:10F0B0004BF000084BF000084BF000084BF0000844
:10F0C0002DF2000827F300084BF000084BF0000871
:10F0D0004BF000084BF000084BF000084BF0000824
:10F0E0004BF000084BF000084BF000084FF200080E
:10F0F0004BF000084BF000084BF000084BF0000804
:10F100003BF200084BF0000887F300084BF00008C2
:10F110004BF0000873F20008BEF1050F18D9B9F1E1
:10F12000050FA8D80A2E17D102EB820214F8011B92
:10F1300006EB4202A1F1300C5FFA8CF0A1F1610EF6
:10F14000A1F14109A1F137060928E5D86646EBE7A8
:10F15000A1F157060A2EE7D0572994D825297FF424
:10F1600074AF2646252138460135C04716F8011BE5
:10F1700000297FF470AF284609B0BDE8F08FA17870
:10F18000012303346FE714F801CBBCF1780F3FF68D
:10F190005CAFBCF1570F64D9ACF1580120293FF6A0
:10F1A00054AF01A050F821F0D5F200084BF0000850
:10F1B0004BF000084BF000084BF000084BF0000843
:10F1C0004BF000084BF000084BF000084BF0000833
:10F1D0004BF000082DF2000837F400084BF000084F
:10F1E0004BF000084BF000084BF000084BF0000813
:10F1F0004BF000084BF000084BF000084BF0000803
:10F200004FF200084BF000084BF000084BF00008EC
:10F210004BF000083BF200084BF00008DDF300085B
:10F220004BF000084BF00008D5F200085BF8041B17
:10F2300038460135C9B2C04707E75BF8040B002325
:10F24000414600903846FFF767FA0544FDE65BF853
:10F25000043B1D60F9E6002980D1284609B0BDE8CD
:10F26000F08FBCF1000F86D0BCF1250F3FF479AFD1
:10F27000EBE65BF804EB0120BEF10F0F40F22181B9
:10F280000001BEFBF0F60F2EFAD8002800F01D8119
:10F290000DF1140AD14601E0BEFBF0F6092E4FF045
:10F2A000300C05DD58290CBF4FF0370C4FF0570CD0
:10F2B000B44400FB16EE000909F801CBECD10021A3
:10F2C00089F8001041463846CDF800A0FFF724FA2F
:10F2D0000544BAE65BF8049B0121B9F10F0F40F237
:10F2E000F2800901B9FBF1F00F28FAD8002900F0EB
:10F2F000E2800DF1140AD64601E0B9FBF1F00928CD
:10F300004FF0300604DDBCF1580F0CBF37265726EE
:10F31000064401FB109909090EF8016BEDD100219B
:10F320008EF80010CEE75BF8046B002EC0F2BA80B6
:10F330000DF1140AD646092EB4464FF0010108DD3E
:10F3400001EB81014900B6FBF1F00928F8D800294A
:10F35000E5D0DFF880910393A9FB0163BCFBF1F0DA
:10F360000A284FEAD30301FB10CCB4BF302657263E
:10F370000929194606440EF8016BEDD8039B0021BC
:10F380008EF800109EE75BF8040B0121092809D9CB
:10F3900001EB81014900B0FBF1F6092EF8D80029F4
:10F3A00000F089800DF1140ADFF828910393D64606
:10F3B000A9FB01C3B0FBF1F60A2E4FEAD30301FB10
:10F3C0001600B4BF4FF0300C4FF0570C0929194606
:10F3D000B4440EF801CBEBD8039BD0E75BF8040BE9
:10F3E0000121092808D901EB81014900B0FBF1F6A0
:10F3F000092EF8D800295ED00DF1140ADFF8D49058
:10F400000394D646A9FB01C4B0FBF1F60A2E4FEADD
:10F41000D40401FB1600B4BF4FF0300C4FF0570C72
:10F4200009292146B4440EF801CBEBD8039C0021F6
:10F430008EF8001046E75BF8040B002829DB0DF17D
:10F44000140AD64609284FF0010109D901EB8101C0
:10F450004900B0FBF1F6092EF8D800293FF45FAF60
:10F46000DFF870900394A9FB01C4B0FBF1F60A2EFB
:10F470004FEAD40401FB1600B4BF4FF0300C4FF03C
:10F48000570C09292146B4440EF801CBEBD8039C54
:10F49000CDE72D2140420DF1150E0DF1140A8DF826
:10F4A0001410CFE72D2176420DF1150E0DF1140A3F
:10F4B0008DF814103FE70DF1140AD6462FE70D46DC
:10F4C00059E67646E4E6484613E70DF1140AD146BC
:10F4D000F5E600BFCDCCCCCCF8B5114C07460D46B7
:10F4E0001646606DA0B10F49FFF782FB3946606D8B
:10F4F000FFF77EFB0C49606DFFF77AFB0B49334643
:10F500002A46606DFFF78EFD0949606DFFF770FBBD
:10F5100094F8583013B1012384F85930F8BD00BF76
:10F52000CC500120658206083B9C0608EDEB0008E4
:10F53000728206080EB400B584B0084905AB01908C
:10F5400001A853F8042B0393FFF76CFD0022019BE5
:10F550001A7004B05DF804EB03B0704795E700083B
:10F56000F7B5114E074600230C46304615460F49A5
:10F570005A3600F85A3F04EB45050D4B002F18BFD3
:10F5800019460C4F49F03AF8AC4202D10A4803B090
:10F59000F0BD394634F8022B6846FFF7CBFF6946C9
:10F5A000304649F02BF8EFE7CC5001207F82060867
:10F5B000768206088882060826510120F7B50023C6
:10F5C0000B4E044600EB41050A4F06F88B3FAC4258
:10F5D00002D1094803B0F0BD394634F8022B684621
:10F5E000FFF7A8FF6946304649F008F8EFE700BF8B
:10F5F000CC5001202C83060857510120F8B54E1E2F
:10F60000054601F11F04054F16F8012F284639461B
:10F610000235FFF78FFFA642F6D1F8BD8D820608AE
:10F6200003685A1C02601970090A03685A1C0260B8
:10F630001970704702681346511C016013F802CB21
:10F640000360D31C5178036093781B0443EA0123C1
:10F65000111D43EA0C030160D07843EA0060704753
:10F66000A0F13003092B07D920F0200041381928D8
:10F670008CBF0020012070470120704730380928D6
:10F680008CBF002001207047413819288CBF002012
:10F6900001207047613819288CBF00200120704775
:10F6A00020280BD0092809D00A2807D00D2805D01A
:10F6B0000B3801288CBF00200120704701207047C3
:10F6C000A0F14103192B98BF20307047A0F16103CE
:10F6D000192B98BF2038704702B3844610B58418A0
:10F6E00003E0981A15D1A44514D01CF8013BA3F1EE
:10F6F0004100192811F8010BA0F1410E98BF2033E9
:10F7000000F12002BEF1190FEBD91B1A04D1002819
:10F71000E9D110BD002010BD184610BD104670473D
:10F7200070B5044608460D4647F014FA064602E056
:10F7300014F8013F43B1324629462046FFF7CCFF7B
:10F740000028F5D1204670BD1C46204670BD00BF84
:10F750002DE9F043064686469EF800C074460EF139
:10F76000010EBCF1200FF7D0BCF1090FF4D0BCF1B1
:10F770000A0FACF10B00EFD0ACF10D05B5FA85F531
:10F780006D09002DE8D10128E6D9BCF12B0F3DD041
:10F79000BCF12D0F39D0102A3ED04FF0FF3E9046DD
:10F7A000BEFBF2FE02FB0EF7FF43FFB2002014F88F
:10F7B00001CBBCF1390F4CF02009ACF1300C0DD865
:10F7C0005FFA8CFC944510DA7045264602D819D1B0
:10F7D000674517D21D404FF0FF30E8E7A9F1570CFD
:10F7E000B9F1600F5FFA8CFCECD801B10E6003F048
:10F7F0000103D5B9002803DA002B18BF6FF00040D1
:10F80000BDE8F08300FB08C0D1E70125102A94F879
:10F8100001C004F10104C0D1BCF1300F10D06FF071
:10F82000704E0F274FF01008C0E7B0F1004F04D919
:10F830001BB14FF00040BDE8F0834042BDE8F083CB
:10F8400060786FF0704E0F274FF01008A0F141065E
:10F85000192E04F1010698BF203078280CBF02341D
:10F860003446A3E701230A22002171E770B50D4653
:10F870001446FFF726FA0646A0B1FFF7F3FF40F65D
:10F88000340319229842A8BF1846B0F5617FB8BF6B
:10F890004FF46170A0F56173B3FBF2F32B70237822
:10F8A000013323703046FFF70CFA0646A0B1FFF78C
:10F8B000D9FF40F6340319229842A8BF1846B0F584
:10F8C000617FB8BF4FF46170A0F56173B3FBF2F3D1
:10F8D0006B70237801332370304670BD2DE9F04101
:10F8E00016461F46404D0446394630464FF47A725C
:10F8F000002347F037F93D4B05443D4F3D4E83FB18
:10F900000510E9172844C1EB601183FB0103C817F8
:10F910000B44C0EB631087FB003CC317C3EBAC0385
:10F9200086FB03764FEAE37ECEEBE61EC1EB0116C3
:10F93000A5EB860CC0EB00154FEA8E0684F806C0D6
:10F94000A1EB8501617103EB4301A0EBC10040F223
:10F95000B55101FB1E332071B3F5896F33DA40F2E4
:10F96000DA218B4237DCB3F5B77F234FB4BF4FF0BA
:10F97000000E4FF0010E0EEB4E0175464FEA4E0899
:10F9800007EBC101C88A08EB0E0C0B2107EBCC0C6E
:10F990000CF1160C01E03CF8020D984210DD013923
:10F9A000F9D1F044012137F8380006F5FA6E013339
:10F9B000A17075441B1A22812580E370BDE8F08197
:10F9C0000131C9B2F1E7032540F296500A4F4FF0DA
:10F9D0000608AE46D7E7022540F22940064F4FF011
:10F9E0000408AE46CFE700BF80BC92C789888888EC
:10F9F000ABAAAA2A73B06D16849E05080D4B10B5EC
:10FA0000D3E9004354EA03020AD10146002340F23D
:10FA1000011218460B80C1F802208B710B8110BDBA
:10FA2000054A1268121943F10003FFF757FF01203E
:10FA300010BD00BFE8290120641C01202DE9F04120
:10FA40000446154608469442B4FBF2F607D205FB7D
:10FA50001644134B1B5D00F8013BBDE8F081964254
:10FA6000B6FBF2F70CD20E4B05FB176705FB1644ED
:10FA7000DA5D1B5D00F8012B00F8013BBDE8F08169
:10FA8000BA42B7FBF2F807D905FB1878044B13F814
:10FA9000082000F8012BE7E74046FFF7CFFFF3E728
:10FAA0009C0F060830B56D4C83B0B4F8E034B3F564
:10FAB0007A7F03D94FF47A73A4F8E034B4F8E234CF
:10FAC000B3F57A7F03D94FF47A73A4F8E234B4F82B
:10FAD000E414B1F57A7F04D94FF47A731946A4F887
:10FAE000E434B4F8E604B0F57A7F03D9002318466D
:10FAF000A4F8E634B4F8E834B3F57A7F4AD94FF481
:10FB00007A73B4F8EA249A42A4F8E83447D9002377
:10FB10008842A4F8EA3480F08B80B4F8F624B4F874
:10FB2000F8349A4202D90023A4F8F6344C4B1B88CF
:10FB3000EBB14C4DAA78062A4ED9297900297AD101
:10FB40009FED497A94F8002507EE903AAB7906EEDE
:10FB5000902AF8EEE77AB8EEE66AC6EE276A0BB1AD
:10FB600037EE077AB4EEE67AF1EE10FA42DC62780C
:10FB7000032A23D83D4B03EB42132278C4F80835FF
:10FB8000032A14D8EA213A4B02FB0133C4F80C359E
:10FB900003B030BDB4F8EA24B2F57A7F16D88842B3
:10FBA00010D29A42B9D30023A4F8E834B5E7002272
:10FBB0002F4B2270C4F80C3503B030BD00222B4B04
:10FBC0006270DAE70021A4F8E414EAE70022884230
:10FBD000A4F8EA24E5D3F5E7264901EB820191ED8B
:10FBE000187A29790029ADD0531F032BBFD9002AD9
:10FBF000BDD025E067EE877ABCEEE77A8DED017A1D
:10FC00009DF8043007EE103AB8EEC77AF4EEC77AE2
:10FC1000F1EE10FA01DD0133DBB2EBB1102BA8BF1E
:10FC20001023DBB2934238BF134684F800359EE7B9
:10FC3000A4F8E43471E7053A032A98D99FED0A7ACB
:10FC4000B7EE000A80EE070A47F072FF2B88834266
:10FC500028BF03462B808AE70123E2E7CC5001202E
:10FC60009C1E00201C2801206F12033880510120A7
:10FC700000520120849E05082DE9F04FA84E83B064
:10FC800096F8103500AFA3F11702022A00F2A38202
:10FC9000A44B7B6096F820350024DFF8A0A23B60DF
:10FCA000A14B03F1540998461FE098F90420142A47
:10FCB00000F02283584648F079FD1BF4003F21D024
:10FCC000012800F01983082800F3168315B11BEAF8
:10FCD0000A0F06D13968584645F0B0FF002800F0F9
:10FCE0000B8308F10C08C14512D0D8F800B01BF006
:10FCF0000105DAD05846013448F058FD1BF4003FA6
:10FD0000E4B2DDD10128DEDC08F10C08C145ECD1FC
:10FD1000013C022C00F2F0820023022086F8A43578
:10FD20000DF064FC96F8AC35D6F8A895022B00F0DF
:10FD3000EE82002800F051837C4B4FF47A7C96F8D9
:10FD400009A6002503F56A7E4FF0640B33F8082CF2
:10FD5000B2F57A7FB3F8462088BF23F808CCB2F515
:10FD60007A7F33F8062C88BFA3F846C0B2F57A7FB5
:10FD700033F8042C88BF23F806CCB2F57A7F02D979
:10FD8000002223F8045C33F8061C9142B3F85A10A1
:10FD9000B3F85C2098BF23F8065C914293F86B207F
:10FDA00003F1650102F1FF3288BFA3F85A50632ABC
:10FDB00093F86C2002F1010288BF83F86BB0D2B2D5
:10FDC000092A4FF0000288BF83F86C5013F8320004
:10FDD000013211F8014F844238BF0D70032AF5D16A
:10FDE000BAF1010F03F1EA0318BF03F8645C9E4502
:10FDF000ACD1DFF84CA19AF80230042B00F0C0829D
:10FE00002BB9BAF80030B3F5F07F00F20282FFF7A9
:10FE100049FE96F82336092B1AD0B3FA83F2520919
:10FE2000B3B1013BA6F824265A0003F00303C3EB49
:10FE3000031302F00802C3EB03139B00A6F8283655
:10FE40009300A3EB9203C3EB03139B00A6F82636A3
:10FE5000B6F83226B6F830361343B6F834261343D4
:10FE60001BB213B10123A6F83636314B09EA03035E
:10FE7000002B00F0BF8219F0010F40F07C8219F4D2
:10FE8000804F40F0CB8119F0080F00F03A82294AE8
:10FE9000D6F8FC3509EA02091340C6F8A895C6F859
:10FEA000FC3519F4004F00F0CE81002386F8273589
:10FEB00086F8373519F4805F00F0D18196F8433623
:10FEC000012B02D9012386F84336DFF86C904B46AC
:10FED00009F1780402E006339C420CD01A780A2A11
:10FEE000F9D19978DA78914202D35A79002AF2D07E
:10FEF0000A201CF0DDFB00234FF4806086F8A43557
:10FF00000DF074FB002800F054820B4DAB469BF8BB
:10FF1000051011B39BF80000E8B14B4615E000BF97
:10FF2000CC500120849E0508185601200A52012059
:10FF300009600002FE9FFFFD14570120BC02020071
:10FF40001C28012006339C4207D01A788A42F9D136
:10FF50005A79002AF6D01CF0ABFB0BF1060B5C457E
:10FF6000D5D19AF80290B9F1080F00F0DE8196F829
:10FF70000936D6F8FC25A3F10103C2F3C031B3FA68
:10FF800083F386F8C3165B0986F8C03696F80A36FE
:10FF9000A3F10103B3FA83F35B0986F8C63696F83A
:10FFA000DD34032B02D9002386F8DD34BE49D6F8B0
:10FFB000A8350A400B40B17BC6F8FC25C6F8A83529
:10FFC000002900F0CA81B6F8DC36002B40F0BB8176
:10FFD000D6F8E036B3F5000F02D30023C6F8E036BA
:10FFE000D6F8E836B14A1A401AB140F20223C6F8F0
:10FFF000E83696F8E436013B042B02D9012386F853
:020000040801F1
:10000000E436A9F10509AA4BB9F1030F93F8FC8373
:1000100040F23781B8F1000F1CD000233B60DFF8BD
:10002000B49206E0ABF1060BABEB0A0BD84540F2FD
:10003000F780CB4619F8010F0028F3D00AF0F6F844
:100040000028EFD081798B07ECD53B680122002B8B
:1000500040F0EB809AF8063013B100238AF806309E
:10006000B6F8F23603F00F02042A03D8C3F30313E1
:10007000022B03D94FF42063A6F8F236B6F8F43613
:1000800003F00F02042A03D8C3F30313022B03D98E
:1000900040F60123A6F8F43696F8611796F86D2716
:1000A00096F86037914205D9002286F8612753B14E
:1000B000A6F8642796F86C279A4204D2002386F8A3
:1000C0006037A6F8643796F8622796F856389A4251
:1000D00002D9002386F86237DFF8FCC10CF1800BEF
:1000E0006346796813F8032D02EB42020A4492F842
:1000F00034A292F8359292F836E213F8010F99790A
:100100005045DA78A8BF50464945A8BF49467245D0
:100110001870A8BF724663459971DA70EDD103F18A
:10012000200CDC45DCD1D6F84425002A00F01D81E6
:100130000020012102E00635AC420ED02B782B2B9B
:10014000F9D16B78043301FA03F31342F3D0063587
:1001500022EA03020120AC42F0D108B1C6F84425DE
:10016000544C6D4604F10808234602E0434500F074
:10017000928013F8012F072AF8D9002304F8013FD1
:100180000133082BFAD1B6F80226AD46B6F8003690
:100190009A4202D3484BC6F80036484BFF22484CDF
:1001A00003F1540086F8882813F9082C142A05D086
:1001B00053F80C1C34EA010100F0DF800C33984244
:1001C000F2D1404B5A79022A01D100225A710C37E0
:1001D000BD46BDE8F08F3C4A11467A60DA0001EB7B
:1001E000C30393F87C1021B1D3F88030002B00F0CA
:1001F000DC807B68134493F87D20002A3FF44AADED
:1002000093F85C31002B7FF445AD182386F8103548
:1002100040E54FF4F073AAF80030F8E52B4A37E6D2
:100220003B680022002B3FF415AF9AF81130002BE9
:100230007FF416AF9AF80530012B3FF40BAF002A7C
:100240007FF408AF0CE796F82735002B00F0BE804E
:10025000002319F4805F86F837357FF42FAE19F04C
:10026000800F3FF42BAE96F81025182A04D8184BAF
:10027000D340DA073FF522AEDFF8609009F1780449
:1002800039E600238AF80430B8F1000F00F0B0809E
:1002900001233B60C3E688B02022FF21E94648469F
:1002A00048F0A4F9034A20E0BDD45518FDFDFFFF36
:1002B0009C1E00202E280120AE014A012456012058
:1002C00001000200A42C0120849E0508F6DFFFFD3A
:1002D00000410001232801208551012014570120ED
:1002E000424549F823303FF44EAF12F8013F59F828
:1002F00023100131F4D040E7434944483AF02CFD43
:100300000AE519F4005F3FF4CCAD414AC0E500288E
:100310003FF412AD90F90440FF2500E0057220463D
:100320000DF054F90028F9D106E59AF80630002BB3
:100330003FF41DAE9AF81130012B7FF418AE022362
:100340008AF8113013E696F8D80609F06FFF0028F6
:100350007FF43EAEA6F8DC063AE62E490B430A438C
:10036000C6F8A835C6F8FC252DE62B201CF0A0F910
:10037000D6F84425DCE6284A8AE586F8882820E76E
:10038000D6F8FC3529F4805923F48053C6F8A89593
:10039000C6F8FC35BAF82030B3F57A7FBFF437AD34
:1003A0004FF47A73AAF8203031E5172386F8103518
:1003B0001FE7D6F8A83523F00063C6F8A835D6F8AD
:1003C000FC3523F00063C6F8FC359EE542F20103DC
:1003D00019EA030F7FF43CAF6CE5D6F8FC3529F041
:1003E000800923F08003C6F8A895C6F8FC35A3E47D
:1003F00042461AE7D6F8FC3549F0080943F00803ED
:10040000C6F8FC3543E500BF1856012048E606084B
:10041000F6BFFFFD00040500F79FFFFD2DE9F04F3B
:10042000A64E2DED028B96F88C3883B0013B012B44
:1004300040F22E81D6F8BC28A14BDFF8B88202F238
:10044000DC524345C6F8BC2880F03481DFF8A8921E
:1004500001229B469B4D09F102070192B9F8021057
:10046000002900F000817A18AA4280F0FC8005295A
:1004700040F2F980BBF800003C46C0F30B000BE0F3
:10048000118814460A44002900F0ED80AA4280F049
:10049000EA80052940F2E78061888142F0D16179E4
:1004A0008B07EDD123885846DBF8081094F804A098
:1004B00000933AF051FCBBF80010BAEB113F00F08A
:1004C000D88000230193BBF804100BF11C0B5BF8E0
:1004D000140CC1F30B015BF8044C40F03BFDC34529
:1004E0002060BBD3D6F8A835774CC6F8FC35FFF7AB
:1004F000C3FB3378EA22754D03FB0242A4F180036B
:10050000C6F80C25727803EB4213C6F8083519F0CB
:1005100091FB4FF0FF33D6F80C056B6022F0DEFF45
:100520001CF00CF904F2145304F28C5103E006336E
:10053000994200F0A8801A78002AF8D19C78D878DF
:10054000844202D358790028F1D096F840362A72B6
:100550006422B6F8441603EB83035D4C02FB01F101
:1005600003EB83030022DFED5B8A9B006429C6F85E
:10057000BC28B8BF6421642BC6F8C028B8BF642368
:10058000C6F8B818C6F8D0185349C6F8C428C6F833
:10059000C828C6F8CC28A6F8D42886F8D628C1F8EA
:1005A0007C45C6F8B43824F077FDB6F9EA389FEDFB
:1005B0004B7A08EE103AB6F8E638DFED496A07EEF6
:1005C000903AB6F8E438B8EEC88AB6F8D858F8EEDB
:1005D000E77A96F8DA7828EE268A67EE877A38EE98
:1005E000280AC4EDAB7A07EE903AF8EEE77A67EEA8
:1005F000877AC4EDAC7AFEF735FCB0EE480AFEF718
:1006000031FC96F8E838B0EE680A9FED367A07EECE
:10061000903AF8EEE77AA7EE870AFEF723FC07EE9A
:10062000905ADFED316AF8EEE77A84EDAF0AC6F84A
:10063000F47886EEA77A84EDB07A32F0D7F911F02B
:1006400083FC96F88C38013B012B2BD9274B0122D8
:1006500001981B6886F8D528C6F8BC3803B0BDECF5
:10066000028BBDE8F08FDBF8081058463AF074FBB7
:1006700027E7009BA11D58469A1F3AF0A3FB0028CC
:100680007FF421AF1DE7F27B003A18BF01225CE73F
:10069000FCF7C0FA164B0222034486F8AC28C6F8D1
:1006A000A838C7E6FCF7B6FA0223C6F8A80886F809
:1006B000AC38CBE70123019314E700BFCC500120F5
:1006C000A0E5060800800008005201207803012000
:1006D000FC560120DB0FC93F9C1E002017B7D13804
:1006E00088C3E43A35FA8E3CC0C9FB48641C01203B
:1006F00060E31600D0EE060800400008114B01220E
:10070000032810B5044683F8842505D9601CBDE88C
:100710001040C0B20DF020BB0B4BEA2203F59A70DB
:100720001C7004FB0200C3F80C0522F0D7FE21F078
:1007300011FA21F0F3FA601CBDE81040C0B20DF0D0
:100740000BBB00BF9C1E0020CC500120054B01219B
:10075000D3F8FC2883F8F81842F40012C3F8FC28F8
:10076000704700BFCC5001202DE9F043D0F8008045
:1007700087B005460C46C8F30D03002B3FD1394A1C
:100780000120394E0221B242CDE90233CDE9040104
:100790001ED3364B9A421AD303F580439A4222D392
:1007A000334B9A4221D903F580339A421FD903F57E
:1007B00000339A421DD903F500339A421BD903F541
:1007C00000339A4219D90520FCF7FAFEFBE70346ED
:1007D00001A902A8039341F075FD80B14FF0FF30ED
:1007E00007B0BDE8F0830B46F2E70323F0E70423EC
:1007F000EEE70523ECE70623EAE70723E8E71D4ECB
:10080000D4F8009096F81439012B09D0012386F80A
:10081000143941F0F9FC074628B1002386F8143951
:100820006FF00100DCE7144C236923F4407323616B
:10083000236943F400732361236943F001032361B7
:10084000C8F80090BFF34F8F41F0DEFC236923F01E
:100850000103236186F814790028E1D12B68043361
:100860002B60BDE700400008004000080080000841
:10087000FFFF0008CC500120003C02402DE9F04170
:100880005A4E8AB03378B12B71D1FEF776FA80F0E8
:100890000104E4B2564B04F00104564DB3F8433260
:1008A000554FADF80430BD4263D3002C00F09C805E
:1008B00000230596CDE907330993504B9B1B069304
:1008C0004F4B1A69002A05DA4E4A5A6002F1883203
:1008D0005A601B694FF48073022201A905A8ADF884
:1008E000243045F065FE022201A94FF6FF70414D0C
:1008F000FEF728FA4FF000080446BD4249D3002510
:10090000022202A905A8ADF8085045F051FE0222C6
:1009100002A92046FEF716FA40BA022203A9C043F4
:10092000ADF80C0005A845F043FE089878B107AB78
:10093000C0F104022946184447F058FE9DF92400EE
:1009400018B907A905A8FFF70FFF8DF824009DF837
:10095000253023B12A4A136943F0004313619DF9FE
:100960002400B0FA80F040090AB0BDE8F08101240B
:1009700090E7AB691C3535F8181CD3F8008055F8A2
:10098000140CC1F30B0140F0E5FA804518BF0124B7
:1009900089E7AE8803A905A88DF81180C6F30B0678
:1009A0001C35B31DADF80C3035F81C3CC3F30B02FD
:1009B0001B0BADF80E2006228DF8103045F0F8FD27
:1009C000062203A92046FEF7BDF9044655F8141C7B
:1009D000324605A845F0ECFD204655F8141C324679
:1009E000FEF7B0F9044688E70120BDE700400008A3
:1009F000849E0508A0E50608D0EE060800800008E1
:100A0000003C02402301674570B5264CFFF734F9DE
:100A100094F88C38013B012B31D9D4F8BC3803252C
:100A2000214E03F2DC53C4F8BC38FFF727FF58B15E
:100A30003378B12B08D1FEF7A0F9013D1CD040B9A5
:100A4000FFF71CFF0028F3D1013DEED10520FCF794
:100A5000B7FD94F88C380022013B84F81C29012B47
:100A600017D9124B012100221B6884F8D51884F88D
:100A70001D29C4F8BC3870BD0028EAD1E6E7FCF7B0
:100A8000C9F80B4B0222034484F8AC28C4F8A838F8
:100A9000C3E7FCF7BFF80223C4F8A80884F8AC3811
:100AA000DFE700BFCC50012000400008641C01209B
:100AB00060E3160010B5074A0124074B82F884450D
:100AC0009C73FFF7A1FFFFF7A9FC2046BDE810408B
:100AD0000DF042B99C1E0020CC50012090F89230BD
:100AE000B7EE007ADFED6A6A014607EE903A90F8B9
:100AF0009630684AB0EE476A05EE103A90F89430A6
:100B0000F8EEE77A04EE903A90F89530B8EEC55AD0
:100B100005EE903A90F8983067EEA67A04EE103A17
:100B200025EE265AF8EEE44AF8EEE55AB8EEC44A45
:100B300025EE275A64EEA64A65EEA65A24EE264A0A
:100B400064EE854A65EEA75A24EE274AB0EE473A8E
:100B5000F0B590F8917000F16F0602F11A050024CB
:100B6000137807EE903AF8EEE77A67EE857A67EE4B
:100B7000867AFDEEE77A17EE903AFA2BA8BFFA23B1
:100B800023EAE3730B72537807EE903AF8EEE77AB4
:100B900067EEA47A67EE867AFDEEE77A17EE903A72
:100BA000FA2BA8BFFA2323EAE3734B72937803EE80
:100BB000903AF8EEE33A63EEA57A67EE877AFDEEB7
:100BC000E77A17EE903AFA2BA8BFFA2323EAE373E9
:100BD0008B72938807EE903AF8EEE77A67EE847AA4
:100BE00067EE867AFDEEE77A17EE903AD5ED007A59
:100BF000B3F57A7FF8EEE77AA8BF4FF47A7323EA69
:100C0000E3738B812B68002B3FDD90F89730B0EEBB
:100C1000436A02EE903AF8EEE22AA2EEE66A63EE4A
:100C2000863A83EEA76AA2EEA66A65EEA77A013439
:100C300067EE877A67EE867AFDEEE77A17EE903AEE
:100C4000FA2BA8BFFA23BC4223EAE37306F8013F5C
:100C500000DDF0BD012C13D190F8933007EE103A6F
:100C600090F89B3006EE103AB8EEC77AB8EEC66A36
:100C700027EE267A26EE266A0435083208316FE719
:100C8000B7EE007AB0EE476AF6E7B7EE006ACCE757
:100C90000AD7233CCAA0050890F899306BB3B0F886
:100CA00064308BB190F89A20642102EB8203C3EB8D
:100CB0000313B3FBF1F3A0F86430962312FB03F3A4
:100CC000B3FBF1F3A0F8663043884BB190F89A304B
:100CD000642203EB8303C3EB0313B3FBF2F3438000
:100CE000B0F850304BB1962290F89A3013FB02F3D3
:100CF0006422B3FBF2F3A0F85030704790F8213033
:100D00004BB3438B83B190F82230FA22642113FB5A
:100D100002F203EB8303B2FBF1F2B3F57A7F428375
:100D2000A8BF4FF47A738383838843B1FA2290F883
:100D3000223013FB02F36422B3FBF2F38380C388F7
:100D40004BB190F8223003EB8303B3F57A7FA8BF51
:100D50004FF47A73C380704770B50B4C002504F5CF
:100D60006A7694F8913013B12046FFF7B7FE20461B
:100D70000135FFF791FF3046FFF7C0FF042D04F166
:100D8000EA04EED170BD00BF0052012010B5064C40
:100D90004FF48072002104F61E1047F027FC002358
:100DA000C4F8203A10BD00BFCC500120034BD3F84B
:100DB000240A08B108F016BF704700BFCC500120CC
:100DC00008B50B4605490246D1F8240A28B1044962
:100DD000FEF728F9BDE80840E8E708BDCC5001203F
:100DE000EDEB0008024B0146D3F8240AFDF700BFE3
:100DF000CC5001200048F5E7469206080CB4C30623
:100E000007B500D561B905A904980191FFF7D8FF8E
:100E1000FFF7F0FF012003B05DF804EB02B070476C
:100E20000020F8E708B5FFF7DDFFBDE80840E1E77F
:100E300010B504460348FFF7D5FF2046BDE8104033
:100E4000F0E700BF9282060810B508460749FDF793
:100E5000A7FC002815BF0124002405480548FFF71A
:100E6000E7FF2046BDE8104007F06EBF97820608F6
:100E7000A0820608C7820608034B0146D3F8240A5D
:100E800008B108F09BBE7047CC5001200CB407B5E8
:100E900010F020000BD079B92320FFF7EDFF05A952
:100EA00004980191FFF78CFFFFF7A4FF012003B026
:100EB0005DF804EB02B070470020F8E70FB407B507
:100EC00004A951F8040B0191FFF77AFF03B05DF814
:100ED00004EB04B07047194B1B682DE9F04153B384
:100EE0000025174FDFF864801648FFF79BFFFFF7D8
:100EF0005DFFFCF70FFEFCF743FE044640B11320F4
:100F00000CF078FEFFF776FF0F48BDE8F04189E767
:100F10003B78012BF3D040466E1CFFF7CFFF792DB5
:100F200002D12646FFF766FFFFF740FF64203546F3
:100F3000FCF72AFADFE7BDE8F08100BF2C1C012096
:100F4000E2290120E3820608FD820608A0A3060824
:100F50000FB407B504A951F8040B0191FFF730FF56
:100F6000FFF748FF03B05DF804EB04B070472DE9CC
:100F7000F041037903F0E002402A4AD009D82ABBA5
:100F800003F00703052B1CD8DFE803F0161B161B24
:100F9000090F602A44D0802A3ED0BDE8F081D0F805
:100FA00005102148BDE8F041D2E7D0F805205142B4
:100FB0001E48BDE8F041CBE7B0F80720B0F80510B7
:100FC000F6E7B0F90720B0F90510F1E746790024FB
:100FD000174D184805EBC605FFF704FF012395F8E8
:100FE0007072A74202D8BDE8F04103E7D5F86C6201
:100FF0004FEA840856F824204AB113B90E48FFF787
:10100000F1FE56F808100D48FFF758FF0023013491
:10101000E7E741790A48C5E7827941790948C8E795
:101020000948BDE8F04193E70383060819830608E1
:10103000849E05083083060884850608F89B060808
:101040004183060852830608698306082DE9F043A8
:1010500085B0224EFCF74EFD026983890025018888
:10106000044602928268DFF8888001924288DFF8A5
:1010700084901B4F009242681A48FFF769FF15B928
:101080001948FFF7CFFED8F800309D4212DA3378C6
:10109000052B20D809EB8303D3F82424B3882946F1
:1010A000013538460093063636F8043CFFF750FF0A
:1010B000062DE4D141F048F84288838864689B1A81
:1010C00003FB0444FCF7A8FD02460848214605B08E
:1010D000BDE8F0433CE70022E0E700BFF45A0120FE
:1010E000EB83060881830608DF830608FA83060877
:1010F000D8290120849E05080249034801F5216191
:101100000EC925E70070F01F1784060870B500228D
:10111000124C134D134E94F8FF3403F0010302B147
:1011200070BD002BFCD001212846FFF711FF752070
:1011300027F06AFD01463046FFF70AFF1A2027F024
:1011400063FD01460848FFF703FF1B2027F05CFD05
:1011500001460648FFF7FCFE0122DCE7CC500120E7
:101160002B840608378406084A8406085D8406082E
:10117000BE4BBF491A68BF4BBF482DE9F047BF4C73
:1011800090B0BF4D4FF00008BE4F4646B2FBF3F2A1
:10119000FFF794FEB4F84C2A4FF47A730A20B2FB9E
:1011A000F3F103FB1122B4F94E3A92B2B2FBF0F222
:1011B000B548FFF7CDFEB54AB549B648FFF77EFE04
:1011C000FFF718FEA17BB44A05EB8101B34BB4488D
:1011D000D31AD1F83C14B4F85220FFF7B9FEFFF748
:1011E00009FEB048FFF7FEFD94F8501AAE48FFF72D
:1011F00065FEAE48FFF7F6FDB4F8522A94F8541A8B
:1012000092B2AB48FFF75AFEFFF7F4FDA949AA488E
:10121000FFF754FEDFF8149394F8FB3403F0010356
:10122000B8F1000F00F0EA80002E40F01B81A348C7
:10123000FFF7F8FDA24F0126D4F85C8ADFF8F092A0
:1012400007F1180A0123B34013EA080F15D019F863
:10125000062057F826305AF8261053F822209948CD
:10126000FFF72CFE012E06D1864B93F8A51511B180
:101270009548FFF723FEFFF7BDFD0136062EE1D1AD
:101280009248FFF7AFFDD4F8FC351B0640F183818F
:1012900094F87C3A032B8CBF8D488E48FFF7A2FD53
:1012A00094F8AC35022B40F045818B48FFF79AFD4E
:1012B00094F87C3A042B00F265818848FFF792FD90
:1012C00094F88C3A002B00F0648105EBC303D3F84B
:1012D0001C158348FFF7F2FDFFF78CFD94F8943A54
:1012E000D4F8906A05EB83037E48D3F85015FFF7D6
:1012F000E5FD26B1327A717A7B48FFF7DFFDFFF713
:1013000079FDFCF7F7FB016921B182687748120D7E
:10131000FFF71EFEFFF76EFD754B764819684FF418
:101320007A73B1FBF3F1FFF7C9FD05A8FEF766FB81
:1013300038B105A908A845F0BFFA08A96E48FFF71B
:10134000BDFDFFF757FDD4F8208BB8F1000F00F07A
:10135000268107EE908ADFED696AB8EEE77AC6EE7D
:10136000877AFDEEE77A17EE903A654F97F86001BD
:1013700030B1644A039392ED050A46F0D9FB039B12
:10138000D4F8A06A5EB107EE906ADFED5C6AF8EE11
:10139000E77A86EEA77AFDEEC77A17EE906A394AA9
:1013A000B2F8F41542466429CDE90006A8BF6421CD
:1013B0005548FFF7CDFDB7F8642164235348544ED8
:1013C000B2FBF3F103FB112297F8753105EB8305AE
:1013D00092B2D5F864350125009397F87431FFF780
:1013E000B7FD4C48FFF7FEFCD4F8FC48002C40F059
:1013F000D880FFF7FFFC10B0BDE8F087002B3FF46A
:1014000013AF16B14846FFF7EDFC01214248FFF744
:1014100055FD94F8583A3E4805EB8303D3F844143D
:10142000FFF74CFD97F8D633DA0702D53B48FFF7B4
:1014300045FD97F82031032B09D03948FFF73EFDD1
:1014400097F82031012B02D13648FFF737FDFB6CAE
:1014500001265B7BB046B3427FF6DEAE3248FFF733
:101460002DFDD7E6FFF7C6FCE4E600BFBC1C01205B
:101470007884060840420F0082840608CC50012080
:10148000849E05089C1E002094840608000001200C
:1014900000080000B684060800800008004000082C
:1014A000C8840608DF840608F1840608F984060863
:1014B000FB8406080F850608148506083385060890
:1014C0002CA30508F69F0608388506083C85060803
:1014D000428506084E8506085E850608F7A20608BE
:1014E000A2850608BE850608C7850608D1850608B8
:1014F000641C0120EC850608068606080024744951
:10150000C461012078030120198606085F86060859
:10151000AE8506088486060819850608E69B060837
:101520001E850608268506082B850608848506087C
:101530008403012002200CF077F8064608B9204801
:10154000B4E690F904003EF021FF074631F038FA86
:1015500005EB80003946D0F8D8241A48FFF7AEFCD6
:1015600094F8AF35012B04D11748FFF73BFC17481F
:101570009CE6B379164805EB8303D3F8D814FFF73C
:101580009DFCF4E794F8AE350BB9124896E6124884
:1015900094E612499DE61248FFF724FC9CE6434678
:1015A000E3E694FAA4F0B0FA80F005FA00F024EA39
:1015B00000040BF047FF01463046FFF77FFC15E7BC
:1015C000648506086E8506087E85060883850608FC
:1015D000B69406088785060897850608708406086D
:1015E000B28506082DE9F04FDFF86C8199B098F8C4
:1015F0000330002B00F093804E4800254E4EDFF85C
:101600005CB1FFF70FFC2F46DFF85491DFF854A1CF
:101610000BA9E8B210F006FF9DF83430002B53D030
:10162000139C54B107EE904A9FED440AF8EE677A96
:1016300080EE270A46F07CFA04460B9A2946584663
:10164000FFF73CFC109A002A6BD002FB04F04FF429
:101650007A73B0FBF3F30993DDF848C0BCF1000FD7
:1016600061D00CFB04F142F21073B1FBF3F1082DD1
:1016700098F8033018BF7F18002B56D017984FF4F6
:101680007A7E0A230790159806901698059011986F
:10169000B0FBFEFECDF810E00998B1FBF3FE03FBB2
:1016A0001E11CDE902E10999B1FBF3F103FB110031
:1016B000BCFBF3F3CDE9001021465046FFF748FC90
:1016C0000023B362C6E90D33013540361F2D9FD18B
:1016D00098F8033003B31A4C4FF47A731948D4E9DD
:1016E0005E12B1FBF3F3D208D4F88011FFF730FC9F
:1016F0000A22154897FBF2F102FB1172FFF728FC52
:10170000124B1B78432B04D11148D4E96121FFF718
:101710001FFC0023C4F8803119B0BDE8F08F0D48DC
:101720006BE7099298E76146A1E721464846FFF733
:101730000FFCC5E79A860608645B01208096184B6B
:10174000C461012041870608618706080529012038
:1017500085870608F8860608CC500120028706080F
:10176000949B060811870608234870B5FFF73AFBDB
:10177000224B93F86031002B38D0214B93ED050AB2
:1017800046F0D6F901461F48FFF7E2FB1E4C1F4802
:10179000FFF728FB1E4B94F839051E4A00280CBFA2
:1017A00010461846FFF73EFB94F8393513B31A4C30
:1017B0001A48B4F88A16FFF781FB194E94F8880688
:1017C000184D00280CBF30462846FFF72BFBB4F815
:1017D0008C161548FFF772FB94F8890600280CBF99
:1017E00030462846BDE87040FFF71CBB0F48FFF7A6
:1017F00019FBCBE770BD00BFBF870608C46101209D
:1018000078030120D9870608CC500120E887060814
:101810007E83060821A806089C1E0020F98706087A
:10182000B8870608AF87060820880608DE870608FE
:101830000EB403B503AA52F8041B0192FDF74CFE47
:10184000064BD3F8242A1AB90549586DFDF7D0F98B
:1018500002B05DF804EB03B0704700BFCC5001202C
:10186000469206082DE9F04798460B7981460F46C7
:1018700003F0E0051646402D32D10024634DDFF819
:10188000A881DFF8B09116E03B7903F00703013B34
:10189000042B04D8DFE803F014171A1D2100315D72
:1018A0005A48FFF70BFB7B79013BA34202DD484618
:1018B000FFF798FA01347B79A342E5DCBDE8F087B5
:1018C00031572846EDE736F81410FAE736F91410C8
:1018D000F7E756F824104046E3E756F82410F0E7FF
:1018E00003F00703052B57D8DFE803F0031F272970
:1018F0002C3E3478602D55D02CD8002D75D1B7F8FA
:101900000550B7F8076021464048FFF7D7FAAC42C8
:1019100039DBB44237DCB8F1000FCFD0324629466C
:101920003B48BDE8F047FFF7C9BA96F90040602D83
:1019300038D00FD8002D58D151E03488DAE7B6F905
:101940000040F4E7D6F800A0202D54464DD034D9FD
:10195000602D27D0802DB1D132782E4B2E48002A11
:1019600014BF3146194635E0202D34683DD0EFD8FC
:1019700021462648FFF7A2FAD7F80510A14202DB5C
:101980004B42A34221DDFFF735FA23463A68484629
:101990002249BDE8F0474BE7202D25D01ED9602D08
:1019A000D8D100247B7944FA03F3DB07BDE8F04784
:1019B0004CBF1B481B48FFF781BA51461A48FFF736
:1019C0007DFAD7F805108A45DDD8B8F1000F3FF44D
:1019D00075AF1648BDE8F047FFF770BA0024B7F9B5
:1019E0000550B7F907608EE700247A79104B03EBB6
:1019F000C20393F87022A242C5DDD3F86C3253F8CB
:101A00002400BDE8F047FFF7EDB900BF2D830608BD
:101A1000A8950608C7A20608F89B06084688060887
:101A20007E83060821A80608168306084088060853
:101A3000849E0508F984060870B5164605460C46CE
:101A40000846FDF7E5F83346024621462846BDE83C
:101A5000704007E70EB403B503AA52F8041B0192C5
:101A6000FDF73AFD044B0549586DFDF7C1F802B08A
:101A70005DF804EB03B07047CC5001204692060895
:101A80000049E7E760880608F8B50C4606460846B0
:101A9000FDF7E8FE20210546204646F0BEFD04463F
:101AA00018B93046BDE8F840EAE7114F0134114E4D
:101AB0003B7832789A4201D0FCF7A4F90E4B2046CD
:101AC0001D6045F047F8012201462046FCF738F931
:101AD0003B7832789A4201D0FCF794F9204645F0E1
:101AE00039F82A4601460548BDE8F840FFF730BA04
:101AF000281C0120E3290120241C012077880608E6
:101B00002DE9F0410D4688B006460846FDF7AAFECD
:101B100020210446284646F080FD20B9304608B012
:101B2000BDE8F041ACE7FDF79DFE224605460146C3
:101B30000F48FFF70DFA85B1202D2A466946204649
:101B400028BF2022E846FCF7A5F900270646B74241
:101B500008DBAD1B3444002EEDD1FFF74BF908B084
:101B6000BDE8F08118F8010B0137FFF785F9EEE7C2
:101B70008D88060810B504460748FFF753F9FCF7AF
:101B8000B9F920B10548BDE81040FFF74BB9204630
:101B90000349BDE810405DE7A5880608AF88060840
:101BA000B7880608154BD3F88C312DE9F04104466F
:101BB00088B0F3B11A6804A91846D56A6A46A847DE
:101BC000064688B104AC6D460027DFF83C8001373B
:101BD00035F8022B34F8021B4046FFF7B9F9BE4234
:101BE000F5DC08B0BDE8F08105492046FFF732FF7B
:101BF000F7E7044908B0BDE8F0412BE7C4610120D4
:101C0000D8880608F0880608BE88060870B505461C
:101C100008460C4644F09EFF024668B10F2804D1E6
:101C20002146084846F017FD30B12846054B064AC4
:101C30000649BDE870400DE702490548BDE870401F
:101C4000FFF786B9F788060807890608128906088B
:101C50003C89060870B5054608460C4644F07AFFF4
:101C6000024668B1042804D12146084846F0F3FC36
:101C700030B12846054B064A0649BDE87040E9E602
:101C800002490548BDE87040FFF762B94A89060875
:101C90004F890608128906085F8906082DE9F04376
:101CA00007469BB008460C4644F054FF06462022E7
:101CB000002101A846F09AFC2EB3402E07D0402305
:101CC00032463A4938461BB0BDE8F043C2E601ADA2
:101CD00004F140084FF0000902222146684646F010
:101CE000CCFC0023102209A968468DF80290FDF76C
:101CF0002FFD099B0DF10202934223D1023405F816
:101D0000010BA045E8D109AC41220021284D204615
:101D100046F06CFC002E3DD095F89061D6B12022A3
:101D200005F2911101A846F037FC98B105F2911126
:101D30002046FDF763FC23461E4A38461E49FFF73E
:101D400089FE04E01A7838461C49FFF783FE1BB071
:101D5000BDE8F0831A4B93F83030DBB9D6B901AB4C
:101D6000184E1A46083603CAA24246F8080C46F82E
:101D7000041C1346F5D101232046124985F8B131E0
:101D8000FDF73CFC1048FFF753F821460F48FFF7DA
:101D9000DFF8DCE795F8B1311BB995F89031002BED
:101DA000F3D008492046FDF729FCEEE772890608C2
:101DB000C4610120B08906081289060894890608C2
:101DC000CC50012055630120BA890608C98906084C
:101DD0002DE9F74FDFF82081834608460C4644F092
:101DE000B9FED8F8A875064628B102463349204600
:101DF000FDF772FC80B9394631483EF04DFA314961
:101E0000314821EA07013EF047FA3049304803B033
:101E1000BDE8F04F3EF040BA23782D2B23D101349A
:101E2000013E4FF0010A2B4B4FF000094FF0FF35F8
:101E300053F8041B51B1324620460193FDF74CFC88
:101E40000028019B0ABF4D460021012109F101092B
:101E5000A1B9B9F11D0FEBD122461F49584603B075
:101E6000BDE8F04FF6E54FF0000ADCE73B431B49C5
:101E7000C8F8A8351A4B12E01A4913E00123114A99
:101E8000AB401A40002AF7D007EA0302BAF1000F6C
:101E9000ECD027EA03031449C8F8A835134B002AED
:101EA00018BF1946124B134803EB8503D3F8782566
:101EB00003B0BDE8F04FFFF74BB800BFFD86060842
:101EC000018A0608BDD455180B8A0608422BAAE7DA
:101ED000178A0608FCA30508258A0608F98906085A
:101EE000F2890608D6890608E2890608E989060803
:101EF000849E0508EB940608CC5001202DE9F74F8D
:101F0000019008460E461746984644F023FE0446C4
:101F1000E8B93F4D3F48FEF7D1FF20460BF0AAFA43
:101F20003B68184206D020460BF0B6FA0146284618
:101F3000FEF7C4FF0134172CEFD13B6813B93648C4
:101F4000FEF750FF03B0BDE8F04FFEF753BF024667
:101F500032493046FDF7C0FB0546A8B92C46304D46
:101F60003048FEF73FFF20460BF084FA10EA080FD6
:101F700006D020460BF090FA01462846FEF79EFF59
:101F80000134182CEFD1DDE733782D2B29D1013620
:101F9000013C01254FF0000948F4000B48460BF0C6
:101FA0007BFA2246824601463046FDF795FB18BB78
:101FB00048460BF05FFA1BEA000F1DD09DB1B9F146
:101FC000170F02D03B6840EA03081748C7F80080A3
:101FD000FEF708FF5146124803B0BDE8F04FFEF788
:101FE000B7BF0025D6E7B9F1170F02D03D6825EA43
:101FF00000050E483D60EBE709F10109B9F1180F42
:10200000CCD132460A49019803B0BDE8F04F21E532
:10201000AD850608368A0608408A0608FD86060849
:10202000AE850608478A0608E9890608F989060880
:10203000258A060840F20223004A5FE7B4570120D0
:10204000014B024A5AE700BFFFFF7F00AC57012057
:1020500010B5044622F0B6FF20B920460449BDE879
:102060001040F7E40348BDE81040FEF771BF00BF21
:10207000528A0608618A06087FB505460C4611F8A3
:10208000013B202BFAD033B10622B1492046FDF79F
:1020900023FB00285FD1AF4C94F81402FCF7F8FC46
:1020A000D4F818220146AC48FEF752FF94F81432D7
:1020B000882B04D1D4F81C12A848FEF749FFA84B7E
:1020C00094F82A02A749B4F82822002818BF194614
:1020D000A548FEF73DFF94F8212294F82012A3486A
:1020E000FEF736FF94F84422D4F84012A048FEF7D9
:1020F0002FFF94F8FC21032A29D8012A06D09D4BF2
:1021000003EB8203D3F8EC15002207E09A4BD4F8D6
:1021100000221B689949D21A22EAE2729848FEF717
:1021200017FF94F80A22042A13D8924B03EB820378
:10213000D3F8FC1594F81002924A934B002818BF6C
:102140001A46924804B0BDE87040FEF701BF9049BE
:10215000DAE78F49EEE708228E492046FDF7BCFA00
:1021600040BB7C4C94F8542252B91146232030F0E5
:1021700009FF28B98849284604B0BDE8704069E4E1
:1021800094F84F328548019394F84E320093B4F896
:102190004C32B4F84A22B4F84812FEF7D9FE94F84B
:1021A000540270496E4BD4F85022002818BF1946CB
:1021B0007B48C7E707227B492046FDF78DFA024698
:1021C00038B90146012030F0DDFE624B93F85C42E5
:1021D00010E00A2274492046FDF77EFA58BB5D4C98
:1021E000012304227149162084F8103230F0CAFE0F
:1021F00094F85C42032C00F275815E4B03EB840380
:10220000D3F81016534D95F81402FCF741FC95F8DD
:10221000213202466648009395F82032FEF798FE78
:10222000012C40F06181B5F82032B3F5837F40F096
:102230005B81604831E008225F492046FDF74CFA97
:1022400030B9444C04225D4984F810021720CDE7D0
:1022500008225B492046FDF73FFA18B90422594984
:102260001120B0E7062258492046FDF735FA18B983
:10227000042256491020A6E7042255492046FDF7BE
:102280002BFA042270B95349252030F07BFE314BE4
:1022900093F85C42002CADD14F4804B0BDE87040CB
:1022A000FEF756BE4D492046FDF716FA0028DFD04E
:1022B00004224B492046FDF70FFA002840F0F78032
:1022C0000434264601343378202BFAD000230A2226
:1022D00044493046ADF80E30FDF7FEF9C0B90DF1B6
:1022E0000E0306F10A024049284601934FF6FF7398
:1022F000009301233DF004FF002800F0F580BDF8B5
:102300000E30022203A920205BBAADF80C305AE748
:102310000F2236493046FDF7DFF900286AD10DF16A
:102320000E0306F10F023249284601934FF6FF7360
:10233000009302233DF0E4FE002800F0D580BDF8B4
:102340000E30022203A921205BBAADF80C303AE727
:102350008A8A0608C4610120918A0608AF8A0608A5
:102360006C8A0608708A0608EC8A0608078B06083D
:102370002E8B0608849E0508641C0120738A0608BB
:102380005C8B0608868A06087D8A0608878B060805
:102390002EA30608C79C0608A48B0608C48B060853
:1023A000328C06084E8C0608568C0608AC1E0608B1
:1023B000CC8D0608F38D0608588C0608B41E060856
:1023C000618C0608BC1E06086A8C06081C180608E4
:1023D000DB9C0608C41E0608A48D0608718C06083E
:1023E000768C06087B8C0608868C0608908C06087E
:1023F000A08C060811223D493046FDF76DF9B8B9A9
:102400000DF10E0306F1110239492846019347F6F2
:10241000FF73009332233DF073FE002864D0BDF8B3
:102420000E30022203A922205BBAADF80C30CAE6B6
:10243000112230493046FDF74FF90346B8B90DF186
:102440000E0201242C492846019206F11102009443
:102450003DF056FE002847D09DF80E30224603A9D5
:102460002420003B18BF01238DF80C30ABE6172267
:1024700022493046FDF730F90346B0B90DF10E029E
:1024800001241F492846019206F1170200943DF0ED
:1024900037FE48B39DF80E30224603A92620003BA4
:1024A00018BF01238DF80C308DE6164963E6032230
:1024B00015492046FDF710F9042210B913491320DD
:1024C00081E613492046FDF707F918B9042211499E
:1024D000142078E622461049284604B0BDE8704032
:1024E000FFF7B8BA0D498DE604B070BDAF8C060891
:1024F000C18C0608D28C0608E48C0608F58C060808
:102500000D8D0608248D06086D8C0608CC1E060865
:10251000888D0608D41E06088D8D06082EA3060891
:10252000074B10B50446D3F8600230F0C1F928B962
:1025300020460449BDE81040FFF78CBA10BD00BF2B
:10254000C4610120708E060870B50546084616461F
:10255000FDF788F90D4B041E93F8FC230EDB944223
:1025600005DA21460A48FEF7F3FC204670BD2EB17D
:10257000FF2C03D10748FEF7EBFCF6E7013A0649CA
:1025800028464FF0FF34FFF765FAEEE79C1E002067
:10259000868E0608978E0608AA8E06082DE9F04F4B
:1025A000074691B082480E46824DFEF7D1FC0023CB
:1025B00081494024062285F868323046012391F88B
:1025C000FC13C5F864D285F8694207F0CDFA0A20F9
:1025D000FAF7DAFE95F868320C2BDAB240F2E480B2
:1025E0009DF80C60FE2E2CD0FF2E15BF0F24152455
:1025F00000250125944240F0D780611E6846C9B28B
:1026000037F020F804F140030DEB030414F8413CCB
:10261000834240F0C4806A1E9DF80D30012A12D911
:1026200003F01F075C0961376448FEF7DBFB022DEE
:1026300039D0013C042C34D8DFE804F00B2D2F33C3
:1026400031000225D6E79DF80E701E469DF80F401A
:10265000EAE75B486C464FF00008DFF8BC91FEF7F4
:10266000E1FBDFF8B8A1DFF8B8B15648FEF7BAFBD6
:1026700008F1010814F8011B4846FEF71FFCB8F1E9
:102680000C0F16D00AFB08F3B3F1553FF0D85846AB
:10269000FEF7A8FBECE74C48DCE74C48DAE74C488F
:1026A000D8E74C48D6E700230DF11F008DF83F30E6
:1026B000D0E7FEF79FFB022D3AD064223B46464806
:1026C000B6FBF2F102FB1162C9B2D2B2FEF740FCD6
:1026D00085F001035B42DBB2012B59D83F4A404BE6
:1026E0009DF810103F4800290CBF114619463E4E78
:1026F000FEF72EFC9DF811103C4B3D4800290CBF05
:1027000031461946FEF724FC022D41D19DF81240B6
:102710003848FEF767FB8CB1FF2C1FD00A233648E0
:10272000B4FBF3F103FB1142D2B2FEF711FC08E057
:102730003A4631463148FEF70BFCCFE73046FEF70C
:1027400071FB9DF813402E48FEF74CFB44B1FF2C63
:1027500021D021462B48FEF7FBFB04E02A48EEE798
:102760002148FEF75FFB0DF1130500241E4E1F4F9D
:10277000DFF8948015F8013F7BB1FF2B14BF3A4678
:102780004246214601342148FEF7E2FB042CF1D1F8
:1027900011B0BDE8F08F1C48E3E73246F1E71C4971
:1027A0003846FFF757F9F3E71A48FEF73BFBEFE728
:1027B000EC8E0608C46101209C1E0020FD8E0608D8
:1027C000088F06082E8F06080F8F0608178F060839
:1027D0001F8F060870840608408F0608D98E0608E9
:1027E000D08E0608778F0608868A06084B9D060855
:1027F0008E8F0608958F0608A98F06085C8F06083D
:10280000B18F06082D830608E08E0608C18F0608E2
:10281000CC8F0608DC8F06088D820608ABAAAAAA10
:10282000C7A206082DE9F84307460C46DFF8A49036
:10283000204644F08FF9064660B91E4B1E4893F8B7
:1028400010251E4B03EB8203D3F81C16BDE8F8439A
:10285000FEF77EBB024649462046FCF73DFF60B1CD
:10286000DFF86080002558F8041BB1B922463846CD
:102870001349BDE8F843FFF7EDB8124C124D134869
:10288000FEF7B0FA54F8041B19B12846FEF716FB00
:10289000F8E7BDE8F843FEF7ADBA32462046013509
:1028A000FCF71AFF0028DED1024B094C83F81055C3
:1028B000BEE700BFCC500120E58F0608849E0508C6
:1028C000258A0608A4A40508AE850608478A0608D6
:1028D00010A90608FD86060838B50D4604460522EF
:1028E00019492846FCF7F8FE68B9184B93F85820A8
:1028F00022B9012183F8592083F858101448BDE803
:102900003840FEF78FBA032212492846FCF7E4FE4E
:10291000A0B90E4D95F8583063B195F859304BB1C8
:102920000D492046FFF796F8002385F8583085F8C2
:10293000593038BD0948FEF775FAF5E720460849D1
:10294000BDE83840FFF786B8A29C0608CC500120AD
:10295000EF8F0608F49D0608059006083C900608CF
:102960005090060870B5194C054694F858307BB164
:1029700094F8593063B11649FFF76CF828461549A9
:10298000FFF768F8002084F8580084F8590070BDFB
:10299000114B93F8B121B2B193F890219AB903F297
:1029A000911203F51B7503F2B1161068083252F844
:1029B000041C2C46B24203C42546F6D1012283F8FA
:1029C000A72208F015FB0120E1E700BFCC50012051
:1029D000059006085F900608C461012008B503460B
:1029E00010460AB9002008BDDB0601D50029FAD03F
:1029F000FEF71EFAF6E7F8B50D4E054696F83030AC
:102A000093B9F8BD25B12388C3F30B039D4204D0CD
:102A1000A288D4E9020145F0F3FC1C34BC42F1D396
:102A2000002386F83030ECE7024C034FF6E700BF96
:102A3000CC500120A0E50608D0EE06082DE9F04FA5
:102A4000164685B0334C1A464FF00009A246CDE930
:102A5000010100213046FFF7C1FF06F0100300908E
:102A60000393FEF7A3F92379029A03F01803934224
:102A700003D0002A44D1182B42D14FF00D0B0BFB91
:102A800009A3B3F8090038F051F980462046FBF756
:102A9000AAFF0746D8E90221024401442046FBF779
:102AA0005BFF80F001010546009AC9B23046FFF78E
:102AB00095FF039B009003B115BB0BFB09FBB3060D
:102AC0005AF80BB00ED56DB959461348FEF7F6F912
:102AD000D8F808202B4621463A440198FEF7C2FE5A
:102AE000FEF788F959460D48FEF7E8F9D8F80C20AA
:102AF000002321463A440198FEF7B4FEFEF77AF926
:102B000009F1010940F271230D349945A9D105B0AD
:102B1000BDE8F08F20B705087D9006087E90060876
:102B20000149FEF797BF00BF8890060838B50C46EC
:102B3000054615492046FBF733FE30B9FEF70CF980
:102B40001248BDE83840FEF76DB911492046FBF741
:102B500027FEA0B90F4B83F8C50183F8CD0183F898
:102B6000AF0283F8B70283F8990383F8A10383F8CF
:102B7000830483F88B0483F8FD040748E1E72846C3
:102B8000BDE83840CCE700BF979006089D90060846
:102B9000B8900608CC500120C09006082DE9FF47E8
:102BA000074608460D4643F0D5FF082846D105F1F3
:102BB000FF3801AE073531464246B14612F8010FE3
:102BC000FCF784FD01F8010BAA42F7D10023DFF8DE
:102BD00080A08DF80C30A84518D11C49484622F039
:102BE00083F91A4808231A4910F8012B013B11F800
:102BF000014B02F110026A4402F80C4CF4D101A915
:102C000014488DF80C30FEF7A3F914E018F8010F02
:102C1000FCF75CFD0446014606F8010B504645F002
:102C2000FCFC28B12146304645F0F7FC0028D2D004
:102C30003846FFF775FF04B0BDE8F0870028D0D014
:102C4000384604B0BDE8F047FEF71ABFE45501204E
:102C5000601E0608DC90060807B5009313460A4676
:102C60000249FEF7F7FE03B05DF804FBE3900608A7
:102C700020B10078B0FA80F0400970470120704719
:102C80002DE9F74F81460846FFF7F2FF0E4605464D
:102C900070B1002401A9204601343DF08DFB0146AE
:102CA0004846FFF7EDFF122CF4D103B0BDE8F08FDA
:102CB0000846FCF7D7FDC4B2112C71D83C4D701CEE
:102CC000FBF7FFFF3B4E05EB44088346670098F88F
:102CD000A8A2B8B9AAF102014B424B413D4495F874
:102CE000A822B25C002B54D095F8A932192040F2EA
:102CF000EE2100FB031321462F4803B0BDE8F04F3F
:102D0000FEF726B90178304645F087FC80B1032CE8
:102D10002A49A0EB060394BF0022012202EB4202E3
:102D20000A4452FA83F393F890A6BAF1030F04D140
:102D3000484603B0BDE8F04FF2E65846FBF7C1FF46
:102D4000F0B1BAF1020FF3D1FCF78CFD40F6CA03E3
:102D500080B29842A8BF184640F2EE239842B8BF0E
:102D600018461923A0F2EE20B0FBF3F088F8A90270
:102D7000AAF1020253425341EA1982F8A8A2ADE730
:102D8000BAF1020FF4D1484603B0BDE8F04FFEF7A8
:102D900077BE21460A4803B0BDE8F04FFEF7D8B829
:102DA00011232A460749484603B0BDE8F04F53E7D0
:102DB000C4610120E4200608FC900608849E0508F2
:102DC0000C910608199106082DE9F04F0346A1B0B1
:102DD0000846FFF74DFF054628B1184621B0BDE86B
:102DE000F04FFEF74DBEFF23DFF8C09207464FF0CD
:102DF000FF388DF82830D9F860320B9093F83820DE
:102E0000ADF830000D908DF838200F90ADF84000EF
:102E100011930991CDE90500934909A845F0BAFA43
:102E2000044618BB01460AAC904F0B0190481A5754
:102E3000002310F9016BB24240F0D2804E1C1046C4
:102E40003DF0A4FA024631463846FEF781F8022EDC
:102E50004FF00101E9D19DF938A09DF92830534583
:102E600040F0C5808348FEF773F84DE02378002BCF
:102E7000D2D0032FD4BF00260126062F00F2A9804E
:102E8000DFE807F00447509104475000042F10D0AA
:102E900079492046FCF744FC58B14FF480600AF0B1
:102EA000C3FB002800F0B58190F9040001230693CC
:102EB0000AE072492046FBF773FC70B9D9F860321A
:102EC00093F93800042F22D0119B119320AB03EB10
:102ED000061606F8580C01379EE720463DF04CF9DF
:102EE0000028EFDA01230A2212A92046FCF730FC61
:102EF00040B2002803DB129B1B78002BE2D0224655
:102F0000711C5F48FEF724F821B0BDE8F08F002364
:102F1000DBE72046FCF7A6FC20AB03EB061646F8E1
:102F2000540CD8E757492046FCF7FAFBB0F1000AE9
:102F30005549204618BF4FF0010AFCF7F1FB08B1D4
:102F40004AF0020A3301DFF868C1079320AB03EBB4
:102F50000616BCE80F0006F850AC12AE0DF1480A98
:102F60000FC6BCE80F000FC6BCE80F000FC69CE8F8
:102F7000030086E803000026B346DAF80010204676
:102F800045F09AFB10B19AF804301E430BF1010B87
:102F90000AF1080ABBF1070FEFD1079B80336B449E
:102FA00003F84F6C97E739492046FBF7F9FBA0B1CE
:102FB00037492046FBF7F4FB00288CD02046FCF76D
:102FC00051FC0328804686D901463248FDF7C0FFF0
:102FD0009AE722460821304894E7012305937AE7CF
:102FE0000133072B7FF425AF01312C488AE70B9B77
:102FF0001BB9AAF114025542554100235F1CE36836
:10300000002B62D194F900B058460AF0DFFAD4F8E8
:10301000049018B10668002E40F08B80B9F1000FC3
:10302000237A14BF4E464FF46146666023B91C48AC
:10303000FDF78EFF03232372627A2AB139461948BD
:103040000792FDF785FF079A02925846237ACDE949
:10305000006300231A4619460AF028FBE06048BBCB
:1030600039461148B2E700BFE6A30608A391060857
:1030700054A50508C09106083C910608479106082A
:103080004B91060866910608789D06086991060826
:10309000428A06086F91060887910608AE910608D5
:1030A000D9910608F49106080F920608C461012020
:1030B0001CA5050858493346584A5948B9F1000F2C
:1030C00018BF0A463946FDF7F9FE022F04F1100435
:1030D0004FF0010392D1119E0D9F4DB15148FDF764
:1030E000A1FE33681B6A1BB13A464F4930469847E8
:1030F000059B002B50D04D49474BBAF1140F18BF18
:1031000019464B48FDF724FFBAF1140F09D1059B6E
:10311000002B43D03368DB691BB1002245493046A0
:103120009847069B002B43D10022314638463DF09C
:103130003BF8E660B9F1000F2CD04946304602F06A
:103140006BFF3D4AB36839463C48FDF701FF94F8F0
:103150000890B9F1000F0CD03279914509D04B4657
:1031600039463748FDF7F4FE3368494630469B69D7
:103170009847637A23B1727939463248FDF7E8FE01
:10318000F36A002BA1D039462F48FDF7E1FE00235A
:10319000F3629AE7204AD5E71F49B2E7B8F1000F7A
:1031A000BFDB3368DB69002BBBD042462749B6E75B
:1031B000DFF89C900025DFF89CA04FF0030B06F091
:1031C00043FF0520FAF7E0F89AF8FC33AB42ABD99D
:1031D00019F8014FC4B1204607F028F8804698B18D
:1031E0002046F7F713FD0446EBB210B180F806B0A5
:1031F000C37120460121F7F797F998F80630204669
:10320000DB0703D5F6F74CFD0135DDE7F6F742FDA8
:10321000FAE74FF0FF3049E610A9060821910608A9
:103220002B920608E1920608196001082F91060802
:103230000A930608DBEC00082A9106084992060862
:103240006E92060891920608C892060851EA000894
:10325000232801209C1E00202DE9F74F0546084633
:10326000FFF706FD0B46044618B9334A92F8CC72B4
:1032700027B9284603B0BDE8F04F51E42646DFF8F1
:10328000CC90DFF8CCA001AA2C49184645F0AFF845
:1032900010B906F0E5FE08E056B9012201462846BD
:1032A000FFF752F9421C04461BD103B0BDE8F08F72
:1032B000FCF7D8FA2F28834637D80FB106F0C4FEA2
:1032C000BBF1060F14D01E4901235FFA8BF291F86F
:1032D000FC13E0B206F048FC002759464846FDF7CB
:1032E00037FE01AA15490020013645F080F8CFE7E6
:1032F000DAF8FC351B0114D5FF2C0ED0E1B22846BC
:10330000FFF74CF9E8E701372846FFF747F9F9B22C
:1033100098F8FC238A42F6D8DEE70027DFF8208001
:10332000F5E70848FDF77EFDD6E72F220649284637
:10333000FEF790FBD5E700BFC4610120E6A30608B5
:103340009C1E0020528A06083E9306082D9306080C
:10335000CC5001202DE9F74307460846FFF788FCCB
:103360000B46044628B1384603B0BDE8F043FEF7EB
:1033700087BB01AA2E491846264645F038F8A046D4
:103380000546DFF8AC9065B92A4B3246A1B2D3F8B6
:10339000600241F0FDFC68BB27493846FEF75AFB46
:1033A00028E0B8F1000F06D0B8F1010F25D038465B
:1033B000FEF766FB1EE0284643F0CCFB1F4906469D
:1033C00002462846FCF788F950B332461C49284685
:1033D000FCF782F930B332461A492846FCF77CF9EB
:1033E00010B3324618492846FCF776F9F0B1384652
:1033F000FFF796FB03B0BDE8F083B31E29463846BD
:103400005A425A41FFF7A0F8421C0446F2D001AAE2
:103410004946002008F1010844F0E9FF0546B2E7FB
:103420004646F4E70126F2E70226F0E70426EEE737
:10343000E6A30608C46101206A9306085E930608A5
:103440006193060864930608679306082DE9F7431D
:1034500080460846FFF70CFC0B46054628B140465F
:10346000FEF70EFB03B0BDE8F08301AA2D49184614
:103470002F4644F0BCFF2E460446DFF8A8907CB9E6
:10348000022DECD1A7F57A73B3F57A7F21D94FF4E9
:10349000FA634FF47A7224494046FFF7DDFBE1E717
:1034A0004DB1012D10D001AA49460020013544F04C
:1034B0009EFF0446E3E7012221464046FFF744F819
:1034C000431C0646EFD1CDE72046FCF7CBF9074673
:1034D000E9E7164DB8B2D5F898365B689847FCEE28
:1034E000C07AFF2E17EE902A0BD195F8FC13B6EE9A
:1034F000C00A0F4BA14210DC11460E48FDF728FD13
:10350000B0E70D4B31460D48B6EEC00A03EB86031B
:1035100083EDB40AFDF71CFDA4E70134A3EC010A16
:10352000E8E700BFE6A30608789406089C1E002082
:103530009464012095930608C461012088930608CD
:10354000F8B507460846FFF793FBC8B11F4B9E69C5
:1035500001363046344609F09FFF0546F0B9013484
:10356000182CA8BF0024204609F096FF0546A8B9EC
:10357000B442F4D138461649BDE8F840FEF76ABABD
:103580000846FCF76FF9044609F086FF054628B99E
:1035900021461048BDE8F840FDF7DABC0B4B9C61B2
:1035A0000AF0ECFA2A4621460B48FDF7D1FC172C0D
:1035B00009D80A4B0C2202FB043393F8D806BDE865
:1035C000F8400AF017BB0020F9E700BF780301209C
:1035D000A4930608B8930608CE930608849E0508AF
:1035E00038B50446114D0846FFF742FB68B1104B51
:1035F00093F900104B1C06D10E4B19780E48BDE80C
:103600003840FDF7A5BCC9B2F8E70846FCF72AF92F
:10361000032804D8C0B2FDF771F82946E3E7204635
:1036200003220649BDE83840FEF714BA10A906087F
:1036300078030120CC500120E7930608F793060891
:1036400038B50446114D0846FFF712FB68B1104B20
:1036500093F901104B1C06D10E4B59780E48BDE86A
:103660003840FDF775BCC9B2F8E70846FCF7FAF830
:10367000032804D8C0B20EF0FBFB2946E3E720463E
:1036800003220649BDE83840FEF7E4B910A9060850
:1036900078030120CC500120E3930608F29306083A
:1036A000444B2DE9F74FDFF8249105461A78009135
:1036B00089F800205A7893F8303089F801200BB946
:1036C00005F060FB00263C4C37F06AFBB0460D234A
:1036D000394A0099734352F803A05046FCF720F88A
:1036E000002841D0B8F1000F01DDFDF783FB514602
:1036F0003248FDF7E3FB002221462846FEF79CF9FD
:10370000FDF778FB237903F01803082B45D0102B25
:1037100048D02046FDF72BFC0D22274B02FB063339
:10372000B3F8090037F002FB8346D8B12046FBF717
:103730005AF90746DBE90221024401442046FBF71F
:103740000BF978B9514601901D48FDF7B7FBDBF83E
:103750000810019A28461346CA192146FEF782F836
:10376000FDF748FB08F10108013640F271230D34E2
:103770009E42ACD10020FFF73EF9FF2389F80030CC
:1037800089F80130B8F1000F11D1009A28460D498F
:1037900003B0BDE8F04FFEF75DB90B492846FFF7CF
:1037A0001FFFB6E708492846FFF74AFFB1E703B015
:1037B000BDE8F08FCC50012020B7050882900608A4
:1037C00012940608258A060810A906087803012025
:1037D0002DE9F74F804608460F4643F0BBF90446F3
:1037E00020B1012824D13B782A2B21D1A94E0025D4
:1037F0004FF00D0AA84FB14604F00104A748FDF7A9
:1038000011FB0AFB05F33846013559F80310FDF7A3
:1038100055FB314622464046FEF70EF90D36FDF7C0
:10382000E9FA40F271239D42EBD103B0BDE8F08F7D
:103830003D21384644F0F1FE002800F02481034683
:103840009A4613F8012D202AFAD0AAEB070A013074
:10385000054610F8013B202BFAD05FFA8AFA4FF0A8
:103860000009DFF830B20D235246384603FB09F356
:103870005BF803100BEB03040091FBF72DFF0646EA
:1038800070BB0099084643F065F9824528D1277935
:1038900007F0E001402900F08A8012D871B3667900
:1038A0007F4A002702EBC606BA463B4696F87022CE
:1038B0000092009ABA4202D9BAF1000F63D02BB13C
:1038C0002DE06029ECD0802900F0A58040467549A4
:1038D000FEF7C0F8204603B0BDE8F04FFDF747BB48
:1038E00009F1010940F271239945BCD13A466E496C
:1038F000404603B0BDE8F04FFEF7ACB807F0070351
:10390000042B1CD10B460A222846FBF721FFD4F8D2
:10391000053001468342D9D32046FBF78FF90D23AA
:10392000624803FB09F95BF80910FDF7C7FA0022AA
:103930002146404603B0BDE8F04FFEF77DB8052BA9
:103940000DD101230A222846FBF702FFD4F80530E7
:1039500001468342BADB5B428342B7DCDCE72846A0
:10396000FBF780FF17F0050F014607D1B4F80520DB
:10397000B4F807309142A9DB9942EEE7B4F905208B
:10398000B4F90730F6E7D6F86C1251F8270060B1A9
:1039900029460193FAF704FF019B30B94FF0010A61
:1039A00039462046FBF74AF95346013781E707F0CD
:1039B00007076379013F0093009BB342AFDDAA463E
:1039C00015F8013B202BFAD02046FBF721F90546DC
:1039D000042F04D8DFE807F0030E0E141D00504634
:1039E000FBF740FFA8552C21504644F016FE013647
:1039F000451CE1E75046FBF735FF25F81600F2E7D6
:103A000000230A2200215046FBF7A2FE45F82600BB
:103A1000E9E70123F5E7284643F09CF8E3790646F9
:103A200094F805A0DB07A7790AD52046FBF7F0F844
:103A30000378014623B13246284644F00CFEE0B933
:103A4000DEB1B74219D32046FBF7E2F83A4600212F
:103A500044F0CCFDB2453FF662AF324614492846E9
:103A600044F0F9FD00283FF45AAF2046FBF7D0F8A8
:103A70003246294644F0C4FC51E73A460D494046D7
:103A8000FDF7E8FF22E73946404603B0BDE8F04FB6
:103A900006E600BF20B705088290060822940608B3
:103AA000849E050870940608258A06086594060811
:103AB000C7A20608359406082DE9F04F914687B055
:103AC0000C461A46002180464D46FEF787FF002728
:103AD0000646B9F1000F63D029460622204644F07D
:103AE0005BFD00283246404613BF012100214FF004
:103AF000010A4FF0000AFEF771FF064628780EF023
:103B0000C9F98346F8B168790EF0C4F94FF46171D0
:103B10004FF0190CAB78EA789BF805E01CFB031317
:103B20001CFB021295F801B0297900B14079CDE96A
:103B30000410CDE9023251463B461A4A4046CDE9CF
:103B400000EBFDF7A3F920780EF0A4F98346F8B155
:103B500060790EF09FF94FF461714FF0190CA37862
:103B6000E2789BF805E01CFB03131CFB021294F89F
:103B700001B0217900B14079CDE90410CDE90232DC
:103B800051463B46074A4046CDE900EBFDF736F982
:103B9000013706340635142F9BD107B0BDE8F08FEE
:103BA000CA46D0E77E9406082DE9F041054686B066
:103BB00008460F46FFF75CF8064638B100235B491C
:103BC00001201A4606B0BDE8F04175E70846FBF74C
:103BD00049FE1328044600F3A08006258DF81760DF
:103BE000534E4543781CFBF76CF8074660B1FBF772
:103BF00039FEC0B20EF022F930B17319027983F8A0
:103C0000482601238DF817303846FBF75AF8074647
:103C100068B1FBF727FE0D2809D8062303FB0463D0
:103C200083F849069DF8173001338DF81730DFF817
:103C3000FC80A91C0DF1170238464144FBF716FE23
:103C4000FBF73FF8074668B1FBF70CFE012809D8DF
:103C50009DF817300622013302FB04628DF81730FD
:103C600082F84C063846FBF72CF880B1FBF7FAFDDA
:103C7000C0B20EF0E3F850B19DF81730062201797A
:103C800002FB0462013382F84D168DF817309DF85F
:103C900017200623042A2FD103FB04630022A3F874
:103CA0004C26062518F04AFD05FB046595F84806E4
:103CB0000EF0F0F895F84B1695F84A7619234FF464
:103CC0006172804695F84D0613FB012613FB07270A
:103CD0000EF0E0F84379214698F80520039395F813
:103CE0004C3614480097CDE9016395F84936FDF745
:103CF0002FF906B0BDE8F081052A05D103FB046366
:103D0000002283F84D26CCE7062ACAD0002308EB10
:103D1000050248F805309380C3E71323324606496D
:103D2000284606B0BDE8F041FEF796BF14570120C3
:103D3000CC5001207E940608979406082DE9F04F98
:103D4000904689B01A460C46002181464546FEF74A
:103D500045FE3A4E08F154030746DFF8E4B00793F6
:103D600094F9040009F032FC00285CD0B8F1000F8F
:103D700061D029460C22204644F00EFC00283A4629
:103D8000484613BF012100214FF0010A4FF0000AFD
:103D9000FEF724FE074695F904003CF0F7FAEA79AD
:103DA0000346514606EB82024846D2F8D8240492D4
:103DB0002A7A06EB8202D2F8D8240392AA7906EB7B
:103DC0008202D2F8D82402926A7906EB8202D2F8F3
:103DD000D82401922A6800925A46FDF757F894F9C0
:103DE00004003CF0D3FAE2790346514606EB820226
:103DF0004846D2F8D8240492227A06EB8202D2F8FE
:103E0000D8240392A27906EB8202D2F8D824029237
:103E1000627906EB8202D2F8D824019222680092DD
:103E20005A46FCF7EBFF0C35079B0C34AB4297D19D
:103E300009B0BDE8F08FC246D1E700BF849E0508F7
:103E40009D9406082DE9F04780468CB00846FEF7A1
:103E50000FFF054638B10023594901201A460CB01E
:103E6000BDE8F0476AE7CDE909000B9007A8079184
:103E7000544944F08FFA06463CF07EF9431C044650
:103E80000CD12B460A2208A93046FBF761FC089B9F
:103E90001B781BB9C4B2132C0BD944B2204609F0CD
:103EA0003DFB054640B94046FEF73AFE0CB0BDE882
:103EB000F087333464B2F1E7424907A88DF828400F
:103EC00044F068FAB0B3002302260A221946FBF731
:103ED0003FFC09900027DFF8EC90DFF8F0A049469E
:103EE00007A844F057FAF8B1FBF7BCFC364A0023A8
:103EF00052F8041B88421FD1DBB20AEB8302D2F8CE
:103F0000D824904210D1022F20D0032F23D05A1E44
:103F1000012FD2B215D00B2A03D88DF829300136E3
:103F2000F6B20137042FDAD1052E1AD84046FDF734
:103F3000A7FDBBE70126CDE70133102BD8D1002325
:103F4000DBE7052AEDD88DF82A30E8E7092BE8D819
:103F50008DF82C30E3E79A1E0D2AE2D88DF82B302D
:103F6000DDE709AB03CB286018686960A8602046CC
:103F70003CF00CFA154A9DF82B10034602EB810128
:103F8000D1F8D81404919DF82C1002EB8101D1F8DE
:103F9000D81403919DF82A1002EB8101D1F8D814AE
:103FA00002919DF8291002EB81020021D2F8D82459
:103FB00008460192099A0092054AFCF71FFF75E72F
:103FC00018560120E6A306085CA30508849E050890
:103FD0009D9406082DE9F04F90468BB000264FF0D7
:103FE000190A45464FF461790C461A4600210746E6
:103FF000FEF7F4FC0990B8F1000F49D029460A22D7
:10400000204644F0C9FA0028099A384613BF012116
:1040100000214FF0010B4FF0000BFEF7DFFC2A8967
:104020000990334606925946EA88384605922A791D
:104030000492EA780392AA781AFB029202926A78B2
:104040001AFB029201922A780092124AFCF71EFF94
:10405000228933460136594606923846E2880A35A7
:10406000059222790492E2780392A2781AFB0292D6
:10407000029262781AFB0292019214F80A2B0092C3
:10408000044AFCF7BBFE1E2EB5D10BB0BDE8F08F85
:10409000C346DDE7BA9406082DE9F04380468BB0AD
:1040A00008460F46FEF7E4FD044638B100235E499A
:1040B00001201A460BB0BDE8F0438BE70846FBF73A
:1040C000D1FB1D28054600F3A5800A268DF8274060
:1040D0004643781CFAF7F5FD10B101238DF827301F
:1040E000FAF7EFFD514C074668B1FBF7BBFB0D2813
:1040F00009D80A2303FB054383F8F0029DF8273013
:1041000001338DF82730DFF82091711C0DF1270263
:1041100038464944FBF7AAFBFAF7D3FD074668B1D6
:10412000FBF7A0FB232809D89DF827300A2201338A
:1041300002FB05428DF8273082F8F3023846FAF781
:10414000C0FD074668B1FBF78DFB0D2809D89DF827
:1041500027300A22013302FB05428DF8273082F80E
:10416000F4029DF82730062B0CD0002309EB060241
:10417000404649F80630536013810BB0BDE8F04368
:10418000FDF77EBC0A260023384606FB0546A6F846
:10419000F632A6F8F832FAF794FD074618B1FBF7A5
:1041A00061FBA6F8F6023846FAF78BFD30B1FBF753
:1041B00059FB0A2303FB0543A3F8F8021C4B4FF0FD
:1041C000FF324FF461705A600A2303FB0542B2F8D4
:1041D000F8320693B2F8F632059392F8F43204936B
:1041E00092F8F3320393192392F8F21213FB0101B0
:1041F000029192F8F11213FB01030021019308468A
:1042000092F8F0320B4A00932B46FCF7F7FD0BB007
:10421000BDE8F0831D232246074940460BB0BDE8A8
:10422000F043FEF719BD00BFB4640120C461012052
:1042300078030120BA940608979406082DE9F04FF8
:10424000804691461E460C4615460027DFF81CA105
:104250002DED088B95B094ED008AB5EE408AF1EE15
:1042600010FA7BD0D4ED019A94ED029AD4ED038A32
:10427000B9F1000F49D0D5ED00BA95ED01BAB4EE11
:104280006B8AD5ED02AA95ED03AAF1EE10FA6AD178
:10429000F4EE4B9AF1EE10FA65D1B4EE6A9AF1EEB3
:1042A00010FA60D1F4EE4A8AF1EE10FA0CBF012147
:1042B000002132468B46404681F00101FEF78EFB1D
:1042C000B0EE6B0A064611A8FAF71EFCB0EE4B0AD8
:1042D00007900EA8FAF718FCB0EE6A0A06900BA831
:1042E000FAF712FCB0EE4A0A059008A8FAF70CFC9F
:1042F0000599069A079B0390404602915946019200
:10430000524600933B46FCF7C1FDB0EE480A11A8A7
:10431000FAF7FAFBB0EE690A83460EA8FAF7F4FB47
:10432000B0EE490A06900BA8FAF7EEFBB0EE680A69
:10433000059008A8FAF7E8FB069B059A0021039070
:1043400040460292524610341035CDE900B33B4648
:104350000137FCF753FD082F7FF47DAF15B0BDEC9E
:10436000088BBDE8F08F0021A3E700BFDD940608AD
:104370002DE9F14F06460C46DFF894B12046FEF7D2
:1043800077FC074638B100235A4901201A4601B08C
:10439000BDE8F04F52E7052257492046FBF79CF94C
:1043A00060B9544B00221A601A611A621A631A64C7
:1043B0001A651A661A6701B0BDE8F08F04225946E3
:1043C0002046FBF789F905462046002D45D1FAF72E
:1043D00078FC07460028EED042F0BCFBDFF834A1A1
:1043E0005FFA80F85AF8049BB9F1000F07D1224612
:1043F0004249304601B0BDE8F04FFDF72BBB4246C5
:10440000494638460135FBF767F984460028E9D16B
:10441000384A034600211746013342F8101B082B87
:10442000FAD1374B03EBC505D5F880E0BEF1000F9C
:1044300005D149463348344CFCF78AFD9EE795F890
:104440007C50AC45F5DA0EEB0C1307EB0C140CF1B9
:10445000010C0FCB84E80F00F3E7FBF703FA072802
:1044600005463DD82046FAF72CFC074658B3FAF724
:10447000BBF9204B012403EB051383ED000A3846FA
:10448000FAF71FFC074638B1FAF7AEF9194B0134B9
:1044900003EB051383ED010A3846FAF712FC0746D1
:1044A00038B1FAF7A1F9134B013403EB051383ED8F
:1044B000020A3846FAF705FC38B9304601B0BDE8C3
:1044C000F04FFDF7DDBA0446D9E7FAF78DF9094B4D
:1044D000032C03EB051383ED030A3FF454AFECE721
:1044E00007233A460949304601B0BDE8F04FFEF7D0
:1044F000B3BB00BFE065012069910608258A060864
:10450000849E0508F694060810A9060897940608E4
:10451000F1940608A4A405082DE9F74F92460C462D
:104520001A46002181465646FEF758FA0025804675
:10453000DFF864B0BAF1000F2CD0314604222046D7
:1045400044F02AF800284246484613BF01210021C2
:1045500001270027FEF742FA738880465A460193E6
:1045600039463AF82530484600932B46FCF78EFC36
:1045700063885A46394648460193043634F8043B6A
:1045800000932B460135FCF739FC042DD2D103B042
:10459000BDE8F08F5746EBE7009506082DE9F3419B
:1045A00005460846FEF764FB0C46074638B1002373
:1045B000334901201A4602B0BDE8F041ACE7314969
:1045C0002046FAF7EDF870B904222D4B4FF47A70BB
:1045D0004FF4FA61013A1880598003F10403F9D1CC
:1045E00002B0BDE8F0812046FBF73CF903280646FF
:1045F00041D82046FAF765FB074698B1FBF732F938
:104600004FF0010804463846FAF75BFB20B1FBF790
:1046100029F9B8F1000F09D1284602B0BDE8F041F0
:10462000FDF72EBA40F2EE248046ECE7A4F2EE222B
:1046300040F2DC539A4203D8A0F2EE229A420AD901
:1046400040F6CA0340F2EE220F49284602B0BDE808
:10465000F041FEF701BB0D4B00210D4A03EB860331
:10466000A3F89C44A3F89E043346CDE900400846D5
:10467000FCF7C4FBB4E703233A460649E5E700BF6D
:10468000606601206991060811950608C461012041
:1046900000950608199106082DE9F04F8FB089465C
:1046A000174600211A4606460024FEF797F90DF139
:1046B000240B0546DFF86CA059F82480594602A85F
:1046C000CDF808803BF012FE4FB357F824302A464D
:1046D00030469845039313BF012100214FF0010894
:1046E0004FF00008FEF77AF904A9054603A83BF04D
:1046F000FDFD04A923465246009130464146FCF791
:10470000C5FB23460134524641463046CDF800B041
:10471000FCF774FB202CCFD10FB0BDE8F08FB8466A
:10472000EFE700BF1F950608F0B5074689B00846B9
:104730000E46FEF79DFA054638B1002319490120BF
:104740001A4609B0BDE8F040A6E70846FBF78AF82C
:104750001F2804461DD83046FAF7B3FA0146204612
:104760002EF096FA78B103AE0E48314600EB840085
:104770003BF0BCFD23460C4A294628460096FCF730
:104780003DFB09B0F0BD384609B0BDE8F040FEF78A
:10479000C7B91F232A460549384609B0BDE8F0408D
:1047A000FEF75ABA706601201F950608979406080E
:1047B0002DE9F04F924685B00C461A4600218146FD
:1047C0005546FEF70BF900268046DFF86CB0BAF1CB
:1047D000000F2FD029460422204643F0DDFE00289A
:1047E0004246484613BF0121002101270027FEF75A
:1047F000F5F8EB7880465A4602933946AB7848463E
:1048000001932B8800933346FCF740FBE3785A462C
:104810003946484602930435A378019334F8043BA3
:10482000009333460136FCF7E9FA102ECFD105B0DC
:10483000BDE8F08F5746E9E729950608F0B5074629
:1048400085B008460E46FEF713FA054638B1002338
:104850001C4901201A4605B0BDE8F040A8E708460B
:10486000FBF700F80F28044623DC3046FAF729FA54
:10487000014620462EF0E6FAA8B104F12002124BC0
:104880002946284603EB820393F8AF24029293F85B
:10489000AE240192B3F8AC340C4A00932346FCF7E3
:1048A000ADFA05B0F0BD384605B0BDE8F040FEF702
:1048B00037B90F232A460649384605B0BDE8F0400F
:1048C000FEF7CAB9F0660120C461012029950608E7
:1048D000979406082DE9F04F85B014461A46054610
:1048E00002910021FEF77AF84FF0000806460623F1
:1048F0004FF0000903FB08F7C037029B13F807B01D
:10490000002C7AD0E35D324628469B45039313BFC3
:10491000012100214FF0010A4FF0000AFEF75EF876
:10492000039B0646374A51462846CDE90093434645
:10493000FCF7ACFA4346334A514628460137CDE9E5
:10494000009B09F10109FCF759FAB9F1060FD4D11E
:1049500008F10108B8F1060FC9D1E427029BA7F1BD
:10496000E40913F807A0002C49D014F807B0324628
:104970002846DA450DBF4FF001084FF0000801212D
:104980000021FEF72BF8062306461E4A414628461C
:10499000CDE9009BFCF77AFA01370623194A414614
:1049A0002846CDE9009AFCF729FAEF2FD6D1029BD1
:1049B00093F8EF70ACB194F8EF8032462846474543
:1049C00013BF0121002101240024FEF707F8002372
:1049D0000C4A2146009328460723CDF80480FCF7B3
:1049E00055FA0023074A21462846009307230197DA
:1049F000FCF704FA05B0BDE8F08FA2469AE7A0469E
:104A0000CAE700BF3B950608F0B5054685B00846E5
:104A10000B46FEF72DF9044638B100231B4901204F
:104A20001A4605B0BDE8F04054E701AE184F6A469B
:104A30001749184643F0DBFC88B1032C04D1284603
:104A4000FDF71EF805B0F0BDFAF70CFF6A4646F810
:104A5000040B39460020013443F0C9FCECE7032C79
:104A6000EDD1039FDDE901463A463146E0B22EF032
:104A700023FA18B92846FEF753F8E3E73B463246D7
:104A800021460448FCF764FADCE700BF70660120A9
:104A9000E6A306083B9506082DE9F04F0E4615469D
:104AA00089B01A4600210446B046FDF797FF2F460D
:104AB00081464FF0000B002D7AD039460C2240463B
:104AC00043F06AFD00284A46204613BF0121002119
:104AD0004FF0010A4FF0000AFDF780FF97F90B2015
:104AE00081465B460492514697F90A20204603927C
:104AF000B7F908200292B7F906200192B7F904200D
:104B00000092364AFCF7C2F998F90B205B460BF18C
:104B1000010B51460492204698F90A200C3708F1FF
:104B20000C08039238F9042C029238F9062C0192F1
:104B300038F9082C0092294AFCF760F9BBF1080FFC
:104B4000B9D14FF0000BDFF898800C2303FB0BF971
:104B500085B3002755F80900012356F8092003FA08
:104B600007FA42403AEA020214BF1946002110EA4D
:104B70000A0F07D05B464246204600970791FCF794
:104B800085F9079956F809201AEA020F05D05B4605
:104B9000424620460097FCF731F901370E2FD9D154
:104BA0000BF1010BBBF1080FCFD109B0BDE8F08FBD
:104BB000AA46A9E72F46012356F8091003FA07F27F
:104BC0000A4206D05B464246012120460097FCF788
:104BD00015F901370E2FEED1E2E700BF4F95060819
:104BE00067950608F0B506468BB008460D46FEF7F9
:104BF0003FF8044620B300233D4901201A460BB07C
:104C0000BDE8F04048E72D2903D0A1F13003092B7E
:104C100049D8052C05DD30460BB0BDE8F040FCF767
:104C20002FBF2846FAF71EFE0AAB621C03EB4404B2
:104C300024F80C0C15F8013F303B092BFAD9144627
:104C400029780029DFD1062CE5D1BDF81C20BDF95B
:104C50001C30072ADFD8BDF91E50A5F5FA7292B2B2
:104C6000B2F5FA6F18D8BDF92070A7F5FA7292B2B2
:104C7000B2F5FA6F10D8BDF922C065450CDC674566
:104C80000ADBBDF924E00EF1640292B2C82A03D80F
:104C9000BDF92640112C11DD164930460BB0BDE898
:104CA000F040FCF7D7BE202902D101352246C6E7E5
:104CB00030460BB0BDE8F040FDF732BF0C200E4A85
:104CC00064B200FB03220846A2F8A055A2F8A27520
:104CD000A2F8A4C582F8A6E582F8A745074A009580
:104CE000CDE903E4CDE9017CFCF788F80BB0F0BD19
:104CF000606701207C950608C46101204F95060875
:104D00002DE9F04F89468DB0164600211A46074618
:104D10000024FDF763FEDFF8DCA00546C4EBC40306
:104D200009EB030259F80300918840F30748927990
:104D30000890ADF824108DF82620B8F1000F53D05C
:104D4000002E54D0F218F0589188937907220A90D7
:104D500008A8ADF82C100AA98DF82E3043F01CFCE1
:104D600000282A46384613BF012100214FF0010BCD
:104D70004FF0000BFDF732FE9DF82E3005465246EF
:104D8000069359469DF92D30384605939DF92C30F0
:104D900004939DF82B3003939DF92A3002939DF8DC
:104DA000293001939DF8283000932346FCF76EF8D4
:104DB0009DF8263052465946384606939DF92530CF
:104DC00005939DF9243004939DF82330CDE90283A7
:104DD0009DF8213001939DF8203000932346013443
:104DE000FCF70CF8102C99D10DB0BDE8F08FB3464C
:104DF000DEE700BF929506082DE9F04F06468BB01E
:104E00000D46DFF8A082284641F0A4FE034630B9E3
:104E10000246964901200BB0BDE8F04F70E705222D
:104E200093492846FAF758FC0446C8B9914D014603
:104E3000702205F2FC5043F0D9FBC5F89C45C5F83B
:104E4000A845C5F8B445C5F8C045C5F8CC45C5F872
:104E5000D845C5F8E445C5F8F0450BB0BDE8F08F7E
:104E6000042241462846FAF737FC044630BB284660
:104E7000F9F727FF81460028EFD041F06BFEDFF8FD
:104E800028B282465BF8047B3FB92A467A4930460D
:104E90000BB0BDE8F04FFCF7DDBD52463946484641
:104EA000FAF71AFC40B92046744D1EF097FC3946BB
:104EB0007348FCF74DF8A6E70134E3E70722714990
:104EC0002846FAF709FC074600287AD1202128460F
:104ED00043F0A3FB044670BB6B4D6C48FBF7EEFF41
:104EE000214601342846FBF7E9FF0E2CF8D10025B6
:104EF000DFF8B891664FFBF77DFFDFF8B4810C2631
:104F00000024DFF8B0A129466E434846FBF7D6FFE0
:104F10000123F2595F48A340013413420CBF4146BC
:104F20005146FBF7CBFF0E2CF2D10135FBF762FFA8
:104F3000082DE4D191E702AC574D01AA564943F040
:104F400056FA002848D0022F11D1029A072A07D812
:104F5000039C0D2C04D80378722B13D06E2B25D014
:104F6000082300224D493046FDF776FE75E7FAF733
:104F700079FC01AA44F8040B29460020013743F0CC
:104F800036FADEE70C233B4903FB02110123D1F87B
:104F90009C15A3400B4337490C2000FB02123949F2
:104FA000C2F89C353046FFF727FF56E7314B0C20FF
:104FB000012100FB0233A140D3F89C3523EA010311
:104FC000E9E72846002402AD334F01AA324943F0F5
:104FD0000EFA80B1082C03D13046FCF751FD3CE7B6
:104FE000FAF740FC01AA45F8040B394600200134C9
:104FF00043F0FDF9EDE7082CEED1029B0F2B30D8E2
:10500000DDF80CE0BEF1070F2BD8DDF810C0BCF1C5
:105010000D0F26D8059F07F16402C82A21D8069DE6
:10502000FF2D1ED8079864281BD80899642918D822
:10503000884216DA099C032C13D8C3EBC3020D4B2C
:10504000134483F8011683F8FCE50C4983F8FDC589
:1050500083F8FE7583F8FF5583F8000683F802464F
:10506000A0E70F493046FCF7F5FCF6E6C0670120E3
:1050700069910608C4610120258A060810A906085E
:10508000F6940608AF950608B7950608F99B06083A
:1050900060670120BC950608E6A30608C2950608CD
:1050A0007C950608F1940608A4A405082D8306083B
:1050B0007C9906087A9506082DE9F04F924600265D
:1050C00089B04FF019095546B3464FF461780C4644
:1050D0001A4600210746FDF781FC0790BAF1000F40
:1050E00027D029460622204643F056FA0028079A80
:1050F000384613BF012100214FF0010B4FF0000B88
:10510000FDF76CFC6A790790334619FB0282594619
:10511000384605922A7919FB02820492EA780392B2
:10512000AA7802926A7801922A780092104AFBF7D4
:10513000ADFE627933460136594619FB0282384684
:1051400006350592227919FB02820492E2780392D5
:10515000A27802926278019214F8062B0092044A17
:10516000FBF74CFE0A2EB9D109B0BDE8F08F00BFA5
:10517000C89506082DE9F04F074689B008468B46CA
:10518000FDF776FD044638B10023544901201A4644
:1051900009B0BDE8F04F8FE7514B084693F86CA774
:1051A00093F86D9793F85688FAF75CFB0928054643
:1051B00000F38B8006268DF81F404A4C46430BF1C6
:1051C0000100F9F77EFD834648B1FAF74BFB0D2845
:1051D00005D8A31983F86C0601238DF81F305846B3
:1051E000F9F76FFD834668B1FAF73CFB504509D8E3
:1051F000062303FB054383F86D069DF81F3001333A
:105200008DF81F305846F9F75CFD824668B1FAF711
:1052100029FB484509D8062303FB054383F86E069E
:105220009DF81F3001338DF81F305046F9F749FDC6
:10523000814668B1FAF716FB804509D3062303FBC4
:10524000054383F86F069DF81F3001338DF81F303A
:10525000DFF88880311D0DF11F0248464144FAF7FE
:1052600005FB9DF81F30062B0BD0002308EB060230
:10527000384648F80630938009B0BDE8F04FFCF797
:10528000FFBB03FB05424FF46170192392F87116BE
:1052900013FB0101059192F8701613FB0103002125
:1052A0000493084692F86F36039392F86E36029391
:1052B00092F86D36019392F86C360B4A00932B46A8
:1052C000FBF79CFD09B0BDE8F08F09232246074992
:1052D000384609B0BDE8F04FFDF7BEBC306801208C
:1052E000CC500120C4610120C89506089794060897
:1052F0002DE9F04F14468BB00F461A4600210646A2
:10530000FDF76CFB0546002C00F0D78022783B7837
:105310009A42024630460DBF4FF001084FF0000898
:1053200001210021FDF75AFB237805469B4A41469F
:105330003046FBF7ABFD3B784146984A3046FBF7D9
:105340005DFD002C00F0BB80627830467B789A428D
:105350002A460DBF4FF001084FF00008012100213F
:10536000FDF73CFB637805468D4A41463046FBF726
:105370008DFD7B7841468A4A3046FBF73FFD07F1B9
:10538000C90307F1020A04F1CA0B0593A31C4FF0ED
:1053900000090693822307933B784B4500F39180E5
:1053A000002C00F0F58097F8EA30304694F8EA20B7
:1053B0009A422A460DBF4FF001084FF00008012124
:1053C0000021FDF70BFB94F8EA300546754A41468B
:1053D0003046FBF75BFD97F8EA304146714A3046AC
:1053E000FBF70CFD002C00F0D58004F1EA0307F177
:1053F000EA0204F1FA014FF0010833F802CF32F863
:10540000020F844518BF4FF000089942F5D188F08B
:1054100001012A463046C9B2FDF7E0FA08210546E7
:1054200004F1EC00FAF7CAF85F4A034641463046F9
:10543000FBF72CFD97F8EA1007F1EC00FAF7BEF83D
:10544000594A034641463046FBF7D8FC002C00F091
:10545000A3804FF0FC094FF0010807EB090104EBB2
:105460000900F9F79DF909F10409002818BF4FF068
:105470000008B9F58E7FF0D188F001012A46304648
:10548000C9B2FDF7ABFA082104F1FC00F9F72BFCD7
:10549000464A034641463046FBF7F8FC97F8EA10C7
:1054A00007F1FC00F9F71FFC404A0346414630462D
:1054B0000BB0BDE8F04FFBF7A1BCA0463BE7A04610
:1054C00057E7079BFB180993002C5FD0079B0998AF
:1054D000E31819460893F9F763F9059B5A789BF886
:1054E00000309A424FD1B0FA80F84FEA5818069A25
:1054F000AAF102030AF10E01023A33F802CF32F8A0
:10550000020F844518BF4FF000088B42F5D188F098
:1055100001012A463046C9B2FDF760FA6278069961
:1055200005469BF81800FAF71BF802909BF800302C
:1055300041461F4A30460193089B009309F101033D
:10554000FBF7A4FC059B51467A7809F10109587EC6
:105550000AF1100AFAF704F8059A0290414612F887
:10556000013F30460BF1010B0193099B059200931B
:105570004B460F4AFBF742FC069B10330693079BF2
:105580000933079308E74FF00008B0E7A046D9E7D2
:10559000A04620E7A0464DE7A0467FE7E195060834
:1055A000F3950608219606083996060850960608CF
:1055B000089606082DE9F04F8FB004460846B24918
:1055C00002AA42F014FF054640B903460246AF491D
:1055D0004120FFF78DFE0FB0BDE8F08FAC49F9F721
:1055E000DFF8064628BB02AAA74942F000FFFAF7F7
:1055F00039F90828054606D908233246A549204628
:10560000FDF72AFBE7E7A44C94F86C3783420CDCE7
:1056100084F86C57DFE731460136384626F08CFBBC
:1056200094F86C37B342F6DCF2E7064604F26C7786
:10563000F6E79A492846F9F7B3F80646E0B902AA10
:10564000914942F0D4FEFAF70DF90828054603D92E
:10565000082332469249D2E78F4C94F86D37834243
:1056600002DC84F86D57B6E73046013629463AF039
:105670001FFD082EF8D1F4E78A492846F9F790F87B
:10568000064600BB02AA804942F0B1FE0028A2D023
:10569000FAF7E8F80828054603D908233246824974
:1056A000ADE77D4C94F85638834209DD014604F29B
:1056B0006C7026F087FB294604F26C7026F090FB94
:1056C00084F8565887E779492846F9F769F8064675
:1056D00018BB06AD704BDFF8B0910146A84610220A
:1056E000284693F8567842F081FFBE4202AA80F223
:1056F0000A814946002042F07AFE10B93A466C49C8
:105700000AE1FAF7AFF8013628F8020BEDE7694C29
:1057100095E80F0084E80F005DE767492846F9F730
:105720003FF80646C0BB5C4B06ADDFF85C9193F8D2
:105730005678BE4202AA80F2F3804946002042F029
:1057400056FE014610B93A465C49E5E0AA464FF0DC
:1057500000080322284642F090FF284641F0FAF95B
:10576000404502D801360435E3E79AF8000008F115
:105770000108F9F7ABFF0AF8010BEEE7B6000446A3
:105780004F4DB4423FF427AF06AB28190322191935
:10579000043426F0BBFAF4E74A492846F9F700F842
:1057A0000746002840F0AC80DFF8EC8002AA3649BA
:1057B00098F86C6742F01BFE00283FF40CAFFAF734
:1057C00051F8451E01D4AE4203DC334601223E4966
:1057D00015E72D4902AA002042F009FE01460028E3
:1057E0003FF4F9AE00260DF10C09082203A88DF84C
:1057F000146042F042FF03A841F0ACF9B0421BD85C
:1058000002AA2149002042F0F2FD00283FF4E3AE55
:105810000026037898F86DA7B1460193564502AA71
:1058200019494FF0000080F2858042F0E0FD834688
:1058300050B9524625496FE099F800000136F9F752
:1058400045FF09F8010BD6E7A6B99BF80030303BBD
:10585000092B0FD91E49F8F7A3FF38B11D49584647
:10586000F8F79EFF70B15A461B4955E04FF0010909
:105870004FF0FF365846F9F7F5FF002830DA5A4660
:10588000164949E0B146F3E7E6A306083858012077
:10589000679606086D960608CC5001207896060893
:1058A000819606088F9606089B960608AD96060810
:1058B0009C97060824590120D7960608BC9706082D
:1058C000345901200197060806970608DC97060858
:1058D0007782060812970608199706084E97060859
:1058E0000EAB03EB4603013623F8200C96E7524635
:1058F0001F4911E033F8022B013724F8022F30E062
:105900002A461C4908E01C49002042F070FD00288E
:105910003FF4FDAE3A4619492046FCF79BF85AE69B
:105920001549002042F063FD00283FF427AF3A46B6
:105930001349F1E742F05BFD0028D8D105EBC50023
:10594000104C082203A98230204404EB051426F0F1
:10595000DDF90198F9F7BAFE08EB050383F836087C
:1059600006ABBE42C6DC454485F84E9833E600BF20
:105970006397060886970608E6A30608B996060800
:10598000E3960608385801202DE9F04F0F4690465F
:1059900089B0002187EA08080646139A0025039378
:1059A000FDF71CF8DFF884906FEA080304460693BD
:1059B000284607F05FFD129B184230D0069BDFF8A7
:1059C00070B0034014BF4FF0010A4FF0000A049377
:1059D00010EA070328460CBF4A465A460593079229
:1059E00007F05AFD039B8046079A514600903046C7
:1059F000FBF74CFA049B22463046B3FA83F149097F
:105A0000FCF7ECFF059A0446039B002A0CBF5A469C
:105A10004A4651463046CDF80080FBF7EFF9013594
:105A2000172DC5D109B0BDE8F08F00BF0198060859
:105A3000EB94060870B504460E46084641F08AF815
:105A40003146054602462046F9F746FE68B9635DD1
:105A50001846F9F725FE00B933B901352C44204624
:105A600001340378202BFAD070BD0020FCE708B584
:105A700004460948FBF7B6F9FBF798F9074BD3F84A
:105A8000600207F0F3FD04F07BFA012C01D13CF039
:105A90008DFCF6F7B7F900BF08980608C46101202D
:105AA00010B5044608460B46FDF7E2F828B9032274
:105AB00008491846F9F710FE28B90748FBF7B8F966
:105AC0000120FFF7D4FF20460449BDE81040FBF752
:105AD000C1BF00BF14980608189806085090060821
:105AE0002DE9F74F4FF0000B064601AA08462E4954
:105AF0005D4642F07CFC01270446DFF8BC80DFF8FD
:105B0000BC90DFF8A4A01CBBBBF1000F28D1274C30
:105B1000002D44D029462648FBF71AFA94F8303075
:105B20000BB903F02FF935F03BF9002384F8593015
:105B3000FBF712F915B12846FCF75DFF9FB130461F
:105B4000FCF710FF78B1FAF75FFF0020FFF78FFF37
:105B5000BBF1000F0AD02046F9F784FE85B2C5B923
:105B60003046FCF7DDFF03B0BDE8F08F414620462C
:105B7000F9F7D6FD80B949462046F9F7D1FD00284E
:105B8000EED05F4601AA5146002042F030FC0446A8
:105B9000B9E74FF0000BF5E74FF0010BF2E70548CE
:105BA000FBF746F9BFE700BFE6A30608CC5001208B
:105BB00043980608669806083A980608D99C06088D
:105BC00010B50C46FCF7CEFE78B1084B01229A7353
:105BD000FAF71AFF0648FBF72BF906492046F8F7B3
:105BE000DFFD10B10020FFF742FF10BDCC500120B7
:105BF0007C980608978206080329F0B5054685B00B
:105C00000C46164614D80B4F3970FBF7F3F80A49C7
:105C10002846FDF7E5FC2246084901A8F9F78AFC69
:105C200001AB324608212846FCF708FFFF233B70F2
:105C300005B0F0BD7803012010A90608E793060817
:105C40000329F0B5054685B00C46164614D80B4F0F
:105C50007970FBF7CFF80A492846FDF7F1FC224698
:105C600008496846F9F766FC6B463246102128461B
:105C7000FCF7E4FEFF237B7005B0F0BD7803012044
:105C800010A90608E393060810B5114B86B0114918
:105C900004460493104B11480393114B114A02938D
:105CA000114B0193114B0093114BFBF707F9FBF7D5
:105CB000A1F810491048FBF74BF93CB10F4A1049C5
:105CC000104806B0BDE81040FBF742B906B010BD61
:105CD000C39806088D980608C8980608989806087C
:105CE000D298060883980608DB980608E798060805
:105CF000D3500120F7980608FF980608F788060891
:105D00004A890608109906080120BDE72DE9F04FE1
:105D10003B4C89B00A4600210546FCF75FFE059022
:105D200094F9000004F0D6F98146608834F0FEFF53
:105D3000344BD0F808B093F8307017B15F46D0F804
:105D40000CB0A3790026012B38BF012306932279DA
:105D5000637906FB02331BF80380002F3AD0FB5C0B
:105D60004345059A2846079313BF012100214FF0B0
:105D7000010A4FF0000AFCF731FE079B013605903F
:105D800053B303F00F021B095146284640330292D9
:105D90001D4ACDE900634B46FBF778F8B8F1000FD8
:105DA00024D008F00F034FEA1818174A51460293FF
:105DB00008F140032846CDE900634B46FBF71EF887
:105DC000069BB342C3DC0834104BA342A8D109B0F0
:105DD000BDE8F08F3B46C3E7002FDFD04B460C4AAF
:105DE000514628460096FBF751F8D7E76B06E7D4F3
:105DF0004B46074A514628460096FAF7FFFFDFE771
:105E00007CA60508CC5001203D9906088CA7050802
:105E10005399060838B50B4D0C4605EBC00595F9AE
:105E2000F80704F057F901460748FBF747F895F8DB
:105E3000FE3733B1611C0548C9B2BDE83840FBF7F5
:105E40003DB838BD849E0508F89B06082C830608DB
:105E500073B50E4610490546F8F7A2FC18B9307024
:105E6000012002B070BD2C78602C8CBF613C413C9D
:105E7000082C0FD8013501230A2201A92846F9F779
:105E800067FC019BAB4205D00F2803D8013440EAE0
:105E90000410E4E70020E4E71B9A060802460846DF
:105EA000531C05D1044B1A681B790A600B717047AB
:105EB0000249F9F73FBB00BF1B9A06082D8306086D
:105EC0000379062B0ED1C9B2C2680D2996BF064BC5
:105ED0000021595601238B40134214BF08464FF04E
:105EE000FF307047481C7047800F0608204BB0F504
:105EF000FA6F1A680346A8BF4FF4FA63B3F57A7FC6
:105F0000B8BF4FF47A73D2041DD540F2DC529042F0
:105F10001CD040F2DB5207EE903A9042F8EE677ADE
:105F200096BFDFED146ADFED146A9FED147A77EE09
:105F3000E67A92BF9FED120A9FED127A9FED120A48
:105F4000A7EE870A7047B0F57A7F02D89FED0F0A57
:105F5000704707EE903ADFED0E6A9FED0E7AF8EE8D
:105F6000677A9FED0D0A77EEE67AA7EE870A70470B
:105F7000C856012000007A4400A0BB44D62000C0CF
:105F800000E08244D620004000008344000000006E
:105F900000407A446610004000004042704700BF55
:105FA00000207047704700BF0020704701207047F5
:105FB000704700BF704700BF704700BF704700BF09
:105FC0009FED010A704700BF0000000000207047ED
:105FD000064B1B78834281BF00EB4000044B03EB70
:105FE000C003586998BF0020704700BFA407002075
:105FF000E006002000EB4000024B03EBC003587C9E
:10600000704700BFE0060020024B1878003818BF28
:1060100001207047A407002003681B6903B11847DB
:10602000704700BF0023084901E0152B09D003EB9E
:106030004302013311F802C00A448445F5D11046E9
:1060400070470020704700BFFC220120F0B1B1FA78
:1060500081F35B09D1B110B50D4C4FF0010E224612
:1060600002E001334E2B0FD092F804C01C3284455D
:10607000F7D10EF1010C71455FFA8CFEF1D1C3EB43
:10608000C30304EB830010BD002010BD0020704747
:106090008C9405082DE9F043070987B091461E4608
:1060A000DDF83880403700F00F0439B3FFF7CEFF3A
:1060B000C3790546164A49463046CDE900433B467A
:1060C000C047C0B12868F3F78DFFAA796B7912F049
:1060D000020F10494FEA93030F4A18BF0A46E979A5
:1060E00001330094CDE90321CDE901030B4A3B467E
:1060F00000213046C04707B0BDE8F0833B46084A60
:1061000049463046C4460E9407B0BDE8F0436047A8
:106110009A9906087F83060810A90608AC99060814
:10612000CE99060870B5094C236873B10546002660
:1061300006E099681A681E7321609047236823B1AE
:106140005A681846AA1A002AF3DA70BDBC7A0120F0
:106150002DE9FF47914604468A461E46FFF7B0FEEA
:10616000421CBDF830700546DDF834801FD0B9F10F
:10617000FF3F1FD0154A3146CDE900093846236854
:10618000C0474A465FFA8AF12079F3F78FFD02464D
:1061900000B10288D3B2314638460393C2F30323D9
:1061A000120B0293CDE90052094A2368C04704B09C
:1061B000BDE8F0877B06FAD40C9031462368384658
:1061C000044AC44604B0BDE8F0476047E0990608B9
:1061D000ED990608119A06082DE9F043154685B099
:1061E000894619466A1CBDF830600D9F25D04FEADC
:1061F000101800F00F04184A304608F14008CDE9A5
:1062000000454346B847A8B12A4699F80510D9F881
:106210000000F3F78DFD68B1038800210278304655
:106220000392C3F303221B0B02920C4ACDE90043F5
:106230004346B84705B0BDE8F0837306FAD40309B6
:1062400000F00F00064ABC460C904033304605B0C3
:10625000BDE8F043604700BF209A0608329A06085E
:106260005B9A06082DE9F04F714C8DB0DFF8CC91A8
:106270000A4604F1800A00218346FCF7AFFB039035
:106280000025A37A99F80060AB4200F390801034A7
:106290005445F5D140F216200DF1180A34F046FDB0
:1062A0000027002E4FF015024FF00001D0E9024503
:1062B000504604BF2546344642F098F92E78002E09
:1062C0003CD069783046FFF7C1FE95F90290049002
:1062D00009F1010253425341002C00F0A580002235
:1062E000A05CB04240F09C80224492F90280C145FB
:1062F00040F0948052788A4208BF0123012203F0C3
:1063000001030AF8072083F00101039A5846059318
:10631000FCF764FB059B039044B1464A3046049960
:10632000CDE900B24246FFF757FF059B424A30468F
:106330000499CDE900B24A46FFF74EFF0137033515
:10634000152FBBD184B3564604F13F07DFF8E48034
:10635000DFF8E49016F801ABBAF1000F21D12078F4
:10636000F8B194F9023001331BD06178FFF76EFE6B
:106370000546039A01215846FCF730FB94F90220A8
:106380005346294603902078CDE900B8FFF724FF53
:10639000207853464FF0FF322946CDE900B9FFF788
:1063A0001BFF0334BC42D5D10DB0BDE8F08FE088AF
:1063B00034F0BCFC002E627AD0E90231207A04BFAE
:1063C0001946334605FB00228F5623B39E56B7422B
:1063D000039A5846049313BF012100214FF001088E
:1063E0004FF00008FCF7FAFA049B039043B1114BFD
:1063F000324629462046CDE900B34346FFF7A8FEC2
:106400000D4B29463A4620460135CDE900B34346B7
:10641000FFF79EFE35E74FF0FF36D8E700236DE724
:1064200003323F2A7FF45CAF4FF0FF386BE700BFC9
:10643000280401208D0E0108FD0D0108FC500120EB
:106440002DE9F04F0C4607468BB040F2162034F091
:106450006DFC2246054600213846FCF7BFFA404B4A
:10646000064615221B78002104A8002BD5E9024519
:1064700004BF25461C4642F0B9F805F13F030393DB
:1064800095F80090B9F1000F30D095F801A0002CDC
:1064900063D0224600231178494557D1283392F81A
:1064A000018001226B4403F8182CD045324638464F
:1064B00013BF012100214FF0010B4FF0000BFCF73F
:1064C0008DFA064654B1B8F1000F07D0254B5A4655
:1064D0004146484600933B46FFF7DCFD224B5A46B7
:1064E0005146484600933B46FFF7D4FD0335039BD6
:1064F0009D42C5D13CB3651C0DF110084034DFF856
:106500006490DFF864A018F8013BCBB915F8013CA2
:10651000B3B116B13046FAF78BFC29783B4615F833
:10652000010C0022CDF800900026FFF7B3FD0022F9
:1065300015F8010C3B461146CDF800A0FFF7AAFD67
:106540000335A542DFD10BB0BDE8F08F0133033234
:10655000152BA0D14FF00008A7E7A046A5E700BF84
:10656000FC5001208D0E0108FD0D010810B5013110
:106570001446FFF76BFD28B9064B1A681B79226099
:10658000237110BDC27920460349BDE81040F8F7D9
:10659000D1BF00BF1B9A0608A799060808B5294B6A
:1065A0001B68DB041ED5B5EE400AF1EE10FA26D0CA
:1065B000DFED257AB4EEE70AF1EE10FA1FD49FED75
:1065C000237AB4EEC70AF1EE10FA2AD870EE677A91
:1065D0009FED1F7A9FED1F0AA7EE870A41F0A8FAE8
:1065E00080B208BDDFED187AB4EEE70AF1EE10FADA
:1065F0000BDA9FED190A41F09BFA80B208BD9FEDBE
:10660000170A41F095FA80B208BD70EE677A9FEDE7
:10661000147A9FED140AA7EE870A41F089FA80B236
:1066200008BDDFED117ADFED116A70EE677A9FED3C
:10663000107AA7EEA67AB0EE470A41F079FA80B256
:1066400008BD00BFC85601200000404200E082445F
:1066500066BEFFBE0060BB4400007A440080BB44BD
:1066600038DFFF3E00407A440000834466BEFF3EB0
:1066700000A0BB446B4B1B782DE9F04F87B0002B7B
:1066800000F0CA80684D4FF000086848A968FAF722
:106690005FFC69686648FAF75BFC664B6648D3E9BD
:1066A0000031C91A654B1A68B1FBF2F2FAF750FCD7
:1066B000FAF7A0FB6248FAF7B5FB6248FAF7B2FBBB
:1066C000614B5FFA88F41B78A34221D85F4D002408
:1066D0005F4EFAF78FFB013455F8041F3046FAF786
:1066E000EDFB162CF7D15B4D0124594EFAF782FBD6
:1066F0002B466968013430461B680435C91AFAF71D
:10670000DDFB162CF4D107B0BDE8F04FFAF772BBF1
:10671000514B14264FF03C0B671C03EB840306FB24
:10672000045693ED000A41F003FA96F81EA081B2D8
:10673000B6F80E901AF0010F80B20CBF2D22522233
:106740001AF0020F049045480CBF2D2354231AF071
:10675000040FB1FBFBF10CBF4FF02D0C4FF0560CAA
:106760001AF0080F05914FF064010CBF4FF02D0E89
:106770004FF0430E1AF0800F01FB09F10CBF4FF0F0
:106780002D0A4FF0530ACDE900CECDE902A13946DA
:10679000FAF794FBB37FDB073AD55C23304A6343B7
:1067A000D118D05891ED010A70B1B8EE400ADFED72
:1067B0002D7A20EE270A07EE900AF8EE677A80EE2F
:1067C000270A41F0B5F900B2642290FBF2F102FB16
:1067D00011022548FAF772FB1421244808F1010838
:1067E00001FB075701FB0454F988628A0491218B4D
:1067F00002F0030392080391E18A0291A18B0191B7
:10680000A18A009119214B43218AFAF7A1FB57E78E
:106810001748FAF7E7FADFE7164807B0BDE8F04F88
:10682000FAF700BBA8010020081D00206F9A060897
:106830007F9A0608101E0020969A0608B4280120A8
:10684000C39A06081F9B060898220020B01D00204E
:10685000CF9B0608B41D0020945300207B9B0608A4
:10686000281A002000401C46989B0608AD9B06088D
:10687000A49B0608D39B06082DE9F84F002607467F
:106880000C461D4DB046DFF87890DFF878A0204622
:10689000FCF7EEF9D5F800B048B921465846F8F7AC
:1068A0003FFF20B921466868F8F73AFF80B15846A3
:1068B000FAF798FA696811B15046FAF7FFFAA96831
:1068C00011B14846FAF7FAFA4FF00108FAF792FACE
:1068D000013610353B2EDAD12046FCF7C9F948B90C
:1068E000B8F1000F06D1224638460449BDE8F84FFA
:1068F000FBF7B0B8BDE8F88FE0D60508FB9B0608AB
:10690000F59B0608EF9B060870B5224C2378012BF7
:1069100000D070BD204B1B68002BFAD01F4D2B6898
:1069200028465B6898470028F3D01D4B1D4E1A6817
:10693000338892889A421BD31B4900222846096853
:106940004968EA622A6803FB01F1D368984740F07E
:106950004DF83388154A013352683380002AD8D065
:10696000116893884A69134218BF1B048B6170BD7C
:106970000E4A00210E4B52681B782170002AC8D0A5
:10698000C3F34003918812681B0101FA03F393617A
:1069900070BD00BFE22901202C1C0120301C012009
:1069A000DC290120E0290120D42901206C1C0120D0
:1069B000781C0120144B1B78222B144B04D0187A1E
:1069C00000F001003AF061BB114A596892F8742254
:1069D000013A18BF012289B1888810B40C68216976
:1069E0005DF8044B08420B490CBF10B201204A80ED
:1069F0000880187A00F001003AF047BB054910B250
:106A00004A800880DBE700BF05290120BC7A01200D
:106A1000F8290120082901202DE9F84FA24C07464A
:106A2000A24B2DED028B227A94F80980D2071E88A2
:106A30005BD59F4DB8F1010F94ED078A00F0888077
:106A4000B8F1020F49D0B8F1000F16D1238A9E4247
:106A500094ED078A974B00F2A8801A68EB7D216AB3
:106A600003EB8303521A03EB8303B2EB830FC0F2F1
:106A70009E804FF0010884F80980EB7B33B1AB892D
:106A800023B18D4B1B78002B40F08480A27A4245C5
:106A900038BF42462B7A632B07D8B8F1020F217D0D
:106AA00000F0C680002940F0D480844B9FED847AAA
:106AB0001A70A97BD4E90B3023631B1A06FB03F37E
:106AC00007EE903AF8EEE77AA7EE878A84ED078A18
:106AD00091BBBDEC028BBDE8F88FE389B342CCD209
:106AE0004FF0010884F809803CE0A8F10302012A74
:106AF0003CD918896E4DC0F30B0041F057FE0928B0
:106B000098DDB5F80690B14502D82B88B34291D2F2
:106B1000B6EB490F8EDC0323DFED6A7A664A6372B7
:106B2000B0EE678AA3720023C4ED077A1370A381C5
:106B3000E381238263822AE0012A00F09180022A05
:106B4000C7D10720BDEC028BBDE8F84F07F052B863
:106B5000638AB3422ED2A389B34203D24FF0000816
:106B600084F80980534B1B68236286E7504DB5F8C3
:106B70000690B14502D82A88B2422DD2B6EB490F11
:106B80002ADCB8F1030F40F0868094ED078A4FF0BD
:106B9000030872E70BF0A2FE002868D102234246E8
:106BA0009845A37238BF1A4674E71B68236294F8AD
:106BB000098062E73F4B216A1A682B7E521A03EB69
:106BC000830303EB8303B2EB830FFFF656AF4FF063
:106BD000020884F8098050E71889C0F30B0041F0DF
:106BE000E5FD09284DDD00226272A2722A7D002A8D
:106BF0006ED0314B1A70AB88698813FB02F311FB1E
:106C000002F2697C9BB292B28B42A381E2818ABF7D
:106C10005B1A00239BB28A428CBF521A0022238245
:106C200088BF92B26282642262750022A2610EE77E
:106C300079B90120A7612075C3F1640301FB03F357
:106C4000214981FB0301DB17A3EBA1536433637577
:106C50002BE7A1691D48791A8142EDDB637524E7B2
:106C6000BDEC028B0820BDE8F84F06F0C3BF2B7CBB
:106C700083420CD3012342469845A37238BF1A467B
:106C800008E7B8F1030F80D094ED078AF5E60023FA
:106C90004246A372FEE61889C0F30B0041F086FD60
:106CA00009283FF730AFEFE7BC7A012028630120C5
:106CB000CC560120641C0120386301203963012077
:106CC000ACC52737000000006BCA5F6B8096980048
:106CD0002888DFF8C890DFF8C880D9F80010B6FB24
:106CE000F0F0013091F976100828CABF0820C2B22E
:106CF0000246814288F800203FF47DAF00293FF42E
:106D00007AAF234991F800B00BF1010101F00301C2
:106D10008B453FF470AF4FF0FF3CDFF888A00BE0ED
:106D2000BCF1000F03DABEF1000F08BF8C46013141
:106D300001F003018B4518D04FF0EA0E0EFB01AEB7
:106D40009EF976E08645EBD18C465FFA8CF6114AC7
:106D50000121032E11700DD9701CC0B206F0FCFF8A
:106D60000D4B98F800201E8845E7BCF1000FFFF698
:106D700042AFEAE7EA22064B02FB06A01E70C9F802
:106D800000001CF0ABFB1AF0E5FE1AF0C7FFE3E7CA
:106D9000CC5001202024002028630120D855012058
:106DA00038630120005201202DE9F843C54B1B68D0
:106DB00013F004051ABFC44C0125C34C2DED048B00
:106DC00014BFD4ED3D8ADFEDC18A13F0200304D057
:106DD00094F8003113F002037CD1227A2E469FED05
:106DE000BC9A12F0010294F8401140F08980002909
:106DF0006BD1D4ED517A9FEDB76ADFEDB76A67EEDC
:106E0000867A94ED537A38EEC77AE8EEA67A84ED66
:106E1000527AC4ED517A63B1012194F85421D4F827
:106E200004318A4284F84111C4F8503118BFC4F8C3
:106E30004831AA4B1F780D2F0BD1D4ED417A9FED2D
:106E4000A87AA84B67EE877AFDEEE77A17EE902ACC
:106E50009A809FED9E0AA44841F06EFEB0EE408AF3
:106E6000A24B83ED000AD4ED577A9FEDA10A78EE8C
:106E7000677AA04884ED578A27EE800A41F05CFECD
:106E800084ED5B0A40F054FE02B282EAE273A3EBA7
:106E9000E2739BB2092B58D9002AACBF0A380A30DA
:106EA0000D2F05B2A4F8705154D0242F6AD0382F7A
:106EB00005D1B0EE480A40F03BFE8A4B988084F83A
:106EC0007261BDEC048BBDE8F88384F8412184F83D
:106ED00040218EE7D4ED447AB4F81431F8EEE77A25
:106EE000C4ED417A002B40F0A8809FED799A227A78
:106EF000012694F8401112F0010233463FF477AFB7
:106F0000002900F0928094ED538A744A78EEC89A72
:106F100094F841911778002B44D0B9F1010F02D0B9
:106F2000002D40F0A580B9F1000F40F0B7800D2F83
:106F3000DFF8B88100F0B780002D68D094F85431A4
:106F4000012B64D8B0EE690A63E000250D2FA4F888
:106F50007051AAD1DFED667A9FED670A69EE277A54
:106F6000604F28EE800AFDEEE77A17EE903A3B80FC
:106F700040F0DEFDFD80788084F87261BDEC048B0A
:106F8000BDE8F883DFED5C7A94ED520A20EE270A23
:106F900040F0CEFD534B84F872615880BDEC048BF9
:106FA000BDE8F8830D2F9FED499ADFF8408151D05D
:106FB000B9F1000FC0D094F8543133BB98ED000AFA
:106FC0003DB370EE687A94F85531DFED4C6A07EE08
:106FD000103A77EE887AB8EEC77AF0EEE77A67EE85
:106FE000877AF4EEE67AF1EE10FAC4BF69EE266A0B
:106FF00086EEA79AF7EE007A77EEC97A67EEA97A5D
:10700000E9EE007AB0EE670A03E0022B94D198ED26
:10701000000A3548F0EE698A41F08EFDB0EE408AF4
:1070200088ED000A84ED520A1DE794ED518A012291
:1070300084ED538A84F8402167E707EE903ADFED4C
:107040002C6A9FED2F7AF8EEE77A86EEA79A89FEF2
:10705000479A4CE7D8ED007A9FED270A27EE800A81
:1070600040F066FD1F4B9880B9F1000FA3D163E794
:10707000D4ED417A012337EEE87A84F8413137EED6
:10708000087A84ED547A77EEC77ADFF860800D2FA6
:10709000C8ED007A8FD194F84191DDE7D4ED417AC3
:1070A00094ED547AEFE7DFED147A98ED000A20EEC4
:1070B000270A40F03DFD0B4B9880002D7FF43EAF3A
:1070C000A5E700BF285B0120BC7A0120000000007A
:1070D0009A99993ECDCC4C3FCDCC4C3E0529012010
:1070E0000AD7233C08290120307C0120CC6C0120E8
:1070F0000000C8421C7C0120CDCCCC3D00401C4689
:107100006666663F2DE9F84FC14C2DED028BA368F2
:1071100020469847002800F0B880B4F90E3004F1FA
:107120004805A17D06EE903AB4F91030092907EE22
:10713000103AB4F91230F8EEE66A07EE903AB8EE7B
:10714000C77AF8EEE77AC4ED126A84ED137AC4EDDB
:10715000147A00F09E80DFF8E89228461EF034F89A
:10716000B9F82C30002B40F0A080AA4B1B685B07BD
:1071700000F1C780D9F828300026D4ED135AB3F9AE
:10718000022094ED127A06EE902AA34AD4ED147AE6
:10719000F8EEE66A92F800B0B3F90420B3F90030D3
:1071A00075EEE65A06EE902A06EE103ADFF8948263
:1071B000F8EEE66A994FB8EEC66A994AC4ED135ADA
:1071C00077EEE67A37EE467AC4ED147A84ED127AD9
:1071D000B4F84430B9F800A007EE903A92F8DA33E8
:1071E000B342B8EEE78A00F08F80BAF1000F40F0AA
:1071F000CE8095ED007AD7ED007A87ED007A77EEB4
:10720000677A67EE887AC5ED037A0136043508F1AE
:107210000C080437032EDBD194ED137ABBF1040F75
:10722000D4ED167A27EE077AD4ED124A67EEA77AE4
:1072300094ED155AD4ED145AA4EEA47A94ED176A7D
:10724000E5EE057AD4ED006AA5EEA57AE6EE067ABB
:10725000B1EEC70AB1EEE77A26EE800A84ED180A8D
:1072600026EE878A84ED198A0CD1DFED6E8A6E4D89
:1072700020EE280A40F05CFC28EE280AA88040F0A6
:1072800057FC2881012384F86830BDEC028BBDE8EF
:10729000F88FDFF8AC9104F1200128461DF02CFF97
:1072A000B9F82C30002B3FF460AFD9F828C029463C
:1072B000DFED5E6A00265E48ACF102020CF10407C5
:1072C000B3F5C87F16BFD0ED007AB0EE667AB8EE9F
:1072D000E77AD1ED007AE1EC016A77EE877AFDEE8C
:1072E000E77AE0EC017A22F8026F9742E8D1012BAD
:1072F00060D0013BA9F82C30464B1B685B077FF53B
:1073000039AF38F045FC35E7BBF1040F22D0BAF1B4
:10731000000F29D195ED000AD7ED007A87ED000A1C
:1073200070EE677A27EE888A85ED038ABBF1040F39
:107330007FF46BAF40F0FCFB9FED3E0ADFF8E8A066
:1073400028EE000AAAF8020040F0F2FB344AAAF83C
:1073500006005AE795ED000A40F0EAFB324B304A4E
:107360001880BAF1000FD5D095ED000A404641F0E3
:10737000E3FBD7ED007A2A4A70EE677A85ED000AC2
:1073800087ED000A27EE888A85ED038ACEE795ED22
:10739000000A404641F0D0FBD7ED007A204A70EE5B
:1073A000677A85ED000A87ED000A67EE887AC5EDF9
:1073B000037A2AE7204A214FD2F88801B4F80C80DA
:1073C000C830DFF884E087FB00BAC017D2E960124A
:1073D000C0EBEA10C831C832A0EB0800ACF80400DA
:1073E00087FB0180C917C1EBE011ACF8001087FBE7
:1073F0000217D217C2EBE712ACF80220CEF80A301F
:10740000AEF80E60F9F756FBB9F82C3071E700BF03
:1074100024240020C856012005290120487C012091
:107420009C1E002000007A44082901200000000072
:107430003C7C01200AD7233CBC7A01201F85EB51FC
:10744000F0230020F4230020F85601202DE9F04F0E
:10745000C44C2DED048B94F8983193B0022BCDE9F8
:10746000000329D112F0B0F90FF08CF9237AD90773
:1074700040F1E6800023BC4E1D4684F89831BB4B9A
:107480001B78002B00F0BE803378472B08D1019980
:10749000B74A04EB8103D3F8F0339B1122F8113083
:1074A00004EB8505D5F8F003801113B0BDEC048B17
:1074B000BDE8F04F41F018BB0123AE4A82F82030FE
:1074C000019B012B00F0928094F89931002B40F041
:1074D0003E8194F89A310493002BCBD00022A64B26
:1074E00084F89A211D78A54A1268002D40F05A812F
:1074F000009B934240F2218394F89B31002B00F0D3
:107500006585DFF898829FED9E8ADFF87C9208F10E
:1075100048079C4EDFF888A20FE05946D9F804309E
:1075200099489847032D47DD013594F89B2104368F
:10753000A8EC010A954280F20A83072DD9F804309D
:107540009148D4BF1AF805B05FFA85FB59469847B1
:10755000DAF82C30A7EC010A002BDED0D9F8043081
:10756000594689489847BAF81A2004EB4B03F0EEC5
:10757000406AB3F830329A4200F2E48207EE903A61
:10758000BAF81C30B8EE677A07EE903AF8EE677AF0
:1075900087FEC70A0123D4F8582203FA0BFB120511
:1075A000DAF82C300BEA030340F12281002BB9D129
:1075B000032DB6EEE60AB7DCB5EE400AF1EE10FA9E
:1075C000B2D0338807EE103A7388B8EE477A07EEE8
:1075D000903AF8EE677A30EE470A77EEC77A20EEF7
:1075E000080A80EE277A37EE080A9DE712F0C6FCFB
:1075F00002235D4E1D4684F898315C4B1B78002BAE
:107600007FF442AFF5F706FB009BC3F10107074487
:1076100041F09EFA019A04EB82039200D3F8F03312
:107620002244B0EBA31F1CBF830198118742CBBF3C
:10763000BF0103F1FF33C2F8F073C2F8F03323E760
:10764000524A0FA9524E02F1080512F8010F0131FA
:1076500004EB8003D3ED987AFDEEE77A17EE903ACB
:10766000B3F5FA6FA8BF4FF4FA63B3F57A7FB8BFEA
:107670004FF47A730128A3F57A73C3EBC3134FEA6F
:107680004303A6FB03734FEA9313A3F17F0308BFE1
:107690005B42AA4201F8013CD7D100263D480127B0
:1076A000354632468DF8446010F8013F07FA02F182
:1076B000013204EB83032943D3ED987AFDEEE77A98
:1076C00017EE903AB3F5FA6FA8BF4FF4FA63B3F52B
:1076D0007A7FB8BF4FF47A73A3F57A73C3EBC31301
:1076E0005B00B3F5FA3FA4BF4DB20126082ADBD1F7
:1076F0000EB18DF84450284B93F87422D3F89812A9
:10770000032A7FF4B7AE00293FF4B4AE0A7B002A07
:107710007FF4B0AE01200873D3F8A832C3F8A820D4
:107720000FAA03F19001C3F89C200922C3F8A420FA
:1077300040F20312A3F890201A698242D2B204BF29
:107740000FA8C3F8A00018683CF016F992E6DFF81D
:107750003890D9F80C3048469847002384F899317E
:10776000B7E600BFBC7A01200529012020240020B3
:1077700008290120945300207859012074590120D0
:1077800000007A4460660120585901208FDA05080C
:10779000D34D621097DA0508F82901205C7C01209E
:1077A000E45501200098C04E904294F89C1137781F
:1077B00001D9013D1D70D4F85403F9B1BB4A009BB7
:1077C0009569002D08BF1D46002840F0BE829FED40
:1077D000B80A4FF4487203463E2FC4F85453A4F835
:1077E000582384EDD70A00F0B483B24B18702AE016
:1077F00094F85C22002A7FF4D9AED9E6002800F084
:107800009D82009B9FEDAC7A1B1A4FF6DC7098426C
:10781000A8BF1846B0F5487FB8BF4FF4487007EED0
:10782000900A82B2181AF8EEE77AB0FA80F087EE82
:10783000270A40099F4D3E2FA4F8582384EDD70A0C
:10784000287000F06583272F03D140F071F99B4B1E
:107850001880DFF89C92D9F80030DD0400F16582D1
:1078600094F86333022B00F02283042B00F013837F
:10787000012B1AD1D4F86833009AD31A002B14DBE9
:1078800044F620631344C4F8683394F8973353B133
:1078900094F89533052B00F2AD83894A02EB43033C
:1078A0009B8CC3F38D03A4F86633D4F8B823009BF4
:1078B00084499B1A8B4239DC0099914239D007EEFA
:1078C000903A814B9FED816AF7EE006AF8EE677A95
:1078D00093F828309FED7E7A9FED7E5A67EE867A88
:1078E00006EE103AB4F86423B8EEC66AB4F866330C
:1078F00077EEE65A9A4237EE467A27EE057AE7EEB9
:10790000256A27EE277A87EE268A40F0A182724DFB
:10791000B5F98030B5F982209A4240F08982B5F9F4
:107920008430B5F986209A4240F05082009BC4F81A
:10793000B8336A4B009A9A4200F2EF8112F0E6FAED
:1079400007460FF011FC237A94F8D48313F0010357
:10795000357800F0D58000285B4BB8BF40425B7E95
:107960005FFA80FB5B459CBF012384F8D533B8F1F7
:10797000010F94F8D63302D0002B40F0228294F805
:10798000D7A3003F18BF0127BAF1000F40F0B5821E
:10799000B8F1010F14BF384647F00100002800F08D
:1079A0006782474A82F8380082F879A24C4A5178B7
:1079B000002900F09F8094F8D813002940F09A80A5
:1079C00094F8D913002940F0958094F8DA1300292F
:1079D00040F090804349029308781AF087FA029B9E
:1079E0003F4A002840F08680D9F80010C90600F10F
:1079F000038311794B004B2BA8BF4B238B45DBB284
:107A000080F01B839B45C0F0FD82374BDFED377A5A
:107A100093ED0B7AB0EEC77AB4EEE77AF1EE10FA96
:107A200040F1F08293ED057AB0EEC77AB4EEE77AD2
:107A3000F1EE10FA40F1E68293ED117AB0EEC77ADA
:107A4000B4EEE77AF1EE10FA40F1DC82D4F8E833D4
:107A500013B9009BC4F8E8335288BBF14A0F009871
:107A600088BF5208D4E9FA135B1A03444FF47A70C2
:107A700000FB02F2934202D9012284F8D8230029A4
:107A800000F0CD821F2D07D14FF47A72B3FBF2F3D1
:107A90000A4AD38001239380B8F1010F00F06E826F
:107AA00001231D46E9E400BF0529012058590120A2
:107AB00000409C44246301200024744908290120CB
:107AC0009453002090D00300E4550120BD37863642
:107AD000000080430000803B28040120404B4C0004
:107AE000CC550120D4680120A85700200000C842CE
:107AF000C85601201F2DCFD1BC4B00225A60CBE7C6
:107B00000122BB48BB4980F879220A6884F8D53342
:107B100092F8362084F8D733003A18BF01221F2D7F
:107B200080F8382001D1B14A5360B8F1020F00F05B
:107B30001982002384F8D433B2E7AF4E94F89C1135
:107B4000377838E607EE902AB8EE670A22E5D4F8CF
:107B5000543294F89C1113F48073DFF8D0E201F0F2
:107B6000010894F85EC218BF4FF00008DEF800B0BC
:107B7000039384F85D82002A00F03A8299F800307D
:107B8000BAF81250013B9D4F09EE105ABAF81A503C
:107B9000DBB2DFED9B8A0295B8EE499A079307F1B5
:107BA0004809984B07F19006BAF81C50A3FB0C301B
:107BB0009FED958A0695002500F0FE03CDF824B0D0
:107BC00003EB5003ACEB0303D8B20BF59673DDF86F
:107BD0001CB005908D48CDF81CC090F803A0CDE9ED
:107BE0000A3153469246CDE90CE0894A02EB850002
:107BF000D0ED007AB8F1000F14D0BCEEE77A17EEA2
:107C0000102A90B2029A90420CD3069A904209D858
:107C10000A9AC9F80020002B00F0B080032D45DC43
:107C2000984607E09BB3032D40DC032D00F06981EB
:107C3000F0EE497ABBF1010FC7FEE87AC7FE887AF9
:107C400044D9013509F104090636E7EC017A5545B6
:107C5000CBD10B99DDF81CC0DDE90CE0DEF800208B
:107C6000B8F1000F00F08F800369C260002B00F0B4
:107C70009981D21A036A934280F29280654A012365
:107C800080F82530136823F00403136088E0039A1A
:107C900062B9D9F80000099A101A0028C0F22A81A6
:107CA000032DDCBF4FF0000884F85D82E8B2089332
:107CB0001DF0D8F807EE900ABBF1010F089BF8EE13
:107CC000677AC7FEE87AC7FE887ABAD8FCEEE77A08
:107CD00094F8382317EE901A88B2059926F8110007
:107CE0002AB9079A022A13D9012084F83803708828
:107CF000B6F800C0484A8444B08884440FFA8CFC2B
:107D000022F815C0454A82FB0CE0A0EBEC7080B273
:107D100007EE900AF8EE677A93E73C4B9A78002AD0
:107D20007FF40CAE01229A7008E6D4F85432D807DA
:107D30003FF596AD04200AF0B5FE91E59FED380AB7
:107D400008464FF448720B4674E52B1A4FF6DC7068
:107D50009FED347A9842A8BF1846B0F5487FB8BF67
:107D60004FF4487007EE900A82B2181AF8EEE77ADC
:107D7000B0FA80F087EE270A40092DE5039A002A21
:107D80003FF458AF92E7234DC3680261D21A2B68C3
:107D900043F004032B6043689A42C8BF80F82580F3
:107DA000154E3778282F07D1D4ED9B7A0F4DFDEE75
:107DB000E77A17EE903AEB800CF1010384F85E321B
:107DC000F9E494F8D5A384F8D7A3DAE507EE903A5E
:107DD000154884EDF48AB8EEE70A40F0B1FEBDEE36
:107DE000C00A10EE103AA5F886309FE50829012058
:107DF00094530020D8550120052901201C7D012025
:107E000000A00C45ABAAAAAA00803B447C590120E3
:107E10005C7C0120C8590120F87D0120565555553C
:107E200000409C4400247449887E0120641C012089
:107E300007EE903A8E4884EDF28AB8EEE70A40F0F9
:107E40007FFEBDEEC00A10EE103AA5F8823066E55E
:107E500007EE903A874884EDF08AB8EE670A40F062
:107E60006FFEBCEEC00A10EE103AA4F864334EE583
:107E7000814A029310781AF039F8029B00287FF4A7
:107E800090AD7E4ADDF810A0126892F836000038F6
:107E900018BF012085E5F4F7BDFED4F8B433C01A4D
:107EA000774B9842C4BF0023A4F86433FDE4754BBC
:107EB000754ADB7B04EB8303D3ED977AFDEEE77A1B
:107EC00017EE903A1BB2B3F5FA6FA8BF4FF4FA63FE
:107ED000B3F57A7FB8BF4FF47A73A3F57A73C3EB27
:107EE0008323A2FB0323C3F38F13A4F86433A4F802
:107EF0006633DAE4D7ED007A9CE650464FF0000A8C
:107F00004FE56248028807EE902AF8EE677A91E61C
:107F10005F4DA8805F48029180FB0370DB17C3EBC5
:107F2000A0035D48A0FB0202D208EA8047F6FF7278
:107F30009342A8BF13462B803FF0FAFD94F86223CA
:107F4000B4F8603302992881002A33D0AB81E981EB
:107F50007FE4524FA7FB05756F094D4D6F80504F61
:107F60003870D6E70B6893F86C30002B3FF498AD6F
:107F7000D4F858325B053FF593ADDAE53F4B1B680B
:107F800093F869305B45BFF48BAD0223002284F87F
:107F9000D433444B5A60DA615A6343F8482F5A602D
:107FA0009A607DE5404D02611A462B6843F0040358
:107FB0002B605FE6642202FB03F33C4A82FB030270
:107FC0001A44DB17C3EB62239BB2BFE7D4F85432E9
:107FD00094F89C1183F48078DFF8DCE094F85EC2BA
:107FE000C8F30028DEF8003001EA080884F85D8252
:107FF0002F4833E6002356E4002F7FF4FAAC002B21
:108000007FF4F7ACD4F8E82332B1D4F8EC339B1A00
:10801000009A1344C4F8EC330023C4F8E8331F2D4E
:108020007FF43AAD4FF47A72D4F8EC33B3FBF2F349
:10803000174AD380002393802EE5DFED1E7A94ED5E
:10804000F77AB4EEE77AF1EE10FABFF6DEAC94ED13
:10805000F87AB4EEE77AF1EE10FABFF6D6AC94ED0A
:10806000F97AB4EEE77AF1EE10FAFFF6CBACCCE495
:10807000807E0120787E0120D4680120D85501201F
:1080800060E31600E4550120D34D6210085701202B
:108090000829012067666666CDCCCCCC1F85EB51E4
:1080A00024630120A8570020C8590120030820801C
:1080B0007C5901209A99193E641C0120C14BDB793F
:1080C000022B40F022812DE9F04FBF4CB4F8FC3375
:1080D000B4F8FE239A422DED028B83B018BFA4F8AA
:1080E000FE33B4F8003414BF0127002713F40063F3
:1080F00000F0228194F80484B8F1000F00F010829F
:10810000DFF8FC92DFF8FCA299F800609AED000A13
:108110004A2EB4F97C2400F04E81492E12D100235E
:10812000B4F810C4B4F812041946B4F832516CF320
:108130000F0362F30F0165F31F4360F31F41A34870
:10814000C0E90031B4F97E14DFF8BCB2531ADFED98
:10815000A06ADFEDA07A07EE103A9BF81C30B8EE6B
:10816000C77AA3F10503B3FA83F3B4EEE67A5B09A9
:1081700067EE277AF1EE10FA84F8143400F20881E1
:108180009FED957A77EE877A4A2EB0EEE78A934D87
:1081900008BF8E4BA4F81214C5ED057A85ED0A8A46
:1081A00004BF1A815981002F66D0D4F880344C2E38
:1081B0008B4907EE903A8B4A91ED000AF8EE677A08
:1081C0009FED897AD2F88800B4F8303130EE670A32
:1081D000C5ED017A67EE876AC1ED007AD2ED237AA8
:1081E000A86120EE270AB4F88E04C5ED026AA4F84F
:1081F000103485ED070A00F03F81A0B307EE903AF6
:1082000094F8A534F1EE005AD1ED116AF8EEE77A50
:10821000F5EEC06A77EEC07AF1EE10FAF0EEE77A8A
:1082200067EE877A07EE103AB8EEC77A87EE876A6C
:1082300036EE257AC5EE877AC5ED1A7A40F3878146
:10824000DFED6A7AB0EE007A66EEA77AC7FEC77AEB
:10825000B8F1040F05D1B0EE0C7A86FE476A76EECF
:10826000277AC5ED0B7A482E00F055814A2E03D1AE
:108270003FF05EFC554B1880F4F7CCFC9BF81C30AB
:10828000052B40F0C38094F8003113F0010200F098
:10829000D980D4F8A8245649821A8A4240F3D4825D
:1082A00003F0020394F83421C4F8A804002B94F9D5
:1082B000AE3414BF0021012184F8AC1414BF012195
:1082C0000021032A8CBF4FF0FF3201221344022BFE
:1082D0001A46A8BF0222012B22EAE27284F8AE24D9
:1082E00000F3BA82002384F8AD3484F87414B8F132
:1082F000080F33D8DFE818F057016A02CC01930168
:10830000F4012E012400270049013A4B03F17801C2
:1083100002E0063399420ED01A780A2AF9D19878E9
:10832000DA789042FFF4CFAE5A79002A7FF4CBAED0
:1083300006339942F0D17047984684F80434DFE65A
:10834000384615F0A9F82C4BD5ED167A93ED187A2E
:10835000B4EEE77AF1EE10FA00F3ED8099F8003010
:108360004A2B21D0242B09D1DFED1A7A95ED0C0A86
:1083700020EE270A3FF0DCFB144B188014F04CFF72
:10838000384603B0BDEC028BBDE8F04F14F042BD9F
:10839000DFED1A6AB4EEE67AF1EE10FAC4BF9FED93
:1083A0000E7A77EEC77AEFE695ED0E0A3FF0C0FB46
:1083B000064BD880E2E701923FF0BAFB034B019AEB
:1083C0009880BFE608570120BC7A012008290120C7
:1083D0000000E1C4CDCCCC3D0000B443C07E012000
:1083E000407F0120280401200AD7233C3EC3AE3938
:1083F0003F420F0014570120242400200000E144D4
:1084000005290120CC6C01202C5B0120002384F87D
:108410007434B8F1080FA1D801A353F828F000BFB5
:10842000A785010839880108918601081F8601087F
:10843000E186010855850108418301084783010849
:108440008B85010884F87424B8F1080F86D801A33D
:1084500053F828F0A7850108418801089186010892
:108460001F860108E186010855850108418301083E
:10847000478301088B850108FDEEC07ADFF830C321
:1084800017EE906AACF8086000283FF4F5AE07EEEE
:10849000903A94F8A534B1EE005ADFEDC36AF8EED5
:1084A000E77A91ED116AB5EEC06A77EEC07AF1EE27
:1084B00010FAF0EEE77A67EE877A07EE103AB8EE38
:1084C000C77AC7EE875A75EE854A65EEA67A85EEBD
:1084D000247AFDEEE77A17EE903AACF80A3085ED93
:1084E0001A7A40F3D3819FEDB17AF0EE007A26EE4E
:1084F000077A87FE677A67EE267AFDEEE77A17EE4F
:10850000903A1BB2B8F1040FACF80C3000F0C28105
:1085100085ED0B7AB0E63FF00BFBA54B9880ABE600
:108520000123404684F8043414F074FC14F074FE03
:1085300094F80484E4E59F4A0720136843F08053CD
:1085400013600AF0AFFA002384F8043406E7DFED85
:108550009A7A7DE694F8B0343846DFED936A07EEF8
:10856000903A9AED007AF8EEE77A67EEA67AF4EEA2
:10857000C77AF1EE10FAC1BF062384F80434002351
:1085800084F8543414F088FFE8E68A4A012013681E
:1085900043F0805313600AF085FA002384F85434C2
:1085A00084F80434DAE6237ADA0704D4834B1B7A9E
:1085B000002B00F08881D5ED0C7A9AED007AC7FE89
:1085C000277AC5ED0C7A002F3FF4C8AEB4F88C348E
:1085D000F6EE006A95ED026A05EE903AB4F8A03422
:1085E00026EE266A85ED0E7A06EE903A94F89B34D4
:1085F000F8EE655A012B86FE656A85ED136A00F078
:10860000A881F8EEE66A9FED686A022B66EE866A3C
:1086100000F0988177EEA67AC5ED0D7A9EE6B7EE6A
:10862000007AD5ED157AF4EEC77AF1EE10FA42BF72
:108630009FED637A77EE877AC5ED157AF3EE0E7AC1
:10864000B4EEE78AF1EE10FA0DD5B4F8883407EEEF
:10865000903A0423F8EE677A84F804340023C5EDD9
:10866000117A84F85434B4F88E3495ED077A07EE15
:10867000903A544B85ED107AF8EEE77AB4EEE77A4B
:10868000F1EE10FA4CBF0122002283F8912065E63A
:108690009AED007AD5ED0D7A4A4AF4EEC77A92F84F
:1086A0009020F1EE10FACCBF01230023934200F09A
:1086B000D8800023C5ED0E7A95ED027AEB63B4F80D
:1086C000963407EE903AF8EEE77AB4EEE77AF1EEF8
:1086D00010FAC4BF032384F80434EB692B643DE62D
:1086E000384AB7EE007AD5ED157A92F89130B4F8A1
:1086F0008E24F4EEC77A9FED346AF1EE10FA44BF8F
:108700009FED2F7A77EE877A95ED107A48BFC5ED09
:10871000157A07EE902AF8EEE77AF4EEC77AF1EED2
:1087200010FACCBF012200229A4202BF77EEC77A2C
:10873000DFED236AA7EEA67AD5ED1B7AF7EE006A85
:1087400076EEE76A08BF85ED107AB0EE007AE6EEC5
:10875000867A37EE677AC5ED1B7A85ED197A002F98
:108760003FF4FCADB4F88834B6EE007AD5ED025A89
:1087700006EE903A95ED136AF8EE666AF4EEC65A84
:1087800026EE877AC5ED116AF1EE10FA67EE277AC8
:10879000C5ED127A3FF6E2AD052384F804340023D8
:1087A00084F85434DAE500BF0000C8423EC3AE3955
:1087B00008290120C8590120000000007856012036
:1087C0000AD7233C280401200AD7A33BF1EE047A00
:1087D00095ED027ADAED006AB4EEE77AF1EE10FA7E
:1087E00074D4B4F8963407EE903AF8EEE77AB4EE23
:1087F000E77AF1EE10FA00F18880D5ED0D7A0023CA
:10880000F4EEE67A594A84F854340023F1EE10FA73
:108810006B65AB646B64EB66EB634FF07E536B662A
:10882000AB66EB692B64CCBF0123002382F8903048
:10883000022384F8043491E594F80031DB07C5D4B1
:10884000072384F8053489E594F8AC343BB994F8EF
:10885000AD1481F0010148E5012384F8AD34002115
:1088600043E5002B46D0B4F89C349FED417A07EEE7
:10887000903AF8EEE77A67EE877A95ED0E7AC5EDD5
:108880000F7A77EE277AC5ED0E7A26E79FED397AD3
:10889000002337E6F0EE0C7A0192C5FEE77A77EE18
:1088A000877AC5ED0B7AF4F7B5F99BF81C30019A7D
:1088B000052B43D194F8003113F001017FF4E9ACAA
:1088C00084F874140DE700232B6347E594F8B03463
:1088D0009FED296A07EE903AF8EEE77A67EE867A1E
:1088E000F4EEE67AF1EE10FA7FF77BAF082384F816
:1088F000043433E5B4F89E349FED207A07EE903AC5
:10890000F8EEE77A67EE877AB7E7B4F8A034B6EE08
:10891000007A9FED195A06EE103ADFED195A67EE0C
:10892000877AB8EEC66AB0EE667AC5ED137AA6EE1F
:10893000057AC7FE257AC5ED0D7A60E7002384F835
:108940007434CEE676EE877AC7FEA67AC5ED0D7A48
:1089500004E5B4F88A349FED087A07EE903AF8EE11
:10896000E77A67EE877AC5ED0D7AF7E428040120EF
:108970000AD7233C000000000000C8420AD723BCED
:1089800000007A442DE9F8439A4B1B685A0701D43A
:10899000BDE8F883DFF8A0820446974F98F80030CE
:1089A00097F89250372B954E04BF954B1D80736BF3
:1089B0001A78012A07D0042D00F21081DFE805F0B3
:1089C00093B7A0AB180093F904308E4A03EB43032E
:1089D00002EB431393F85520202A00F0C2800123B4
:1089E00089488A494FF47A7280F820300B7074E01D
:1089F000D6F8EC3086489847002800F0B8808549C2
:108A0000D6F8F030081D9847D6F8FC90B9F1000F61
:108A100040F3BD8007EE909A9FED7F0ADFED7F0A5D
:108A2000F8EEE77A27EE800A3EF076FFF7EE007A5E
:108A30007B499FED7C7A77EEC07A7B4A087867EEB7
:108A4000877A92ED007A002800F0AA8077EEC77A44
:108A5000C6ED3D7A98F80030372B17D107EE909A83
:108A60009FED720ADFF89881F8EEE77A27EE800A28
:108A70003FF05EF8D6F8F83096ED3D0AA8F802000F
:108A8000A8F804303FF054F8A8F8060096F8D03063
:108A9000002B51D105234FF47A7887F892301F4686
:108AA000594B012206EB850583F82020F4F7B2F834
:108AB000D5F8CC34001B984206EB870388BFC5F875
:108AC000CC04D3F8CC0440F00FF8B8F1000F3FF419
:108AD0005FAF42460A2AB8BF0A22554B1B681B6883
:108AE0001A61BDE8F883D6F8DC3049489847002879
:108AF0003DD001234FF47A7887F892301F46CFE7B4
:108B0000D6F8E430424898470323B6F8D48087F873
:108B100092301F46C4E7D6F8E8303D48984730B356
:108B200004234FF47A7887F892301F46B8E7D6F8D6
:108B3000E03037489847D0B1022387F8923006EBEF
:108B40008505F4F767F8001BD5F8CC34834219D2B9
:108B5000C5F8CC04D6F8D4043FF0C6FF4FF47A78B9
:108B6000B7E75B699B691B047FF525AF37E797F88B
:108B700092300121254A022B1170E0D01F464FF49C
:108B80007A788DE7D6F8D4043FF0AEFFE6E7244BC1
:108B90001B78002B7FF45EAF0023C6F8F43059E752
:108BA000DFF898C077EE877A224BB3F800E0BCF884
:108BB0000030C2ED007A01339BB29E45ACF8003024
:108BC000EAD807EE103A0123ACF80000B8EEC77AF5
:108BD0000B70C7EE876AC2ED006ADDE7D6F8D830C1
:108BE0000B4898470023B6F8D28087F892301F468A
:108BF00056E700BF285B012028040120BC7A012031
:108C0000082901207C2101209453002020240020E9
:108C1000F07A0120B47B012008942537B1DC423E74
:108C200028690120D048874A246901200AD7233CBB
:108C3000905300202A690120052901202C69012078
:108C4000F8B5384C2368002B57D00A2801D00D28DE
:108C500051D1354D95F8E4340BB1F8F7CBF8334EDC
:108C6000232130463FF0D9FC08B1801B20602368E7
:108C7000002273B902B12360F8F788F895F8E4345C
:108C8000F3B12B48BDE8F840F8F7ACB801220B4629
:108C9000EFE7591E705C2028F8D092B90022254CCD
:108CA000224FF2543C26013E0DD13146224B9C42CC
:108CB00012D2E3682068984795F8E534002BDBD1A1
:108CC000F8BD2360EAE721683846FCF7B3FE0146A9
:108CD0000028EBD11034E6E795F8E43423B11749C6
:108CE0001748F8F7A5FDC7E71648F8F77BF80F48CF
:108CF000F8F798F8C0E7FF2BE2D8A0F120025E2A2F
:108D0000DED80BB92028DBD05A1C2260074AD05489
:108D1000054B93F8E434002BD2D0BDE8F840F8F7C7
:108D2000ABB800BFEC5A0120BC7A0120EA590120FF
:108D300092820608E0D6050890DA05080F9C06081E
:108D40002B9C0608319C060838B50546F8F72EF826
:108D50000A4B0024186804F089FCF8F717F8084B50
:108D600083F8E54483F8E44419F0AEF825B12046D1
:108D7000BDE83840FCF77BBE38BD00BF246401204D
:108D8000BC7A012038B5074C074DAC4203D3074BE2
:108D900001221A7038BDA288D4E902103FF030FBDE
:108DA0001C34F2E7A0E50608D0EE0608FC500120CE
:108DB0002DE9F04F0E4693B083469F493046174643
:108DC000FCF738FE0546002840F01F819B493046DD
:108DD000FCF730FE0546002840F0198198493046DE
:108DE000FCF728FE0546002840F0138195493046DF
:108DF000FCF720FE0546002840F00D8192493046E0
:108E0000FCF718FE002805460ABF01240824354651
:108E10007F428E49284607F010073C43FCF70AFEC4
:108E2000002800F0FA8044F02004894B1B780BB92D
:108E3000FFF7A8FF31F0B4FF14F0090F00F05483DE
:108E40008448F7F7F5FF0020FCF71EFF14F4807349
:108E5000049340F0EC808048F7F7EAFF7F48F7F78B
:108E6000E1FF04F01803182B05D17D48F7F7E0FF68
:108E70007C48F7F7D7FF01230393F7F7BBFF7A4945
:108E80007A48F8F765F87A497A48F8F761F804F40F
:108E90008473082B07D178495846F8F72DF976499D
:108EA0005846F8F7FBFE14F0800307930ED1734B7E
:108EB000204693F8E82403F59D63002A704A06BF14
:108EC0000121134600216F4AF7F798FF6E492046AB
:108ED000FCF71CFF6D492046FDF7B2FA6C492046AD
:108EE000FDF7C0F96B4B14F01006D3F800A06A4BE5
:108EF0001D6840F09E806948F7F79AFF0296684B1C
:108F00004FF00008CDE905336AEA05030993069B93
:108F100053F8049B0693B9F1000F21D00127099B58
:108F2000029A204607FA08F73B400CBF01210021B6
:108F30000893F9F753FD65EA0A035A4A029020465E
:108F40003B424B4614BF01210021F7F79FFF0899D0
:108F50004B46544A0039204618BF0121F7F74EFF0F
:108F600008F10108B8F11D0FD1D165EA0A034FF0ED
:108F700000080693059B53F8049B0593B9F1000F75
:108F800024D0012707FA08F73D420AD06AEA050310
:108F9000454A20463B424B4614BF01210021F7F7CA
:108FA00075FF1AEA070F11D0069B2046029A1F4050
:108FB0000CBF01210021F9F711FD391E02904B462B
:108FC000394A18BF01212046F7F718FF08F10108B8
:108FD000B8F11D0FCED1354B2046354A3549FAF749
:108FE000ADFE079B002B6DD0134B2246182158462F
:108FF000F9F724FD039B002B00F0C9812E48F7F7F9
:1090000017FF2E48F7F70EFFC1E1012400E7022405
:10901000FEE60424FCE68124FAE629492846FCF70A
:1090200009FD00283FF401AF44F48074FDE60023FD
:1090300022E71A4B029362E75D9C0608649C0608CF
:109040006C9C0608729C06087B9C06085D980608C6
:10905000FC5001204E8C0608849C06089C9C060847
:10906000A89C0608D09C0608F78806083C890608D4
:109070004A8906085F89060810A90608BC7A0120FB
:10908000C7A20608E09C0608ED9C0608F79C0608A7
:1090900027850608E0790120745601203E9C0608C9
:1090A000FCA30508FD9C0608099D0608149D0608FA
:1090B000185601206C770120D89D0608EE9D060801
:1090C0007F9C0608DFF8C4932046DFF8C4A399F814
:1090D00000209AF80030DFF8BC839A42B34A13BFED
:1090E0000121002101270027F9F778FC9AF80030C8
:1090F00039460546013BAE4A204658F82330F7F77B
:10910000C5FE99F800303946AA4F013BA84A2046CF
:1091100058F82330F7F772FED7ED007AA64A2046BA
:10912000F5EE407AF1EE10FA0CBF01210021F7F7BD
:1091300065FE2B463A46A1492046FBF77FF8A04B37
:10914000A04A2046A049FBF7A7FC2EB19F4B93F9FC
:109150000230002B00F021819D48F7F769FE9D4801
:10916000F7F760FE0023994A20469B49FBF7C8FDAC
:109170009A4B9B4A20469B4F9B4D019300923A6825
:109180002968FCF701FC40F20222984B204600922D
:109190000193BA68A968FCF7F7FB002E40F0FF8046
:1091A0009348F7F745FE3246924F01259248002139
:1091B000DFF8E4C217F8013B10F8018B03F1480E09
:1091C000EE440EF8208C1CF801EB0EF14809E9443E
:1091D00009F8108C002D00F0E480A3EB0E056B4223
:1091E0006B4101311D460829E4D1002783F00101BC
:1091F00020468DF83070F9F7F1FB0EAB7F4A294617
:1092000020468DF84070F7F741FE0AAB7B4A2946AD
:109210002046F7F7F3FD7A4B7A4A20467A49FBF766
:109220003BFA7A4B7A4A20467A49FBF7C1FA7A4BE5
:10923000744A20467449FBF74DFB784B784A204628
:109240007849FAF739FC784B784A20467849FAF79A
:10925000C1FE784B784A20467849FBF75DF9784B98
:10926000784A20467849FCF743F8784B784A2046FC
:109270007849FBF721FF002E40F095807648F7F7FC
:10928000D7FD0296754E0025754FDFF810823946DE
:10929000022230463FF080F9002896F800A02046D0
:1092A00014BF01210021029A0CBF4FF001094FF0B9
:1092B0000009F9F793FBBAF1020F029040F0F08039
:1092C0007B784FF0190A40F2EE22494620461AFBFD
:1092D0000323644A01933B7818F8033000932B462C
:1092E000F7F7D4FD737840F2EE22494620461AFB88
:1092F00003235C4A0193337818F8033000932B461C
:10930000F7F77CFD013502360237122DBFD100215F
:10931000554B22465846F9F791FB210740F1D8807A
:109320000025E9B2013522465846FCF765FC042DBC
:10933000F7D14E4E4E4D33782B70049B33B94D48C8
:10934000F7F776FD4C495846FAF74AF9FF232B7098
:109350000025E9B2013522465846FCF771FC042D80
:10936000F7D17378454C2370049B002B40F0AD80FF
:109370004348F7F75DFD40495846FAF761F941481F
:10938000F7F756FD4048F7F72DFDFF232370002027
:1093900013B0BDE8F04FF9F72EBB0D4BE3E6144ACE
:1093A00002E72B461DE72C4B02936BE74C9C06080B
:1093B0001B9D0608E0650120249D0608D477012046
:1093C000C295060860670120DC6D0120C06701209E
:1093D000469C0608339D0608686D0120409D0608DE
:1093E000FFFF7F00AC570120047A0120479D06084B
:1093F000529C060894780120601E0608DC9006083E
:10940000FD89060870660120406E0120539D060804
:10941000F0660120C06E01204E9D0608599D060889
:1094200014570120AC7201205D9D0608B464012030
:10943000486F0120669D060860660120346F012098
:109440006E9D06083858012038710120779D060866
:1094500030680120E0780120569C060878700120D1
:109460006C640120FC9006085D9C0608CC78012005
:10947000780301207B9D060810A9060879030120C6
:109480009E9D0608C59D0608DB9C0608F87901200C
:10949000DC550120A4A40508E4550120E4200608B9
:1094A0003B7849461A4A204618F8033000932B4669
:1094B000F7F7ECFC3378164A494618F80330204693
:1094C00000932B46F7F79AFC1CE7FF23237091E5E6
:1094D000104D224658462978FCF78EFB22466978C3
:1094E0005846FCF7ADFB85E5A20706D5094B224699
:1094F00058461978FCF780FB49E763077FF547AFCB
:10950000044B224658465978FCF79AFB3FE700BFC8
:109510000C910608CC780120002249E4012247E49E
:109520002B4B30B583B09A790190BAB393F82420CD
:10953000DFED286A07EE902ADB79274CF8EEE77A10
:10954000A3F10203254904F58D62B3FA83F386EE95
:10955000A77A0D785B0984F86C3482ED007ADDB16E
:109560001F4BDDED017AB3F8E235F8EE677ADFEDF7
:109570001D0A00EE103A67EEA00AB8EE400AF5F7B1
:1095800061FC04F58E63002103EBC502196008330A
:1095900003ED010A9A42F9D103B030BD124A1268B4
:1095A0001401F9D593F82420DFED0A6A07EE902A1A
:1095B000DB79094AF8EEE77A981E02F58D6143429D
:1095C00086EEA77A434182F86C3481ED007AE3E7B6
:1095D0001C2801205555554094530020A007002019
:1095E000BC7A0120BD378635C8560120894B1B78CF
:1095F000002B00F0E680884B2DE9F04F2DED028B1B
:1096000093F804A183B0BAF1010F40F09380834B2B
:109610001C78082CA446A8BF4FF0080C002C61D081
:109620007F480021DFED7F7A40F6FF7E00F58D63F5
:10963000794A90F86C748B46D3ED006A7A4D66EEE9
:10964000A76A0091CDF804A0938927B992F81E80EB
:10965000B8F1010F09D913F4706F4FEA2329C3F34E
:10966000032802D019F0010F69D0734500F08980FA
:10967000C3F308085B0A08FA03F31FFA83F8B8F18A
:10968000000F00F09280694E9BB206EB5808B8FBC1
:10969000F3F35FFA81F8444507D9DFF8A08198F821
:1096A0000080B8F12D0F08BF2B804FF6FF76B34234
:1096B00040F0888001311432043002358C45C3D12A
:1096C000BBF1000F0ED0DDED007A594BB8EE677A92
:1096D00007EE90BAF8EE677A27EE267AC7EE276A89
:1096E000C3ED006ADFF85C919FED528A89ED008A34
:1096F000E4B159ED138A09F10408474F0025A9F197
:10970000440AFB890AEBC5000135143700EE103A14
:10971000B8EEC00A20EE280A3FF012FAAC4288FEEA
:10972000408AA8EC010A89ED008AEAD102233A4A6C
:1097300082F8043103B0BDEC028BBDE8F08F3E4EE1
:1097400001EB81095FFA83FA06EB5808324E98F86C
:10975000C08308EB4909B8F1010F06EB4909019EE6
:10976000A9F80EA006FA08F692F81E9049EA060932
:1097700082F81E9040D192F81F80C2459AD9D377C3
:1097800098E7CBB29C422CD92C4B1B782D2B30D098
:109790000023DFED2B7AD381937F43F0010393778E
:1097A0000BF1010BC0ED007A84E7CBB29C4281D96A
:1097B000224B1B782D2B7FF47DAF4FF6FF732B8050
:1097C00078E77047009E07EE903A1E449BB2F8EE91
:1097D000E77AD381937F67EEA67A009643F0010380
:1097E000DDE70023DFED167AD381937F43F0010399
:1097F000D5E700232B80CBE7B8F1000F7FF45AAFF9
:1098000007EE90AA009BF8EEE77A5344009367EEC8
:10981000A67AC5E7A8010020081D0020A0070020A7
:10982000945300200000704208290120C02709003D
:1098300044580020FFFF7F7FE0D60508052901205E
:109840000000000048580020F0B41A4C1A4BA4FB4A
:10985000024290F858505209A3FB0243DB0803EB85
:109860008303A2EB43030268DCB2A54220D000EBE5
:10987000830C476800269B00DCF80850521BDCF87C
:1098800030507D1B4560CCF80860CCF8306080F823
:1098900058400344013202609A6801329A6029B943
:1098A0004268013242601A6B01321A63F0BC7047A1
:1098B0009B00EEE71F85EB51CDCCCCCC38B5094DE4
:1098C0002B7963B100242B6820465B6B13B1013404
:1098D000984708B9002038BD2B799C42F3D301206A
:1098E00038BD00BF342500200C4B93F8982012B9E6
:1098F0000B4B987970470A4A906800B9704709493C
:1099000040F6B83C0968091A614504DD00219079E8
:1099100083F8981070470020F0E700BF280401206A
:1099200034250020641C01202DE9F04FDFF834922B
:109930001F46531E83B016460546D9F80040142B27
:1099400000F2CD80DFE803F05959595959CB0B0B80
:109950000B0BCB0B0B0BCBCBCBCBCB0B0B004FF4B5
:109960007A734FF00A0A0193012F4CD0002F41D196
:10997000774A784B14781878631C03F0030383420A
:1099800038D0137004EB4403DFF8D4814FF47A72BB
:109990004FEA440908EBC30383F80CA09A60C1B1F5
:1099A0001822A5F1FF0002FB0482B0FA80F00C320D
:1099B000400905E038B9013702F8013F8F4208D06D
:1099C000AF420346F6D1013733468F4202F8013FDA
:1099D000F6D1FFF773FF002800F0A98009EB04011E
:1099E000012342F21070C90008F8013041443FF0F1
:1099F00073F8486003B0BDE8F08F574B012F4FF06C
:109A0000010A0193B2D1554A537C012B03D0022B9A
:109A100000F09880002799F8040008B34D4B1821F6
